:020000040800F2
:1080000010C00020498100083D9A0008959400089E
:1080100025990008CB8F000823AC00080000000061
:1080200000000000000000000000000041A1000866
:10803000E390000800000000F59E0008BDA10008C4
:108040006381000863810008638100086381000880
:108050006381000863810008638100086381000870
:108060006381000863810008638100086381000860
:108070006381000863810008638100086381000850
:108080006381000863810008638100086381000840
:108090009FA300086381000863810008F79100082E
:1080A0006381000863810008638100086381000820
:1080B00035A20008DDA2000889A30008638100083A
:1080C0006381000863810008638100086381000800
:1080D00063810008638100086381000863810008F0
:1080E00063810008638100086381000863810008E0
:1080F00063810008638100086381000863810008D0
:1081000063810008638100086381000863810008BF
:1081100063810008638100086381000863810008AF
:10812000638100086381000863810008638100089F
:10813000DFF810D000F06CF80048004711F8000894
:10814000AFF3008010C00020064880470648004773
:10815000FEE7FEE7FEE7FEE7FEE7FEE7FEE7FEE7F7
:10816000FEE7FEE7C5A10008318100080649074A7D
:108170000868504343F239021044086040087047D1
:108180000149086070470000900600206D4EC6410E
:1081900010B5431A934209D28318881803E010F8E7
:1081A000011D03F8011D521EF9D210BD40EA010362
:1081B0009B0703D009E008C9121F08C0042AFAD29D
:1081C00003E011F8013B00F8013B521EF9D210BD4B
:1081D000D2B201E000F8012B491EFBD27047002209
:1081E000F6E710B513460A4604461946FFF7F0FFB6
:1081F000204610BD30B504460020034600E05B1C5D
:10820000934203D2E05CCD5C401BF8D030BD00004F
:10821000064C074D06E0E06840F0010394E80700D3
:1082200098471034AC42F6D3FFF786FF8C5801080C
:10823000AC58010870B58C1810F8015B15F00703F5
:1082400001D110F8013B2A1106D110F8012B03E0EF
:1082500010F8016B01F8016B5B1EF9D12B0705D4F7
:108260000023521E0DD401F8013BFAE710F8013B40
:10827000CB1A921C03E013F8015B01F8015B521E5C
:10828000F9D5A142D8D3002070BD00002DE9F041FE
:1082900007460C4615461E461EB980200B4908604D
:1082A00003E04FF4807009490860102229462046F7
:1082B00005F054FB8046102241463846FFF768FF20
:1082C000404606F0C7F9BDE8F081000048060020EE
:1082D0002DE9F04784B01F46DDF830A0914688466E
:1082E000060018BFB8F1000F4AD0002F18BFBAF12E
:1082F000000F45D0B9F1000FA8BF19F00F0F1EBF36
:1083000040F61D4004B0BDE8F087307910F0020F50
:108310001EBF40F61E4004B0BDE8F0870024B9F14E
:10832000100FA8BF6D4625DB5FF0000004EB800155
:1083300058F8011009BA45F82010401C0428F5DB54
:108340006846014606F12802736A00F0BFF84FF054
:10835000000C00BF55F82C0004EB8C0100BA0CF1A6
:10836000010C7850BCF1040FF4DB04F12000103450
:108370004845D9DDCAF8004004B00020BDE8F087C8
:1083800004B04FF44260BDE8F087002812BF002A15
:108390004FF442607047017941F002010171002001
:1083A00010607047032300F04BBD00002DE9F0473B
:1083B00084B01F46DDF830A091468846060018BFFD
:1083C000B8F1000F4AD0002F18BFBAF1000F45D006
:1083D000B9F1000FA8BF19F00F0F1EBF40F61D40E6
:1083E00004B0BDE8F087307910F0020F1EBF40F6F0
:1083F0001E4004B0BDE8F0870024B9F1100FA8BFFB
:108400006D4625DB5FF0000004EB800158F8011099
:1084100009BA45F82010401C0428F5DB68460146DF
:1084200006F12802736A00F0DFF94FF0000C00BF7C
:1084300055F82C0004EB8C0100BA0CF1010C7850BB
:10844000BCF1040FF4DB04F1200010344845D9DD01
:10845000CAF8004004B00020BDE8F08704B04FF433
:108460004260BDE8F087002812BF002A4FF4426046
:108470007047017941F002010171002010607047DE
:10848000022300F0DDBC00002DE9F04180460C46DF
:1084900015461E4600271EB980200B49086003E0E0
:1084A0004FF48070084908602946404605F012FDE7
:1084B0000746102239462046FFF76AFE384606F086
:1084C000C9F8BDE8F0810000480600202DE9F80F4A
:1084D0004FF0030C0CEBE308DB1002EB431202F14C
:1084E0006003BE4A4FF0010CC2F808C0D2F808C0C1
:1084F000D2F800C0CDF800C0BCF1FF3F08D1DDF8D4
:1085000000C0C2F800C012680092002A00F0E680A5
:108510004268D3F804C0006882EA0C071A68424037
:1085200094466446AE483D0E02F0FF0A50F82560BE
:10853000C4F3074550F82AA050F8255004F0FF0B6B
:1085400086EA3526C2F3072550F82BB050F825509F
:10855000A8F101084FEA35490CF0FF0550F8255005
:1085600089EA3565754053F8106CC7F307496E40CA
:108570004FEA1C6550F8299050F8255085EA3925B6
:10858000C4F30729240E50F8299050F824404FEAEC
:10859000394989EA3A6985EA090953F80C5CCCF350
:1085A000074A89EA05054FEA1269C2F30742CCF38C
:1085B000072C50F8299050F82AA050F8222050F8A3
:1085C0002CC089EA3A2984EA3222C7F3072A4FEA03
:1085D0003C4407F0FF0C50F82AA050F82CC04FEA9A
:1085E0003A4A8AEA3B6A84EA3C6C89EA0A0982EAE6
:1085F0000C0253F808AC53F804CC203B89EA0A0972
:1086000082EA0C04B8F1000F7ADD320EC4F3074C95
:1086100050F8222050F82CC0EFB282EA3C22C9F375
:10862000072C50F8277050F82CC009F0FF0A4FEAC9
:108630003C4C8CEA376C82EA0C02D3F800C050F84C
:108640002AA082EA0C072A0E04F0FF0B50F822C081
:10865000C6F3074250F82BB050F822208CEA322C97
:10866000C4F30722240E50F8222050F824404FEA89
:10867000324282EA3A628CEA0202D3F804C0C5F3BD
:10868000074A82EA0C0C4FEA196250F82AA050F807
:108690002220C5F3072582EA3A22C6F3072AC9F346
:1086A0000749F6B250F82AA050F8255050F8299002
:1086B00050F826604FEA3A4A4FEA35458AEA3B6A63
:1086C00084EA392485EA366582EA0A026C40D3F8E6
:1086D00008A0DD6882EA0A026C4024E70268D3F849
:1086E00000C09C6882EA0C074268D3F804C082EAA2
:1086F0000C0C8268C0686240DC68444012E7FFE707
:10870000384850FA85F200EB166C12789CF800C0DD
:10871000C9F3072742EA0C62C4F3074CC75D10F89F
:108720000CC04FEA0C4C4CEA072C42EA0C02D3F87E
:1087300000C082EA0C020A6050FA89F200EB156C64
:1087400012789CF800C0C4F3072742EA0C62C6F313
:10875000074CC75D10F80CC04FEA0C4C4CEA072CD4
:1087600042EA0C02D3F804C082EA0C024A6050FAD2
:1087700084F200EB196C12789CF800C0C6F307274E
:1087800042EA0C62C5F3074CC75D10F80CC04FEA13
:108790000C4C4CEA072C42EA0C02D3F808C082EADF
:1087A0000C028A6050FA86F200EB146C12789CF886
:1087B00000C0C5F3072442EA0C62C9F3074C10F865
:1087C0000CC0005D4FEA0C4C4CEA00201043DA6804
:1087D0005040C860BDE8F80F70470000003002400C
:1087E000544301082C3E01082DE9F80F4FF0030C0B
:1087F0000CEBE308C24B4FF0010CC3F808C0D3F8F0
:1088000008C0D3F800C0CDF800C0BCF1FF3F00F0B5
:10881000E5804368D2F804C0006883EA0C07136857
:1088200080EA0304A4466346B6483D0ECCF30746EF
:1088300050F8255050F8266004F0FF0985EA3625E7
:10884000C3F3072650F8299050F8266007F0FF0A76
:108850004FEA364686EA396675401669C3F307491A
:108860006E404FEA1C6550F8299050F8255050F89A
:108870002AA085EA3925C4F307290CF0FF0B50F82C
:108880002990CCF3072C4FEA394989EA3A6985EAFD
:108890000905D2F81490C4F3074A85EA09054FEA9E
:1088A000136950F82AA050F82990240E89EA3A2931
:1088B000C7F3072AC7F30747DBB250F82AA050F8DE
:1088C0002CC050F82BB050F8244050F8277050F8C6
:1088D00023304FEA3A4A4FEA3C4C8AEA3B6A84EA40
:1088E00037248CEA336389EA0A0984EA030CD2F854
:1088F00018A0D3692032A8F1010889EA0A098CEA94
:108900000304B8F1000F7CDD330EC5F3074C50F8BB
:10891000233050F82CC0E7B283EA3C23C9F3072C7C
:1089200050F8277050F82CC006F0FF0A4FEA3C4C74
:108930008CEA376C83EA0C03D2F800C050F82AA006
:1089400083EA0C072B0EC9F3074C50F8233050F87C
:108950002CC005F0FF0B83EA3C23C4F3072CC5F3BE
:10896000072550F82CC050F825504FEA3C4C8CEAB3
:108970003A6C83EA0C03D2F804C0C4F3074A83EAD2
:108980000C0C4FEA196350F82AA050F82330240E3B
:1089900083EA3A23C6F3072AC6F3074650F8244071
:1089A00050F8266050F82AA084EA362409F0FF0621
:1089B00050F82BB050F826604FEA3A4A4FEA354556
:1089C0008AEA3B6A85EA366583EA0A036C40D2F894
:1089D00008A0D56883EA0A036C4026E7DDF800C0EA
:1089E000C3F800C01B68009363B14368D2F804C0A9
:1089F000006883EA0C07136880EA030C6346644648
:108A000012E710E00368D2F800C0946883EA0C070C
:108A10004368D2F804C083EA0C0C8368C0686340E2
:108A2000D468444000E7384850FA84F300EB166CF1
:108A30001B789CF800C0C9F3072743EA0C63C5F311
:108A4000074CC75D10F80CC04FEA0C4C4CEA072CE1
:108A500043EA0C03D2F800C083EA0C030B6050FA1F
:108A600086F300EB156C1B789CF800C0C4F3072755
:108A700043EA0C63C9F3074CC75D10F80CC04FEA1A
:108A80000C4C4CEA072C43EA0C03D2F804C083EAEE
:108A90000C034B6050FA85F300EB196C1B789CF8C3
:108AA00000C0C6F3072743EA0C63C4F3074CC75D55
:108AB00010F80CC04FEA0C4C4CEA072C43EA0C03AC
:108AC000D2F808C083EA0C038B6050FA89F300EBFC
:108AD000146C1B789CF800C0C5F3072443EA0C63B0
:108AE000C6F3074CD26810F80CC0005D4FEA0C4C7E
:108AF0004CEA002018435040C860BDE8F80F7047AA
:108B000000300240543F01082C3D010870B50C466E
:108B10008446002315462046B3EBA20F09DA00BFB6
:108B20005CF8231009BA40F823105B1CB3EBA20FCA
:108B3000F6DB214600F096F8E910052000EB410332
:108B4000002BD8BF70BD04F11002454800F5C56187
:108B5000D2F800C000EB1C64CCF307452478455DD7
:108B600051F8244051F8255084EA3524CCF30725E8
:108B7000455D51F825504FEA354550FA8CFC9CF87C
:108B800000C051F82CC085EA3C6C84EA0C0C42F819
:108B900004CB52F804CB00EB1C64CCF307452478DB
:108BA000455D51F8244051F8255084EA3524CCF332
:108BB0000725455D51F825504FEA354550FA8CFCA4
:108BC0009CF800C051F82CC085EA3C6C84EA0C0C7F
:108BD00042F804CC52F808CB00EB1C64CCF30745F8
:108BE0002478455D51F8244051F8255084EA352415
:108BF000CCF30725455D51F825504FEA354550FA2D
:108C00008CFC9CF800C051F82CC085EA3C6C84EACE
:108C10000C0C42F808CC52F804CC00EB1C64CCF3EA
:108C200007452478455D51F8244051F8255084EAE1
:108C30003524CCF30725455D51F825504FEA3545DD
:108C400050FA8CFC9CF800C05B1E51F82CC085EAE1
:108C50003C6C84EA0C0C42F804CC7FF479AF70BD14
:108C60002C3D010870B400239510002D15DDA0F1F6
:108C7000040C081F12F0040F03D05CF8044F40F8F6
:108C8000044FD21009D000BFDCF8044044605CF807
:108C9000084F40F8084F521EF6D1684C042DA4F539
:108CA000007005D0062D34D0082D6DD070BC7047F3
:108CB000CA6800EB126CC2F307459CF800C0455D22
:108CC0004CEA056CC2F30725455D2D0450FA82F687
:108CD000367845EA06254CEA050C54F823600D6801
:108CE0005B1C75408CEA050CC1F810C04D680A2B5E
:108CF0008CEA050CC1F814C08D688CEA050C8CEA6E
:108D00000202C1F818C0CA61B8BF1031D0DB70BC14
:108D100070474A6900EB126CC2F307459CF800C02B
:108D2000455D4CEA056CC2F30725455D2D0450FAFC
:108D300082F6367845EA06254CEA050C54F823609D
:108D40000D685B1C75408CEA050CC1F818C04D68B5
:108D5000082B8CEA050CC1F81CC08D688CEA050C48
:108D6000C1F820C0CD688CEA050CC1F824C0A4BFAE
:108D700070BC70470D698CEA050C8CEA0202C1F8E0
:108D800028C0CA621831C4E7CA6900EB126CC2F38A
:108D900007459CF800C0455D4CEA056CC2F3072509
:108DA000455D2D0450FA82F6367845EA06254CEAF0
:108DB000050C54F823600D685B1C75408CEA050CAB
:108DC000C1F820C04D68072B8CEA050CC1F824C0FF
:108DD0008D688CEA050CC1F828C0CD688CEA050CBA
:108DE000C1F82CC0A4BF70BC704750FA8CF52D7828
:108DF00000EB1C66367845EA0665CCF30746CCF3F3
:108E0000072C865D10F80CC0360446EA0C2C45EAA7
:108E10000C0C0D698CEA050CC1F830C04D698CEA68
:108E2000050CC1F834C08D698CEA050C8CEA02028D
:108E3000C1F838C0CA632031A6E700002C3F010802
:108E40002DE9F0410E46002818BF002E04D003F093
:108E500006012AB9022903D04FF44260BDE8F0812F
:108E6000D0F824C0BCF1100F1CBFBCF1180FBCF12E
:108E7000200F08D102290AD0D0F810C0ACF1010CA3
:108E8000BCF1100F03D340F61F40BDE8F081C26073
:108E900090F804C002292CF0060C80F804C048D0D9
:108EA000002141618161C1610162D0F810C0BCF153
:108EB000000F3EDD1CF0010F4FF01804A2F101027B
:108EC00004D012F8011F0906416101215FEA6C0C10
:108ED0002FD0CF1701EB977727F00307CF1B5578DB
:108EE0007F4204EBC70705FA07F721F003050544A5
:108EF000D5F8148047EA08076F614D1C4FEAE57802
:108F000005EB987828F00308A5EB080512F8027F16
:108F10006D4204EBC505AF404D1C25F0030505442B
:108F2000891CD5F81480BCF1010C47EA08076F6171
:108F3000CFD1017911F0010F0DD113F0010F86602F
:108F40001CBF062131EA030108D000F12801426A62
:108F50003046FFF7DBFD0020BDE8F08100F128017D
:108F6000426A0020B0EBA20F09DA00BF56F82030A9
:108F70001BBA41F82030401CB0EBA20FF6DB0846CC
:108F8000FFF770FEE7E7000030B50246130100204E
:108F900013E000210EE00A4C1C4404EB8004645CE6
:108FA000084D05EB81052D5C6C40064D05EB8105F8
:108FB0002C54491C0429EEDB401C0428E9DB30BD9D
:108FC000C1AA0020B1AA0020704700BFFEE772B618
:108FD0007047000070B5002600240DE0002508E071
:108FE00005EB84001C49085C1C4901EB8501085510
:108FF0006D1C042DF4DB641C042CEFDB0020FFF758
:10900000C3FF012609E001F0BFF801F09BF800F072
:109010008BFC3046FFF7B8FF761C1148006886428B
:10902000F1DB01F0B1F801F08DF80D480068FFF7B1
:10903000ABFF00240DE0002508E0084800EB8500A8
:10904000005D05EB8401074A50546D1C042DF4DBD0
:10905000641C042CEFDB70BD81AA0020B1AA0020A3
:109060004006002091AA0020024600210AE00F4B92
:1090700013F81100904203D14800401C185C70475F
:10908000481CC1B21229F2DB00210AE04800401C52
:10909000064B185C904202D113F81100EFE7481C10
:1090A000C1B21229F2DB0020E9E70000DE39010835
:1090B00030B591B004460D46402101A8FFF78FF866
:1090C00094208DF804000B208DF805002A462146D7
:1090D0000DF10600FFF75CF801A80AF00DF911B0D8
:1090E00030BD7047FEB506460C4617461D46022D9C
:1090F00001D1012500E000250A484078012809D166
:1091000002A823463A461021CDE90005304600F07A
:10911000A3FF05E02B463A4631462046FFF7B6F856
:10912000FEBD0000384B002010B504460A2001F0B7
:10913000C5FF10BD2DE9F04104460E46174605F067
:10914000F1FEA02005F08EFEC4F3072005F08AFE94
:10915000E0B205F087FE05F0E5FEA12005F082FEF5
:10916000002504E005F03CFE7055681CC5B2BD4208
:10917000F8DB05F0FBFE0120BDE8F0812DE9F047AA
:10918000054689461646002400BF281900F01F0036
:10919000C0F120008046311B884203DB301B00F009
:1091A000FF0800E000BF05F0BDFEA02005F05AFE5C
:1091B0002919C1F3072005F055FE2919C8B205F099
:1091C00051FE002706E0E11919F8010005F04AFEFA
:1091D000781CC7B24745F6DB05F0C8FE0A2004F04C
:1091E000A7F804EB0800C4B2B44200DB00E0CCE70F
:1091F00000BFBDE8F08710B5802005F0BBF828B1AE
:10920000032008F0EBFA802005F0AEF810BD000056
:10921000FEB506460D4617461C46022C01D1012418
:1092200000E000240A484078012809D102A82B4612
:109230003A461021CDE90004304600F047FF05E032
:1092400023463A4629463046FFF71EF9FEBD000088
:10925000384B002000B587B072211F4805F0F6FC9E
:1092600040F207111D4805F0F1FC4FF440711C4815
:1092700005F0ECFC72200190102002900020039079
:109280000420049001A9144800F045F840F20710AA
:10929000019010200290002003900420049001A966
:1092A0000E4800F038F88020019004200290002041
:1092B000039001A9084800F02EF84FF44070019087
:1092C00010200290002003900420049001A904487B
:1092D00000F021F807B000BD001001400008014077
:1092E000000C014070B504460D462A46214602484E
:1092F00004F0AEFA70BD00009C06002000B50146E7
:1093000000F026F8024600BF00F022F8801A8842DA
:1093100000D300BDF8E770B505460C462846D4E9F1
:109320000031E26805F0EEFC70BD70B504460D46F4
:109330002946204605F044FD012804D1294620464F
:1093400005F084FC03E02946204605F081FC70BD51
:10935000014800687047000044030020024800688C
:10936000401C0149086070474403002000B587B0E5
:1093700040F2026008F058F840F2046008F054F837
:109380004FF4C06008F050F840F20C6008F04CF860
:109390004023032210211F4805F0B4FCA023032220
:1093A00018211D4805F0AEFC4023032204211A4871
:1093B00005F0A8FC802303220421164805F0A2FC36
:1093C000002001904FF482700090002002900590E0
:1093D0004FF400700390102006900020049069461E
:1093E0000E4808F0F4FC0D4808F0DEFC00220321D2
:1093F000172007F055FA0721022005F037FC01225B
:109400000021802004F054FF802004F0ADFF07B05D
:1094100000BD000000100140000801400030014084
:109420002DE9F04104460D4616464FF0000800278E
:109430000AE02A466D1C14F8011B064800F00CF8DF
:1094400040EA0808781C87B2B742F2DB0020BDE88A
:10945000F08100000030014070B506460D4614460C
:1094600000BF02210A4808F0AAFC0028F9D02946CA
:10947000074808F0A2FC00BF0121054808F09FFC46
:109480000028F9D0024808F094FC2070207870BDC4
:109490000030014000BFFEE770B5002600240DE05B
:1094A000002508E005EB84001C49085C1C4901EB21
:1094B000850108556D1C042DF4DB641C042CEFDBC6
:1094C00018480068FFF760FD16480068461E09E06E
:1094D00000F040F900F05EF93046FFF755FD00F06E
:1094E00025F8761E002EF3DC00F034F900F052F976
:1094F0000020FFF749FD00240DE0002508E00848A2
:1095000000EB8500005D084901EB840148556D1CA6
:10951000042DF4DB641C042CEFDB70BD81AA002059
:10952000B1AA00204006002091AA00202DE9FF47A3
:10953000002107E1DFF8189219F801908DF80C90DE
:10954000DFF80C9209F1040919F801908DF80890E0
:10955000DFF8FC9109F1080919F801908DF80490E1
:10956000DFF8EC9109F10C0919F801908DF80090E1
:10957000012056E00DF10C09814419F8019C4FEAD5
:10958000D91909EBC90909EB49090DF10C0A824403
:109590001AF801AC89EA4A090DF10C0A0AF80090A0
:1095A0000DF10809814419F8019C4FEAD91909EB1A
:1095B000C90909EB49090DF1080A82441AF801ACFE
:1095C00089EA4A090DF1080A0AF800900DF1040928
:1095D000814419F8019C4FEAD91909EBC90909EB33
:1095E00049090DF1040A82441AF801AC89EA4A09D2
:1095F0000DF1040A0AF800900DEB000919F8019C1E
:109600004FEAD91909EBC90909EB49090DEB000A21
:109610001AF801AC89EA4A0909F0FF090DF800902F
:10962000401C0428A6DB9DF80E909DF80FA089EA47
:109630000A029DF80C909DF80FA089EA0A039DF894
:109640000A909DF80BA089EA0A049DF808909DF8FD
:109650000BA089EA0A069DF806909DF807A089EA02
:109660000A079DF804909DF807A089EA0A059DF86D
:1096700002909DF803A089EA0A0C9DF800909DF8DD
:1096800003A089EA0A089DF80D9089EA020989EA8F
:1096900006099DF809A089EA0A099DF804A089EA4B
:1096A0000A0989EA070989EA0809DFF8A4A00AF883
:1096B00001909DF8099089EA030989EA040989EA79
:1096C00005099DF805A089EA0A099DF800A089EA24
:1096D0000A0989EA0C09DFF878A00AF1040A0AF8F5
:1096E00001909DF80C9089EA020989EA06099DF823
:1096F00005A089EA0A0989EA070989EA08099DF8A3
:1097000001A089EA0A09DFF848A00AF1080A0AF864
:1097100001909DF80D9089EA03099DF808A089EA57
:109720000A0989EA040989EA05099DF801A089EA7C
:109730000A0989EA0C09DFF818A00AF10C0A0AF8EC
:109740000190491C0429FFF6F5AEBDE8FF87000033
:10975000B1AA00200E49C8798A79CA714A798A71FA
:109760000A794A710871087A897A094A1172114690
:109770008872487ACA7A4A72C872087B497B044A5E
:10978000117311468A7B4A73CA7B8A73C873704708
:10979000B1AA002000200FE000210AE0084A02EBF5
:1097A0008002525C074B9A5C054B03EB80035A54D2
:1097B000491C0429F2DB401C0428EDDB7047000043
:1097C000B1AA0020083A0108F8B5002500264F4844
:1097D000006882004E494F48FEF7DAFC4B480468A7
:1097E0008CE0601E4B4901EB800000680090474808
:1097F000006894FBF0F100FB114080BB9DF8007005
:109800009DF801008DF800009DF802008DF8010020
:109810009DF803008DF802008DF803709DF800009C
:109820003D49085C8DF800009DF80100085C8DF84A
:1098300001009DF80200085C8DF802009DF803000D
:10984000085C8DF803003148006894FBF0F0334960
:10985000085C9DF8001048408DF8000024E0FFE708
:109860002A48006806281FDD2848006894FBF0F1AC
:1098700000FB1140042817D19DF8000005F066F8A0
:109880008DF800009DF8010005F060F88DF80100EA
:109890009DF8020005F05AF88DF802009DF80300CB
:1098A00005F054F88DF80300A006050E174800785F
:1098B000201A8006060E1748805D9DF8001048406B
:1098C000144948550846304440789DF801104840F6
:1098D0001049294448700F48304480789DF80210A0
:1098E00048400C49294488700A483044C0789DF8A3
:1098F0000310484007492944C870641C08480068A0
:10990000401C8000A0423FF76CAFF8BD4406002029
:10991000EDAB0020C1AA0020083B0108083C01086B
:109920004006002000BFFEE730B5002068E0364C5E
:10993000235C245C344D2D1D2D5C6C40324D08356C
:109940002D5C6C40304D0C352D5C84EA05022E4CAC
:10995000255C241D245C85EA0401CC0904EBC404C5
:1099600004EB440484EA4104E1B2274C245C81EA1C
:1099700002056C40244D2C542C1D245C08352D5CB4
:1099800084EA0501CC0904EBC40404EB440484EA32
:109990004104E1B21C4C241D245C81EA02056540AF
:1099A000194C241D2554241D245C174D0C352D5CA9
:1099B00084EA0501CC0904EBC40404EB440484EA02
:1099C0004104E1B2104C0834245C81EA02056C4089
:1099D0000D4D08352C542C1D245C84EA0301CC0960
:1099E00004EBC40404EB440484EA4104E1B22C1DFA
:1099F000245C81EA02056C40034D0C352C54401C5C
:109A0000042894DB30BD0000B1AA0020094800887A
:109A100078B108480088401E80B20649088040B9E5
:109A2000002005494870C1F82404C1F82804C1F891
:109A30002C04704778050020F8460020704700008D
:109A400070B505460C46002605F07005204600F06E
:109A5000E1F806460E4A32F814100E4A52F8240075
:109A600005F0F4F82146272004F002FA45EA060042
:109A7000214604F0FDF9064A32F81410054A52F85E
:109A8000240005F0E5F8204600F0C4F870BD0000A1
:109A9000603901085039010810B504460A4A32F805
:109AA00014100A4A52F8240005F0D0F82146E220AA
:109AB00004F0DEF9044A32F81410044A52F8240083
:109AC00005F0C6F810BD00006039010850390108E2
:109AD00010B504460A4A32F814100A4A52F8240013
:109AE00005F0B4F82146E12004F0C2F9044A32F846
:109AF0001410044A52F8240005F0AAF810BD000022
:109B00006039010850390108F0B5C1B005460E466C
:109B100017461C460D4A32F814100D4A52F824001C
:109B200005F094F82846214604F0A2F923463A4667
:109B3000314601A804F0ABF9044A32F81410044A83
:109B400052F8240005F084F841B0F0BD60390108F6
:109B50005039010870B505460C460D4A32F814100C
:109B60000C4A52F8240005F071F82846214604F00A
:109B70007FF92146FF2004F07BF90646044A32F8BB
:109B80001410044A52F8240005F062F8304670BD03
:109B9000603901085039010830B5C3B005460C469C
:109BA00021460720FFF7D6FFC0F342004190204630
:109BB00000F04EF842909DF80801202805DD20466F
:109BC000FFF76AFF002043B030BD104A32F814108E
:109BD0000F4A52F8240005F039F82146612004F0BC
:109BE00047F923469DF80821294601A804F04FF9BA
:109BF000064A32F81410064A52F8240005F028F8F4
:109C00002046FFF749FF9DF80801DCE760390108AD
:109C10005039010870B504460B4A32F814100B4A4B
:109C200052F8240005F012F82146072004F020F92C
:109C30000546054A32F81410044A52F8240005F08B
:109C400007F8284670BD0000603901085039010846
:109C500070B504460D4A32F814100D4A52F824002B
:109C600004F0F4FF2146602004F002F92146FF20B1
:109C700004F0FEF80546054A32F81410044A52F87A
:109C8000240004F0E5FF284670BD0000603901089B
:109C90005039010870B504460D4629460620FFF7E5
:109CA00059FF20F0070604F0070006432A46314614
:109CB000062000F075F870BD2DE9F04104460E460F
:109CC00015461F46052D01DD052000E02846054606
:109CD000052C01DD052000E02046044604F10A01C0
:109CE000C8B23B462A46314600F032F8BDE8F08162
:109CF00070B505460E46002431460620FFF72AFFC0
:109D0000044624F0280415B944F0200408E0012D8D
:109D100002D124F0280403E0022D01D144F008040C
:109D200032462146062000F03BF870BD70B505466E
:109D30000C461646052C01DD052000E020460446B1
:109D4000334622462946102000F002F870BD00007C
:109D5000F0B5C1B005460E4617461C460E4A32F80D
:109D600014100E4A52F8240004F070FF45F0200051
:109D7000214604F07DF823463A4601A9304604F016
:109D800086F8054A32F81410044A52F8240004F008
:109D90005FFF41B0F0BD0000603901085039010893
:109DA00070B505460E461446104A32F81410104A93
:109DB00052F8240004F04AFF0E4A32F814100E4AFA
:109DC00052F8240004F042FF45F02000214604F040
:109DD0004FF82146304604F04BF8064A32F814108A
:109DE000054A52F8240004F033FF70BDAC39010875
:109DF0009C390108603901085039010870B5C0B0BC
:109E000006460D461446202D00DC0DB940B070BD4D
:109E10000D4A32F814100D4A52F8240004F016FFCF
:109E20002146B02004F024F823462A4669463046ED
:109E300004F02DF8044A32F81410044A52F82400B1
:109E400004F006FF00BFE1E760390108503901085E
:109E50007FB5054611A103C9CDE90201002000909C
:109E600001902B46052202A91020FFF771FF2B4617
:109E7000052269461020FFF747FE00240AE002A8E9
:109E8000005D1DF80410884202D0002004B070BDAF
:109E9000601CC4B2052CF2DB0120F7E71122A3A459
:109EA000A500000010B5002807DA0A07140E054ABD
:109EB00000F00F031B1FD45403E00A07130E024ADD
:109EC000135410BD18ED00E000E400E0BFF34F8F25
:109ED0000648006800F4E06005490843001D034996
:109EE0000860BFF34F8F00BFFEE700000CED00E0FD
:109EF0000000FA05704770B504460D4604F07F0176
:109F00002A460520FFF74CFF70BD10B504462146D8
:109F10007020FFF795FD10BD10B504460A4A32F8CF
:109F200014100A4A52F8240004F090FE2146012041
:109F300000F00EF8044A32F81410044A52F82400D3
:109F400004F086FE10BD0000AC3901089C39010800
:109F500070B504460E46002531460020FFF7FAFD95
:109F6000054614B925F0010503E0012C01D145F0A7
:109F70000105324629460020FFF712FF70BD0000A0
:109F80007CB5044619488169684688477CB99DF8C4
:109F900000109DF8012011449DF8022002EB0121E0
:109FA0009DF803208818FEF7EBF800207CBD012CFB
:109FB00014D10F4808F058F89DF800109DF80120C2
:109FC00011449DF8022002EB01219DF80320114469
:109FD00045182846FEF7D4F80120E7E7FEF7C6F853
:109FE000B0FBF4F104FB1100E0E70000480300209F
:109FF0000010004062B6704700B587B0182101A874
:10A00000FEF7EDF84FF40070019048200290012017
:10A0100003900320049001A90248FFF77CF907B0E0
:10A0200000BD0000000C014000B587B0182101A858
:10A03000FEF7D5F84FF40070019010200290012037
:10A0400003900320049001A90248FFF764F907B0C8
:10A0500000BD0000000C01402DE9F047C8B00646E5
:10A060000F4690469946DDF844A1509C00250020FB
:10A0700001908DF80C00BAF1000F02D110200B9066
:10A0800001E020200B900022414602A8FEF78AF949
:10A090000546BDB901A84B463A463146009002A894
:10A0A000FEF716F905466DB901982060206800EBAF
:10A0B000090101AA02A8FEF768F90546206801997E
:10A0C00008442060284648B0BDE8F0872DE9F047F5
:10A0D000C8B006460F4690469946DDF844A1509C0C
:10A0E0000025002001908DF80C00BAF1000F02D17C
:10A0F00010200B9001E020200B900022414602A886
:10A10000FEF7BEF90546BDB901A84B463A463146B1
:10A11000009002A8FEF74AF905466DB90198206043
:10A12000206800EB090101AA02A8FEF79CF9054688
:10A130002068019908442060284648B0BDE8F087AF
:10A14000704700000F49087949790E4A117111468C
:10A150008A794A71CA798A71C871087A897A094AF2
:10A16000117211468872487ACA7A4A72C872087B9C
:10A17000C97B044A117311468A7BCA734A7B8A736E
:10A1800048737047B1AA002000200FE000210AE0C8
:10A19000084A02EB8002525C074B9A5C054B03EBCA
:10A1A00080035A54491C0429F2DB401C0428EDDBCF
:10A1B00070470000B1AA0020083B010810B5FFF766
:10A1C000CDF810BD08B51848006840F47000164975
:10A1D00008601648006840F001001449086008460D
:10A1E000406840F0800048600020009002E0009845
:10A1F000401C009044F6206100988842F7D300206C
:10A200000A494860C8620846006809490840074989
:10A2100008604FF41F0088600846006820F4802022
:10A22000086007F095FE08BD88ED00E000100240D0
:10A23000FFFFF6FE10B50121880707F078FF40B157
:10A240000121880707F070FF0249C868804708F0BD
:10A2500079FE10BD480300201FB50020009001903A
:10A260000290039040F2AF40ADF800000020ADF83E
:10A270000200ADF80400F92002900020ADF80600BD
:10A280008DF80C0069464FF0804007F0F9FE00227F
:10A2900003211C2006F004FB00214FF0804007F052
:10A2A000E7FE002240F2AF414FF0804007F06CFF24
:10A2B000F921880707F0D6FE0121880707F02CFF57
:10A2C0000121880707F030FF0121880707F028FFE8
:10A2D0004FF0804007F0CEFE1FBD000010B50121F9
:10A2E000064807F024FF40B10121044807F01CFF95
:10A2F00003490869804708F020FE10BD00040040B3
:10A30000480300201FB500200090019002900390A8
:10A3100040F2AF40ADF800000020ADF80200ADF80B
:10A32000040040F2CF7002900020ADF806008DF8D6
:10A330000C006946134807F0A3FE002204211D20EB
:10A3400006F0AEFA00210F4807F092FE002240F21C
:10A35000AF410C4807F018FF40F2CF71094807F0F1
:10A3600081FE0121074807F0D7FE0121054807F0CB
:10A37000DBFE0121034807F0D3FE024807F07AFE16
:10A380001FBD00000004004010B50121880707F040
:10A39000CEFE18B10121880707F0C6FE10BD10B52A
:10A3A00008F052FC10BD000000B591B0402101A89A
:10A3B000FDF715FF2C4890F84E008DF804002A4850
:10A3C00090F84F008DF80500274890F850008DF860
:10A3D0000600254890F851008DF80700FE208DF802
:10A3E000080048208DF80900DE208DF80A007F2043
:10A3F0008DF80B0001208DF80C0002208DF80D0067
:10A40000302219495231002000F030F800909DF8B8
:10A4100000008DF80E009DF801008DF80F00124825
:10A4200040788DF8100030220F49523105A8FDF711
:10A43000AFFE30210C485230FDF7D1FE00200A4912
:10A4400081F88200202101A800F0C4FB00F0D8FBB5
:10A45000142000F03FF8202109A800F0BBFB00F019
:10A46000CFFB11B000BD00006463002070B506464C
:10A470000C4615462946204603F042F9064630466A
:10A4800070BD000010B50446074890F8310440B193
:10A490004FF48062044911312046FDF779FE002017
:10A4A00010BD0120FCE70000305F002030B50A46F7
:10A4B000CD1701EB5575C5F3C703CD1701EB5575E6
:10A4C000ED10A1EBC505ECB2C25C0125A540AA4385
:10A4D000C25430BD10B50446204602F046FF10BD00
:10A4E00030B502460846CD1701EB5575C5F3C703D5
:10A4F000CD1701EB5575ED10A1EBC505ECB2D05CA5
:10A500000125A540284008B1012030BD0020FCE70E
:10A5100070B505460E46144609482968C0F84E1025
:10A52000A0F88860C0F88440C4F38F200449888074
:10A530000846B0F8881003A005F068F970BD000067
:10A54000646300200A433A257800000001464878F9
:10A55000AA2808D18878BB2805D1C878CC2802D190
:10A560000879DD281FD01B4890F84E004A789042A9
:10A5700001D002207047174890F84F008A78904227
:10A5800001D00220F6E7134890F85000CA789042B4
:10A5900001D00220EEE70F4890F851000A7990426E
:10A5A00001D00220E6E748797F2801D00120E1E7C9
:10A5B0008879DE2801D00120DCE7C879482801D05D
:10A5C0000120D7E7087AFE2801D00120D2E7002039
:10A5D000D0E700006463002070B58AB005460C46E1
:10A5E000242101A8FDF7FBFDE0B28DF8040022460E
:10A5F00029460DF10500FDF7CBFD01A8FFF7A6FFE9
:10A60000A0B99DF80E00822801D00AB070BD0120CB
:10A61000274908702748DDF8111001609DF80F00E8
:10A62000254908709DF810004870EEE72048007832
:10A6300001283AD100201E49087020220DF10501A1
:10A64000FFF714FF06461C480088B0422CD11BA01F
:10A6500005F0DCF81B4890F88200102810DA194841
:10A6600090F882001749523101EB800011490968C6
:10A670000160144890F88200401C124981F8820061
:10A6800000200FE001AA411C515C49B10D490A317B
:10A69000095C01AB421C9A5C11430A4A0A3211540C
:10A6A000411CC8B22028EDDBAFE700BFADE70000DA
:10A6B0009C050020A00500209E0500200A4352436F
:10A6C000540000006463002070B58AB005460C4653
:10A6D000242101A8FDF783FD0026344890F84E00A0
:10A6E0008DF80400314890F84F008DF805002F4890
:10A6F00090F850008DF806002C4890F851008DF825
:10A70000070042208DF8080001208DF80900274835
:10A7100000788DF80A008DF80B50FF208DF80C00A2
:10A720008DF80D0000208DF80E008DF80F008DF8CB
:10A7300010008DF811001D4890F884008DF812006B
:10A740001A4890F885008DF81300184890F8860094
:10A750008DF81400154890F887008DF815001348FF
:10A7600090F888008DF81600104890F889008DF850
:10A7700017000E4880788DF818001B2202A90020CF
:10A78000FFF774FEC6B28DF823600AE0202101A80D
:10A7900000F020FA00F034FA3220FFF79BFE601E32
:10A7A000C4B2002CF2D10AB070BD00006463002076
:10A7B00030B589B0054624216846FDF710FD3448C0
:10A7C00090F84E008DF80000314890F84F008DF859
:10A7D00001002F4890F850008DF802002C4890F8A6
:10A7E00051008DF80300FE20294981F84A004821D4
:10A7F000274880F84B10DE2180F84C107F2180F82C
:10A800004D1090F84A008DF80400214890F84B0054
:10A810008DF805001E4890F84C008DF806001C4885
:10A8200090F84D008DF8070020208DF808000120D9
:10A830008DF80900164890F88E048DF80A00144827
:10A8400090F88F048DF80B00114800788DF80C00FB
:10A850008DF80D502021684600F0BCF900F0D0F9C9
:10A86000C820FFF737FE00240EE009498A31202274
:10A8700002FB0410114600F0ADF900F0C1F91420FC
:10A88000FFF728FE601CC4B2202CEEDB09B030BDFF
:10A890006463002010B5012007490870074800785C
:10A8A000401C0649087041F270700549086005486F
:10A8B000816B0020884710BD900500206463002054
:10A8C000940500204803002070B505460C46002082
:10A8D000034981F8310421460A2007F01FFD70BDAD
:10A8E000305F002070B5AF48006878B1AD480068AF
:10A8F000401EAC49086048B9AB48007830B1AA485E
:10A900000078052802D00520A7490870A6480078DD
:10A9100006287CD2DFE800F0030443B9D8FE3EE10C
:10A920001E210120FFF7D0FEA0480088401C9F494F
:10A93000088008460088282830DD00219C48A0F8BF
:10A940008A1440F2FF11A0F88C1401209849087273
:10A9500000204872302196485230FDF740FC00201C
:10A96000934981F882009149088091498871FF22BA
:10A9700040218F480A30FDF72BFC8D4A92F88A144B
:10A980009079FFF7A1FF002189480A30FFF78EFD7B
:10A9900000208749C871022083490870FFE084487D
:10A9A000B0F88A1483A004F031FF8148C0790128EF
:10A9B00016D07F488A30FFF765FD88B901207C49B1
:10A9C000C871002048724FF480628A31FFF74EFD53
:10A9D0007749A1F88E040846B0F88A14A0F88C14C0
:10A9E0007348B0F88C0440F2FF11884219D07048C7
:10A9F000407A401CC0B26E494872C82801DDC820A8
:10AA000048726B4991F88C04FFF7D2FE00E0C5E074
:10AA10004FF4E160FFF75EFD654991F88C04FFF7A4
:10AA2000C7FE6348407A6249097A88422CDB604855
:10AA3000C079012828D100205D49C87100241EE09A
:10AA400021465B480A30FFF74BFD70B1214658485C
:10AA50000A30FFF72BFD5648A0F88A44024692F8C8
:10AA60008A149079FFF730FF0DE051488088401E2E
:10AA7000A04202D103204C490870601CC4B24C486B
:10AA80008088A042DCDC00BF89E0002047490880C4
:10AA900047488078401C46498870202144480A3045
:10AAA000FDF79DFB042040490870414841784078FB
:10AAB000401C3F4A5070C82902DD012011464870F1
:10AAC0003EA004F0A3FE6AE0FFF76EFC3748008862
:10AAD000401C3649088008460088322846DB00259D
:10AAE00000200880002409E0214631480A30FFF7A1
:10AAF000F7FC08B1681C85B2601C84B22C488088C1
:10AB0000A042F1DC294630A004F080FE2DB90520DA
:10AB1000254900E02BE0087041E025488079401C81
:10AB20002349887108200872002416E02146204835
:10AB30000A30FFF7D5FC70B121461D480A30FFF7F7
:10AB4000B5FC1B48A0F88A44024692F88A14907912
:10AB5000FFF7BAFE05E0601CC4B215488088A04229
:10AB6000E4DC00BF02201049087018E017E01E2145
:10AB70000220FFF7A9FD0D480088401C0B49088002
:10AB800008460088282808DD002006490860074993
:10AB900008800549087007F019FB00E000BF00BFFE
:10ABA00070BD000094050020900500209A0500204B
:10ABB000646300200A533A2564000000444F574E56
:10ABC0005F515545525900000A4C4E756D3A256447
:10ABD0000000000070B505460C46002007F092F812
:10ABE0000549C86A80470646E1B204483246836A8E
:10ABF00028469847012070BD48030020B802002075
:10AC000010B54FF4FA7408E004F006F800B110BD76
:10AC10000220FFF75FFC601E84B2002CF4D100BF5D
:10AC2000F5E700BFFEE7002107E048F2782100BF0A
:10AC30000A1EA1F1010399B2FAD1021EA0F101038B
:10AC400098B2F2D17047000010B590B00446207958
:10AC50008DF8000020791E286FD2DFE800F06E1F0B
:10AC60000F5C2B6E6E6E6EAB9F8B7B6E6EC7C26E73
:10AC70006ECCCBDECDF1F2EFEE6E6EED0D22A9497A
:10AC8000601D04F056FE00F02DFF0D22A549C020E6
:10AC900002F070FA01208DF8000000BF0D220DF1C6
:10ACA0000101A04804F045FE0E2269460B2005F084
:10ACB000A1FF34E106229C49601D04F03AFE9B4846
:10ACC00090F8820028B1994890F882009649491E70
:10ACD00088709548401E807820B19348401E807847
:10ACE000042803DD01209049491E88708E48401ECB
:10ACF00080788F49497A884204DD8D48407A8A49B4
:10AD0000491E88708849491EC87806F09BF90420BE
:10AD10008DF8000000BF854890F88400292800D1F4
:10AD2000FDE0824890F88400282800D1F7E07F48B1
:10AD300090F88400332801D1F1E0EAE006220DF119
:10AD40000101794804F0F5FD072269460B2005F062
:10AD500051FFE4E0754890F87F0000B9DFE003227E
:10AD60007449601D04F0E5FD03227249D82002F009
:10AD700001FA00BF6D4890F87F0000B9CFE00B20CA
:10AD80008DF8000003220DF101016A4804F0D1FDA5
:10AD9000042269460B2005F02DFFC0E0634890F8BF
:10ADA000800000B9BBE06079012802D11E20624911
:10ADB000487000BF5D4890F8800000B9AFE00920FE
:10ADC0008DF800005C484078002801DD012000E09B
:10ADD00000208DF80100022269460B2005F00AFFD1
:10ADE0009DE05248816A2046884700BF4F49C86AA3
:10ADF000804794E000BF92E018225049601D04F0A3
:10AE000098FD4E48401E807818B1012006F03EFFA4
:10AE100002E0002006F03AFF00BF15208DF8000088
:10AE200018220DF10101454804F083FD19226946FD
:10AE30000B2005F0DFFE72E066E029E058E000E05C
:10AE40001AE00D223E49601D04F073FD00F04AFE39
:10AE500036480C21D0F80C213948401C9047334922
:10AE6000D1F8FC0080470D223549C02002F082F95C
:10AE700017208DF8000000BF0D220DF101013048B0
:10AE800004F057FD0E2269460B2005F0B3FE46E0A4
:10AE900003222C49601D04F04CFD2A48401EC17855
:10AEA000807801EB00204EF66021884207DDEA2021
:10AEB0002449491E887060212248401EC170214AE1
:10AEC000521ED378927803EB022290B2174AD2F83E
:10AED000041188471549D1F8FC008047032219491D
:10AEE0004FF4856002F046F919208DF8000000BF8C
:10AEF00003220DF10101134804F01BFD04226946F1
:10AF00000B2005F077FE0AE00F48016820468847CD
:10AF100005E00648D0F8E4102046884700BF00BF8F
:10AF200010B010BD59080020D703002044040020B1
:10AF3000EC100020D3030020D0030020DC07002009
:10AF400067080020DF030020380400202DE9F041CD
:10AF50008CB00446002620798DF81000207907284F
:10AF600071D2DFE800F09A0427286271900008226D
:10AF70006946402001F052FB0822A11D684604F0FA
:10AF8000C7FC40B900204B490870084600788DF88E
:10AF9000110002250DE0012046490870084600789E
:10AFA0008DF8110008220DF11201684604F0C1FC71
:10AFB0000A2574E000BF6079042810DD00208DF8B8
:10AFC00011004C208DF812004F208DF81300432003
:10AFD0008DF814004B208DF81500062524E0022082
:10AFE0008DF8100060798DF81100207902280BD1BE
:10AFF0006179502202EB01102F4910224B6A0DF1AA
:10B000001201984712250FE06179502202EB0110DE
:10B01000294910220B6AA11D984710220DF1120137
:10B02000A01D04F086FC122539E008220DF1120162
:10B03000402001F0F3FA03208DF8100000208DF875
:10B0400011000A252BE028E00822A11D402002F073
:10B0500091F803F04DFD0746A01D02F033FA80463B
:10B0600015483A460421036C4046984700208DF865
:10B0700011008DF8120008220DF11301A01D04F03B
:10B0800058FC0B250BE000208DF811000A4841699F
:10B090000DF1120088470E2501E0012600BF00BF18
:10B0A00026B92A4604A9092005F0A4FD0CB0BDE884
:10B0B000F0810000BC030020B8020020002106E05F
:10B0C0001E2100BF0A1EA1F1010399B2FAD1021E8E
:10B0D000A0F1010398B2F3D1704702E008C8121F33
:10B0E00008C1002AFAD170477047002001E001C171
:10B0F000121F002AFBD1704770B590B004460E466F
:10B100001546382D00DD38252A46314602A8FDF7C0
:10B110003FF8C5F1380102AA50192022FDF758F86E
:10B1200061208DF8000063208DF801006B208DF800
:10B1300002002D208DF8030020788DF8040060783F
:10B140008DF80500A0788DF806003A208DF80700EC
:10B150000348402182696846904710B070BD0000E6
:10B16000B802002030B591B00446062520224021C7
:10B1700001A8FDF72DF82A4604F1080101A8FDF702
:10B1800007F8402201A902A0FFF7B6FF11B030BDB9
:10B1900066756E0070B50546284600F028F8041E56
:10B1A00000D170BD6178204602F046FD08B900204C
:10B1B000F7E70120F5E770B50446002502F084FDAD
:10B1C000051E00D170BD702221462846FCF7E0FF25
:10B1D00002F04AFD06463146284602F069FD01208C
:10B1E000F0E700B502F048FD02F052FD00BD70B579
:10B1F0000646002511E0284602F02CFD041E00D171
:10B200000FE00422314604F16000FCF7F3FF10B9AF
:10B210006570204670BD681CC5B202F025FDA842CD
:10B22000E9DC00BF0020F5E700B505F079F905F08D
:10B2300083F901F065F901F06FF900BD704710B5B1
:10B240000346D3F8A400806868B153F8A40F80685F
:10B2500080781C68A468E47840EA0420108053F8E1
:10B26000A409806810BD0020108000BFFAE710B567
:10B27000034653F8A40F406880781C686468E4783B
:10B2800040EA0420108053F8A409406810BD03462A
:10B29000D3F8A400006800781080D3F8A4000068F8
:10B2A000704770B504460D46E07C50B100BFD4F83D
:10B2B000AC10A06C0022CB6A1146984700BF002159
:10B2C000E174A078032808D1D4F8A800006920B15F
:10B2D000D4F8A800016920468847204607F040F8C6
:10B2E000607830B1D4F8AC00C168204688470020AF
:10B2F000607070BD2DE9F04104460D46A07803282A
:10B3000008D1D4F8A800406920B1D4F8A800416958
:10B310002046884705EB450704F1140606EB870035
:10B3200000210A460B4641600281438100BF20464E
:10B3300007F01FF8BDE8F0812DE9F04104460F4603
:10B340000125D4F8AC0000221146036B04F10B0078
:10B3500098470646082E04D0204607F014F8BDE8AA
:10B36000F081E07A00F0600020B1202809D0402868
:10B3700015D10DE004F10B01204607F0C3FD054691
:10B380000EE004F10B01204607F01CF8054607E02B
:10B3900004F10B01204607F0CDFD054600E000BF9B
:10B3A00000BFC5B9B4F8110018B9204606F0E1FF96
:10B3B00014E0E07A00F0800048B100BF4C20035B4D
:10B3C00000212046A26C07F0BBF900BF06E0204632
:10B3D00006F0C6FF02E0204606F0D5FF00BFBEE73C
:10B3E00070B504460D460026287800F0030020B111
:10B3F00001282ED002282DD111E0A078022802D0F9
:10B40000032809D100E000BF6888012803D100218A
:10B410002172002070BD00E000BF00BF1BE02E794C
:10B42000A078032814D1688890B98EB1802E0FD0EF
:10B4300000BFD4F8AC003146826B2046904700BF75
:10B44000D4F8A8002946C268204690470020E1E7CA
:10B4500001E000E000BF00BF0120DBE770B504465B
:10B460000E460125A078022802D0032808D103E067
:10B47000207800B9002504E0207800B1002500E024
:10B4800000BF00BF35B901231A46214604F144002C
:10B4900006F088FF284670BD2DE9F04706460D46A8
:10B4A0000027B8464FF0010906F14404287800F05F
:10B4B000030020B101284BD0022852D150E0688807
:10B4C000070A95F80280102F3FD2DFE807F03E0808
:10B4D000182331323334353E3E3E3E3E3E36781EF2
:10B4E000304951F8203004F108024146304698476F
:10B4F0006060E888402801D10820208126E0781E7D
:10B50000284951F8203004F1080241463046984756
:10B5100060601BE0B8F1060F09DA781E214951F886
:10B52000203004F1080241463046984760600DE043
:10B5300000BF00BF00BF00BF08E004F108024146A1
:10B540003046FFF77CFE606000E000BF00BF09E00E
:10B55000D6F8A8002946C26830469047814601E0E7
:10B5600000E000BF00BF2089C8B1E888B8B12089D9
:10B57000E988884201DA208900E0E8882081218971
:10B58000B6F81100814208DA2089218890FBF1F297
:10B5900001FB120008B90121F1744FF0000948467F
:10B5A000BDE8F0879400002070B504460D46A078F1
:10B5B000012804D0022803D0032810D101E00FE0B5
:10B5C0000EE0287950B9D4F8A800411C01231A468E
:10B5D00004F1440006F0E6FE002070BD00E000BF6C
:10B5E00000BF0120F9E700002DE9F04104460E46B6
:10B5F00035790127307800F0030020B1012823D0ED
:10B60000022845D126E0A078022802D0032818D1CC
:10B6100000E000BF207918B101202449087002E041
:10B62000002022490870207A30B12048007840F08C
:10B6300002001E49087002E000201C490870002723
:10B6400000E000BF00BF24E0A078032801D105B9C5
:10B6500000271EE0A078032819D105F0800080287B
:10B660000BD105F07F0000EB400104F1440000EB3A
:10B67000810080780D49087008E005EB450104F170
:10B68000140000EB8100807808490870002700E072
:10B6900000BF00BF37B902231A46044904F1440031
:10B6A00006F080FE3846BDE8F0810000A0000020D2
:10B6B0000246012070470246888888B9C88878B950
:10B6C000887800F07F0050709078032808D0507878
:10B6D00010B10220907001E00120907000207047AE
:10B6E0000120FCE770B504460D460126A8782549DF
:10B6F000087008460078012842D8A07801283CD07C
:10B70000022802D0032839D110E01E48007858B131
:10B71000D4F8A80042681B48017820469047194891
:10B72000007820700320A070002628E015480078DB
:10B7300060B9D4F8A8008268124801782046904782
:10B740001048007820700220A07014E020780D4985
:10B75000097888420FD02178D4F8A8008268204662
:10B760009047084800782070D4F8A800426805483F
:10B77000017820469047002601E000E000BF00BFAE
:10B78000304670BDA200002002460020704770B510
:10B7900004460D460026287800F0030020B1012859
:10B7A00028D0022827D111E0A078022802D003284F
:10B7B00009D100E000BF6888012803D1012121726E
:10B7C000002070BD00E000BF00BF15E02E79A0781A
:10B7D00003280ED1688860B95EB1802E09D000BF01
:10B7E000D4F8AC003146426B2046904700BF0020A1
:10B7F000E7E701E000E000BF00BF0120E1E702460B
:10B800009078012804D0022803D003280BD101E04E
:10B810000AE009E0087928B98878D2F8A830587089
:10B820000020704700E000BF00BF0120F9E702469A
:10B830000020704710B50346D3F8A440E46854F8DC
:10B8400021000478148010BD10B50A4890F89000CB
:10B8500000B910BD05F004FE01200749487003F04F
:10B8600043F805F019FE00BF00F06AF80028FBD08D
:10B8700000BFEEE744040020384B002070B51248AA
:10B8800090F8900000B970BD1048007800B9FAE750
:10B890000E48807800B1F6E70D4806F0E5FB054656
:10B8A000FCF76EFC002407E0FCF760FCC1B207481F
:10B8B00023300155601CC4B2202CF5DB0348233033
:10B8C00007F0D2FF00BFDEE744040020384B002021
:10B8D0000010004010B50446154890F8900000B9DB
:10B8E00010BD1448007800B9FAE71349086A804788
:10B8F000032801DD132060711048007880F00100FA
:10B900000E4908700B480078A0730846007808B10B
:10B910000320A07207482330084A1278102313FB33
:10B9200002011A4604F10F00FCF732FC00BFD7E712
:10B9300044040020384B00204803002080050020EC
:10B9400030B589B01C208DF8000011208DF8010061
:10B950008DF802008DF803008DF8040013208DF897
:10B960000500062406E004F15B00C0B20DF80400F7
:10B97000601CC4B2212CF6DB684605F09DFE202039
:10B980008DF80000684605F0F9FD20208DF80000D4
:10B990009DF80600612809D19DF81D00782805D181
:10B9A0009DF81E00792801D1012500E000252846D8
:10B9B00009B030BD70B51748807B1649497B00EB54
:10B9C000012084B2214613480F3001F099FE11493D
:10B9D000C978104A927801EB0221884201D00020F8
:10B9E00070BD0C48807A0B49497A00EB012085B282
:10B9F0000DB90220F4E708494988491E064A0C326D
:10BA000002EB01204FF4807202490F31FCF7C0FBBA
:10BA10000120E5E772A9002064A5002010B50446C6
:10BA200044B10121084803F011F90221074803F04D
:10BA30000FF907E00221054803F008F90121024847
:10BA400003F006F910BD000000080140001001409D
:10BA5000194890F87B0020B1174890F87B001749EF
:10BA60008870154890F87C00A0B1144880780228AE
:10BA700002D1012011498870104880781A2802D11B
:10BA800019200E4988700D488078502802D14F2027
:10BA90000A49887009488078002806DD07488078C0
:10BAA000054991F87510884204DD0120034988702A
:10BAB000002070470120FCE744040020C30300205D
:10BAC00007484078012803DB05484078202804DD3A
:10BAD000012003494870002070470120FCE7000066
:10BAE000C3030020114890F87D0020B10F4890F862
:10BAF0007D000F4948700D4890F8810030B10C4826
:10BB00004078042802DA042009494870084840783F
:10BB1000012803DB06484078092804DD0120044998
:10BB20004870002070470120FCE70000440400201A
:10BB3000580800200221084AD1700021918000207D
:10BB400006E0064901EB800100220A60411C88B230
:10BB5000C828F6DB70470000B05E0020905B002034
:10BB60000146002008E0094A02EB800201EB800355
:10BB70001B681360421CD0B21E28F4DB0122034B69
:10BB80009B1FDA7000229A8070470000B65E00208A
:10BB900010B5002005494870087008710449886A8A
:10BBA0008047024948710120C87010BD81050020FE
:10BBB0004803002010B51A4890F8C40000B910BD21
:10BBC0001848C07B00B9FAE71648407C802800DBA3
:10BBD000F5E7144A517C907C00F02AF81148407C2B
:10BBE000401CC1B20F484174807C00EB80220E489B
:10BBF00000EB4200407881420FDB0021094841748C
:10BC0000007C401CC1B2074801740A2905DB0021F1
:10BC1000C1730648816B0120884700BFCFE7000051
:10BC2000440400207B5B00207E4B00204803002062
:10BC300070B58AB004460D4620208DF804002748D0
:10BC400081690DF1050088472449086A8047032867
:10BC500001DC312000E032208DF8090000208DF851
:10BC60000A008DF80B001D49886C8047014604EBE3
:10BC700084221B4810F8120061F31F10C0B28DF827
:10BC8000100000208DF8110004EB8421144800EB13
:10BC9000410040788DF812008DF8135004EB842297
:10BCA0000F4800EB4200801C00EB0511102205A894
:10BCB000FCF76EFA1B210DF1090001F021FDC0B265
:10BCC0008DF824000549C86A804706460348314676
:10BCD000426B01A890470AB070BD000048030020E5
:10BCE0007E4B00202DE9F04190B0804620208DF859
:10BCF00000000DF1010002F059FE00208DF8060051
:10BD00008DF80700B8F1010F23D1002618208DF817
:10BD100005006E4890F87F0080B36D484078002899
:10BD200001DD012000E0002069498978002901DD5A
:10BD3000012100E0002100EB41006549C97800299C
:10BD400001DD012100E0002100EB81008DF80600FB
:10BD50001AE0052619208DF805005C4890F87F0050
:10BD600060B15B484078002801DD012000E0002040
:10BD700057498978002902DD012101E004E0002112
:10BD800000EB41008DF80600002597E05148C07A8D
:10BD9000A84200D190E0504890F8200000285AD1E5
:10BDA000002413E005EBC50202EB4513494A0C32AF
:10BDB0001A44521C331902EB830002AA052303FB29
:10BDC00004211A4603F0B5FD601CC4B2052CE9DB62
:10BDD0003E4890F88400332869D13C4890F88500AB
:10BDE000012864D103F006F9002860D00424002063
:10BDF00004EB4401062202EB41010DF8010004EBC3
:10BE00004401072202EB41010DF8010004EB44015B
:10BE1000082202EB41010DF8010004EB4401092264
:10BE200002EB41010DF801001D210DF1050001F0AB
:10BE300067FC0746381204EB44010A2202EB410179
:10BE40000DF80100F8B204EB44010B2202EB4101B2
:10BE50000DF801002BE0002413E005EBC50202EB16
:10BE600045131C4A0C321A44521C331902EB83004E
:10BE700002AA052303FB04211A4603F05AFD601CA5
:10BE8000C4B2042CE9DBFF208DF81C008DF81D00E6
:10BE90008DF81E001A210DF1050001F031FC074656
:10BEA00038128DF81F00F8B28DF8200000BF294627
:10BEB000684600F0ADFF00BF681CC5B20548007AB7
:10BEC000A8423FF763AF10B0BDE8F0814404002002
:10BED000D2030020EC1000209C07002070B588B031
:10BEE0001C208DF800000DF1010002F05FFD15200F
:10BEF0008DF80500002440E02348C07AA04200D11C
:10BF000039E0002513E004EBC40202EB44131E4A9F
:10BF10000C321A44521C02EB85000DF1060202237A
:10BF200003FB05211A4603F004FD681CC5B20A2D67
:10BF3000E9DB164890F88400332817D1134890F8AD
:10BF40008500012812D103F055F878B100208DF852
:10BF50001A0016210DF1050001F0D2FB0646301241
:10BF60008DF81B00F0B28DF81C0000BF214668461A
:10BF700000F04EFF00BF601CC4B20348007AA0422C
:10BF8000BADC08B070BD0000EC10002044040020B2
:10BF90002DE9F04190B0064623208DF800000DF108
:10BFA000010002F003FD16208DF80500012E01D1DD
:10BFB000002000E005208046002567E03748C07A71
:10BFC000A84200D160E0002415E005EBC50202EBB9
:10BFD0004513324A0C321A44521C08EB040302EB9C
:10BFE00083000DF10602042303FB04211A4603F02B
:10BFF000A0FC601CC4B2052CE7DB294890F8840043
:10C0000033283CD1264890F88500012837D102F02A
:10C01000F1FFA0B30424002004EB4401062202EB4C
:10C0200041010DF8010004EB4401072202EB41013C
:10C030000DF8010004EB4401082202EB41010DF868
:10C04000010004EB4401092202EB41010DF801005B
:10C050001D210DF1050001F053FB0746381204EBDA
:10C0600044010A2202EB41010DF80100F8B204EB91
:10C0700044010B2202EB41010DF8010000BF2946EB
:10C08000684600F0C5FE00BF681CC5B20348007AD0
:10C09000A84293DC10B0BDE8F0810000EC10002055
:10C0A0004404002010B58AB01548007810B900206B
:10C0B0000AB010BD00201249087020208DF8000041
:10C0C000104881690DF1010088471A208DF805009C
:10C0D00001208DF806000C480068CDF807000949DA
:10C0E000886A80478DF80B000649086B8047044634
:10C0F00004482146426B684690470120D8E700007B
:10C1000088050020480300208905002010B5012083
:10C110001B4908701B48007A1A49C97900EB0120B5
:10C1200084B2601C84B220121649C8710846047299
:10C1300005F048FF14480078401CC0B2124908704E
:10C14000192819DB00200870104890F8800038B1D9
:10C150000F48407820B10E484078401E0C49487086
:10C160000C48807828B90C48806A401C0A498862CB
:10C1700002E000200849886205F0F2FB10BD0000D3
:10C18000F1030020CC070020F2030020440400202B
:10C19000D0030020F40700209C0700207047000017
:10C1A00010B50120054908700549486880470128F5
:10C1B00001D000F03BFD07F061F810BDF003002056
:10C1C000DC05002010B500200649887000220521FA
:10C1D0000448C01C03F0B8FB0020034981F820008C
:10C1E00010BD0000F40700209C0700200148807863
:10C1F00070470000F407002010B500F02DFA03F09E
:10C200003DFE07F02FF800F003FA00F0C5F90349EE
:10C210000868804702490868804710BDDC05002097
:10C220002406002010B500F0C2F903F057FA05F01B
:10C230008BFF0548807D28B100200349887503499C
:10C24000C86E804710BD00009C07002044040020F9
:10C250000149887070470000F407002010B50749B5
:10C26000086A8047032804D00449086A80470628E2
:10C2700001D1012010BD0020FCE700004803002090
:10C280002DE9F04104460D46002600F063F9061E34
:10C2900001D1BDE8F08105F10A0221463046FBF7E5
:10C2A00077FF00F025F907463946304600F046F999
:10C2B0000120EEE700B589B026480078022809D1B0
:10C2C000254801780078401E234A107011B90020DB
:10C2D0002049087000F00CF910B11E48007808B130
:10C2E00009B000BD01201B4908700A201A490870D6
:10C2F000002000F0DDF81949086005208DF80700DE
:10C3000001208DF808000846006800798DF80900C2
:10C310000846006840798DF80A0008460068D0F8A1
:10C320000600CDF80B0000208DF80F0020208DF8BE
:10C3300010000B49C86980478DF811000748006854
:10C340000068CDF812000F210DF10700FCF7B0FED8
:10C3500000BFC5E7080600200906002004060020EB
:10C360004803002030B5A1B00446402110A8FBF7D7
:10C3700036FF31208DF84000E1208DF841002F4933
:10C38000C86980478DF8420017208DF843000220CD
:10C390008DF844002A48006800798DF84500284847
:10C3A000006840798DF8460000208DF84700202075
:10C3B0008DF8480020128DF84900E0B28DF84A004F
:10C3C000002528128DF84B008DF84C50002C11DD03
:10C3D000601E1B4A12680A3202EB401120220DF146
:10C3E0005100FBF7D5FE0A201649087002201649B5
:10C3F000087007E000211248006800F049F80020AA
:10C400001149087040216846FBF7E9FEF5208DF8D8
:10C410000000AA208DF801008DF802009DF8400070
:10C42000421C10A90DF10300FBF7B2FE07484021A2
:10C4300082696846904721B030BD00004803002063
:10C44000040600200906002008060020B80200208B
:10C4500010B504462079022800D010BD60790B4940
:10C4600009680979884200D0F7E7207AE17900EB82
:10C470000120202800D0F0E7A17A627A01EB0221A6
:10C4800088B2FFF76FFF00BFE7E700000406002057
:10C4900070B504460D46FF2084F80A042946034877
:10C4A00002F048F90646304670BD0000F80500204D
:10C4B00010B504462146024802F066F910BD00009E
:10C4C000F8050020002100200CE040F20B4242431E
:10C4D000064B1A4492F80A24FF2A01D14A1CD1B211
:10C4E000421CD0B20428F0DB084670473494002088
:10C4F00010B5024802F05EF910BD0000F8050020FA
:10C500000348044908604860002008817047000023
:10C51000F0050020F8050020002009E0FF2240F28D
:10C520000B414143044B194481F80A24411C88B251
:10C530000428F3DB704700003494002070B50446F3
:10C540000D462A462146024802F038F970BD000027
:10C55000F8050020002118E040F20B4048430D4A46
:10C56000104490F80A04FF280DD1012240F20B403C
:10C570004843084B184480F80A2440F20B404843D3
:10C580001A4610447047481C81B20429E4DB00209D
:10C59000F8E700003494002010B503F0CDF805F062
:10C5A000FBFD02F08FFE012000F0F0F910BD00B598
:10C5B00091B0684604F0CEFC08B911B000BD9DF8FA
:10C5C0000100602803D09DF80100612809D19DF881
:10C5D000020030B102F0D8F99DF80210884200D074
:10C5E000EBE704F0A3FF9DF80100602803D1684643
:10C5F00004F0EEF90AE09DF80100612803D16846D5
:10C6000004F04AFB02E0684604F08EFC00BFD4E769
:10C6100010B504F0B9FC05F0CBFD10BD70B5C0B08D
:10C6200005460E461446601CC2B20A486946436A73
:10C63000284698479DF80000F52808D12246314643
:10C640000DF1010003F075F9012040B070BD00202C
:10C65000FBE70000B802002010B5C0B00D2269460B
:10C66000C020FFF7DBFF88B10D22BA49684603F00E
:10C6700060F90D22B849684603F05BF9B7480C2110
:10C68000D0F80C21B448401C904710E00120B1497B
:10C69000491E487000220C21AE48401C03F054F99A
:10C6A000AE480C21D0F80C21AB48401C9047FFF756
:10C6B00019FA032269464FF48560FFF7AFFF80B196
:10C6C0000322A749684603F034F9A54A521ED378DD
:10C6D000927803EB022290B2A04AD2F80411884764
:10C6E00004E09E48D0F804110020884707226946DC
:10C6F0000020FFF793FF28B107229A49684603F00C
:10C7000018F91EE00121974A521E5170917011468E
:10C710000979D27801EB022188B201200112914AF5
:10C72000521ED170114608718979527901EB0221AC
:10C7300088B2012001128B4A521E51711146887134
:10C7400000BFFFF7BDF9FFF783F90D226946082006
:10C75000FFF764FF28B10D228349684603F0E9F82A
:10C7600005E0FF2206218048C01C03F0EDF805F02B
:10C770006FFA042269461820FFF750FF28B10422FF
:10C780007A49684603F0D5F804E0FF22042177488F
:10C7900003F0DAF8062269463020FFF73FFF28B1A0
:10C7A00006227349684603F0C4F80AE00020704985
:10C7B000491E48704870C87008710A2048710820E6
:10C7C00088711A226946A020FFF728FFE0B11A22DB
:10C7D0006849684603F0ADF8604890F8C400C0B1FD
:10C7E0006448401E80780E2813D16248401EC078ED
:10C7F00014280ED15949D1F8D400804748B90120F6
:10C800005D4981F8200004E000221A21594803F014
:10C810009BF8082269464020FFF700FF60B1002026
:10C82000554988859DF80000402811D0684600F0E1
:10C8300049FE514988850BE00924224669464F4844
:10C8400003F077F822466946402000F093FC00BFD1
:10C8500004226946D020FFF7E1FE28B104224849AE
:10C86000684603F066F804E000220421444803F01F
:10C870006BF803226946D820FFF7D0FE28B10322C7
:10C880004049684603F055F806E001203D49491E3D
:10C89000487000208870C87006226946F020FFF7B3
:10C8A000BDFE48B306223849684603F042F82B48DB
:10C8B00090F8820028B1294890F882003249491E38
:10C8C00088703148401E807820B12F48401E807803
:10C8D000042803DD01202C49491E88702A48401E87
:10C8E000C0782049491E8978884219D01D49491EBF
:10C8F000887805F041FA13E0184890F8820030B1CA
:10C90000164890F882002049491E887003E00120F3
:10C910001D49491E88701349491E887805F02CFA74
:10C92000012269464FF4A070FFF778FE20B19DF810
:10C9300000001149C8750AE0084890F8850018B150
:10C9400001200D49C87502E000200B49C87540B0B0
:10C9500010BD000059080020670800204404002092
:10C96000DF030020C40300204B080020CC0300207C
:10C97000CD070020F50700209C070020B4390108EE
:10C98000BE030020D3030020D70300200149087014
:10C9900070470000E010002030B58BB000F02AFE98
:10C9A00008B10BB030BD02F08DFC20208DF80400E2
:10C9B0000DF1050001F0FAFF10208DF8090001F0DB
:10C9C000E3FF8DF80A00A5208DF80B0001F0E8FFC9
:10C9D0008DF80C00554840798DF80D00534880794A
:10C9E0008DF80E0008220DF10F01514802F0A1FF51
:10C9F0004F48401EC07800F00F008DF8110001F084
:10CA0000C9FF022803D001F0C5FF052805D19DF814
:10CA1000110040F080008DF811004648007820B1E8
:10CA2000012815D0022837D120E001208DF8170009
:10CA30000C2206A9404802F07CFF404890F8840090
:10CA40001E2801D1012000E002203A49087027E0A9
:10CA500003208DF81700092206A9394802F069FF62
:10CA600034480078401C3349087019E002208DF8E2
:10CA70001700344840788DF818003348007A8DF854
:10CA8000190004220DF11A012F48001D02F051FF78
:10CA900000202849087003E000202649087000BFE4
:10CAA00000BF002435E02848C07AA04200D12EE023
:10CAB00002F016F820B12448001D005D8DF80C002E
:10CAC0001E4890F884001E280CD01C4890F8840062
:10CAD000332817D1194890F88500012812D102F0A7
:10CAE00089FA78B11A210DF1090000F009FE054616
:10CAF00028128DF82300E8B28DF8240020208DF84C
:10CB0000040000BF214601A800F082F900BF601CAC
:10CB1000C4B20D48007AA042C5DC03200B4908705E
:10CB200000204870887000BF3BE70000C30300206E
:10CB3000CD070020E90300205A080020440400200B
:10CB4000A9070020D6030020EC100020E0100020F0
:10CB500010B588B01F208DF80000134881690DF1D1
:10CB60000100884710208DF8050001F00DFF8DF8B9
:10CB7000060018220DF107010C4802F0DAFE00242D
:10CB800005E02146684600F043F9601CC4B208483D
:10CB9000007AA042F5DC03200649087000204870A6
:10CBA000887008B010BD000048030020DC0700209A
:10CBB000EC100020E010002030B589B004461F20A2
:10CBC0008DF80400154881690DF105008847332070
:10CBD0008DF8090034B917220DF10A01104802F04E
:10CBE000A8FE05E017220DF10A010E4802F0A1FE91
:10CBF00001F0D6FE8DF8230001F078FF05462946A6
:10CC000001A800F005F9032007490870084640789C
:10CC1000401C48700020887009B030BD48030020D7
:10CC20003308002075080020E010002010B503F044
:10CC300083F87248007800B910BD70480078082861
:10CC400072D2DFE800F0D70412153A576AAC01F04F
:10CC5000A1FE032806DD6A4890F87A0010B100F0C2
:10CC600037F901E0FFF798FEC5E000F031F9C2E0C6
:10CC700062488078401CC0B2604988700A2813DA84
:10CC80005F48D0F8F410012088475D48007850B123
:10CC900001F080FE082803D001F07CFE092802D1B3
:10CCA000574908698047A6E05548D0F8F41000209D
:10CCB00088470420514908709DE001F06BFE03286D
:10CCC00005DCFFF70BF906204C49087011E001F074
:10CCD00061FE032807DD4A4890F87A0018B1012068
:10CCE000FFF700F802E00120FFF752F90520434961
:10CCF000087080E001F04EFE032807DD404890F800
:10CD00007A0018B10220FEF7EDFF02E00220FFF7E3
:10CD10003FF90620394908706DE003F027F93949D9
:10CD20008868804708B187E764E004F0AFF840B155
:10CD30000020324948720872334848600720087062
:10CD40002CE02F4890F8340068B12D49486C80479A
:10CD500048B100202949487208722948C06B4860D0
:10CD6000072008701AE001F015FE032803DD2448AF
:10CD700090F87A0048B921484078022805DB002065
:10CD80001E494870FFF708FE08E002F073FF10B973
:10CD900000F09EF802E00020FFF7F8FD2BE01749B5
:10CDA0004868804770B11548407A401C1349487262
:10CDB0000846407A50281CDB0120144908700F49AE
:10CDC000087016E00D49097A491C0C4A11720C4989
:10CDD00091F884101E2901D1142000E05020074949
:10CDE000097A814204DB0121084A1170034A11705B
:10CDF00000BF00E000BF00BF00BF1DE7E010002043
:10CE000044040020240600208D0E0108E9030020C0
:10CE100030B591B005460C462878401CC2B2694630
:10CE2000284602F086FD124890F87E0060B19DF819
:10CE30000000001FC0B28DF800009DF800200DF129
:10CE40000101081D02F075FD0A49085D04F008FEA5
:10CE50000748D0F8A410684688470648025D9DF848
:10CE600000100548836A0DF10100984711B030BDEC
:10CE700044040020EC100020B802002010B590B04F
:10CE80000446F5208DF80000AA208DF801008DF8E9
:10CE900002002078401CC2B20DF10301204602F0CE
:10CEA00048FD9DF80320D21CC2F14002D1B29DF88A
:10CEB00003206B461A44D01C002202F045FD0348B3
:10CEC000402182696846904710B010BDB80200202A
:10CED00030B58BB000F0A6FB08B10BB030BD02F04E
:10CEE000F1F99948D0F8D01000208847012800D1E6
:10CEF000F3E700F095FD95484079401C934948714F
:10CF000008464079072801DD002048718F484079A4
:10CF100078B98F48007880F001008D490870084684
:10CF2000007830B98B498868804707208749487165
:10CF3000D3E789498868804710B107208349487141
:10CF400086494868804710B10720804948717E486B
:10CF500090F87F0040B17C4890F87F0000287DD099
:10CF60007F48C0780028FAD020208DF804000DF109
:10CF7000050001F01BFD01F00DFD032801DC13206D
:10CF800000E014208DF8090001F004FD032806DDFF
:10CF90006D4890F87A0010B117208DF8090071489B
:10CFA000C0798DF80A006F48007A8DF80B001A22BC
:10CFB00003A96D4802F0BDFC6348007878B101F028
:10CFC000E9FC082803D001F0E5FC092807D16648F0
:10CFD000401E807840F040008DF80D0006E0624869
:10CFE000401E807820F040008DF80D005648016A00
:10CFF00001A8884720B15449D1F8B000804770BBE0
:10D0000001F0C8FC032841DD4F4890F87A0038B39E
:10D0100017208DF8090004220DF121014B48401C16
:10D0200002F087FC494840798DF8200001F0B2FCFD
:10D03000052801D1012000E0002044494978084337
:10D040008DF82100414880788DF8220001F0A8FC7D
:10D050008DF823003C4890F8840002E068E01CE072
:10D0600014E0282804D0384890F88400292808D1F2
:10D070001B210DF1090000F043FBC0B28DF8240024
:10D080000BE0324800798DF8240006E0A5208DF8E9
:10D09000210001F085FC8DF82200002444E0334893
:10D0A000C07AA04200D13DE001F01AFD20B12F4826
:10D0B000001D005D8DF82200234890F884001E2892
:10D0C0000CD0214890F88400332817D11E4890F8DE
:10D0D0008500012812D101F08DFF78B11A210DF1E0
:10D0E000090000F00DFB054628128DF82300E8B278
:10D0F0008DF8240020208DF8040000BF9DF80D005D
:10D1000058B19DF80D0000F0800018B920208DF86E
:10D11000040002E020208DF80400214601A8FFF75A
:10D1200077FE00BF601CC4B21048007AA042B6DC93
:10D1300003200F49087008464078401C48700020C2
:10D14000887000BFC9E6000044040020BD03002031
:10D15000EE03002024040020DC0500203804002019
:10D16000D2030020CC070020F5070020EC1000209F
:10D17000E010002070B5C0B006460C461546F520FC
:10D180008DF800002A460DF10101204602F0D1FB86
:10D19000681CC2B203486946036A304698470120BA
:10D1A00040B070BDB80200200348407808B10120AB
:10D1B00070470020FCE70000C8420020002003491F
:10D1C000487003490880034908807047C84200201E
:10D1D000680500206A05002030B59BB037484078CC
:10D1E000082866D2DFE800F065040D10393D575B72
:10D1F000324AD078324A516B8847FF202F49487015
:10D2000058E0FFF7DBFF55E02C4800892B49C9881F
:10D2100000EB01212B480088401C80B2294A108075
:10D22000814200DC46E020208DF84400002403E029
:10D2300011A80455601CC4B2202CF9DB2249C86A2D
:10D240008047054620482946426B11A890471B4A53
:10D25000907A1B4AD16888472CE000201B4908803F
:10D2600028E09DF80400202801D01BB030BD9DF8B7
:10D27000050000B1F9E79DF80600012800D0F4E7A9
:10D280009DF80700022800D0EFE710480088401CF6
:10D290000E4908800EE000200D4908700AE00D4894
:10D2A000007800B906E00649886B80470849087095
:10D2B00000E000BF00BF00BFD7E70000C842002069
:10D2C000B802002068050020480300206A050020FD
:10D2D0006C0500206D050020114A43681360038926
:10D2E0009380837A9371521E52780A700C4A521EB0
:10D2F00092784A700A4A521E12798A70094A128834
:10D300001212CA70074A12780A71074A128812125A
:10D310004A71054A12788A71044A1278CA717047B4
:10D32000C9420020680500206A0500206C05002025
:10D33000002107E048F2782100BF0A1EA1F1010395
:10D3400099B2FAD1021EA0F1010398B2F2D170474E
:10D35000002105E01E2100BF0A1EA1F10101FBD141
:10D36000021EA0F10100F5D17047002105E01E2149
:10D3700000BF0A1EA1F10101FBD1021EA0F10100B4
:10D38000F5D1704710B504464FF4C8714FF4E15021
:10D39000FBF71AFE10BD000070B586B004460020F1
:10D3A00002900390049005903D480068019001268A
:10D3B000E0780B2804D00C2808D00D2864D15DE05B
:10D3C0003848A1880180A17981705FE02079012827
:10D3D00002D02079022827D1A079802800DB55E0EF
:10D3E0002079401EC5B2217905EB85222D48C01C4D
:10D3F00000F8121000F6FD708574617905EB852246
:10D40000A0F6FD7000EB4200417005EB8522254936
:10D41000C91C01EB4201891CA27901EB0210102208
:10D42000E11DFAF7B5FE28E0207900F0800020B376
:10D43000A079802800DB29E0207920F08000401EC0
:10D44000C5B205EB85211748C01C00EB41004078B0
:10D450008DF80500A0798DF8060005EB85221148AE
:10D46000C01C00EB4200801CA27900EB02111022CC
:10D470000DF10700FAF78CFE132607E00A486168F1
:10D480000160A168416001E0002600BF00BF2EB12D
:10D49000E178334601AA602005F064FD06B070BD56
:10D4A000043A01087B4B0020825B002001460448BF
:10D4B0008078401E132202EB4010C0B2704700007B
:10D4C000B493002010B5024600230024002108E098
:10D4D000505C1844C3B2081D105C2044C4B2481C00
:10D4E000C1B20429F4DB83F0A50384F0A50403EBA7
:10D4F000042080B210BD0000014601F10800C0B256
:10D500000246044B93F87530984201DD01207047C4
:10D510001046FCE74404002010B50146132901DC45
:10D52000012012E0A1F11303D81703EBD0604011E2
:10D53000401C1A46D41702EBD4646411A2EB4414C5
:10D540000CB1012400E000242044C0B210BD01460B
:10D5500009B9002003E0481E132202EB4010C0B2BC
:10D56000704702461320704710B501460020002383
:10D5700014E04FF6FF7404EA83028C5C4CB9541C2F
:10D580000C5D34B9941C0C5D1CB9D41C0C5D04B941
:10D5900002E0441CE0B200BF5C1CA3B20A2BE8DB33
:10D5A00010BD00000C480078401CC0B20A49087049
:10D5B000FA2801DA00207047002007490870084661
:10D5C00040782D2803DB002048700120F3E700207D
:10D5D000014948700220EEE78105002004480078E8
:10D5E00020B10348007908B1012070470020FCE712
:10D5F0007005002010B501F073FA08B9002010BDC5
:10D600000748007880F00100054908700846007856
:10D6100018B1FFF79DFA0120F1E70020EFE70000C5
:10D62000EA03002010B5244890F8210080B3234875
:10D63000007880F001002149087048B31E4890F836
:10D640002300A0B11C4890F8240080B11C48007849
:10D6500018B90020FFF7B0FA02E00120FFF7ACFA9A
:10D660001748007880F00100154908700EE0124854
:10D6700090F8230018B10020FFF79EFA06E00E484C
:10D6800090F8240010B10120FFF796FA012010BD98
:10D69000FFE7094890F8220060B10A48807848B94D
:10D6A0000020054981F8220081F8210081F823003B
:10D6B00081F824000020EAE79C070020EC0300200A
:10D6C000ED030020F4070020002001490870704796
:10D6D000D80500200246002107E00748405C904240
:10D6E00001D108467047481CC1B20348407A8842BD
:10D6F000F3DCFF20F6E70000EC100020704700008C
:10D7000070B5024600201CE003134FF6FF7404EAD4
:10D7100000101478E51704EB157583EA25150C4EF7
:10D7200036F81550684003134FF6FF7404EA0010F2
:10D73000147804F00F045C40354635F8144060401E
:10D74000521C0C1EA1F10105A9B2DDD170BD000073
:10D75000083D01087047000070B505460E46D5F833
:10D76000B040012E18D12078F52805D16078AA287C
:10D7700002D1A078AA2802D02046FFF7BFFF0020E0
:10D7800004F0ACFA0548C16CE01C884740232246EF
:10D790000121284604F051FF70BD0000480300201D
:10D7A00070B504460D468121204604F0CFFE0121CC
:10D7B000204604F0CBFE002070BD000070B504468A
:10D7C0000E4643211B48FAF70AFD1B4B4FF4A0728B
:10D7D0000021204604F020FF174BDB1D4FF4807220
:10D7E0000021204604F018FF4023124A0121204660
:10D7F00004F023FF11488169C4F88810C169C4F896
:10D8000084100C48C4F8B000D4F8B40078B10025F6
:10D810000BE0D4F8B40050F8250020B1D4F8B410CF
:10D8200051F825008047681CC5B2042DF1D30020B3
:10D8300070BD000058070020D10000208C0200209D
:10D84000024619B1C2F8B410002070470220FCE76C
:10D8500070B506460C4615462B46224681213046B9
:10D8600004F06EFF002070BD2DE9F04105460C4626
:10D870000127D5F8B06060780C2865D2DFE800F0A9
:10D88000642D394364640664644D595F60882221C5
:10D89000B1EB202F0ED1E088202801D9202000E014
:10D8A000E088024600232B4905F1440004F07EFD88
:10D8B000002711E060882121B1EB202F0CD1E088F6
:10D8C000092801D9092000E0E08802460023224906
:10D8D00005F1440004F06AFD37E0E088022807D132
:10D8E00000230222314605F1440004F05FFD0027C9
:10D8F0002BE00023012206F1410105F1440004F070
:10D9000055FD002721E00023012206F1420105F127
:10D91000440004F04BFD002717E0A07886F8400093
:10D92000E2880023314605F1140004F03FFD002792
:10D930000BE06088001286F84100002705E0A0781F
:10D9400086F84200002700E000BF00BF3846BDE86F
:10D95000F081000030390108C80000202DE9F041B5
:10D9600005460E4690461A490868C11700EBD1617A
:10D970004911184A116010460068801D1649086058
:10D98000102001F08FFF074610213846FAF727FCD8
:10D99000002403E0305D11490855641C0D480068FF
:10D9A000B4EB800FF6DB002403E0285D0C4908553A
:10D9B000641C102CF9DBFBF707FFFBF76DFD102251
:10D9C00008493846FAF7E4FB3846BDE8F081000024
:10D9D000480600204406002040060020EDAB002051
:10D9E00081AA002091AA002010B50A48007978B9D0
:10D9F000084890F8060858B900210748C17307493C
:10DA0000886E80470548816B01208847012010BD42
:10DA10000020FCE77B4B00207B5B002048030020BC
:10DA200010B50C480078401CC0B20A4908700A289A
:10DA30000ADD084600780C2801DD00200870064841
:10DA4000816D0120884703E00348816D00208847ED
:10DA500010BD0000EB030020B80200202DE9F041CA
:10DA600004462CB90F488178001D00F089F816E0B3
:10DA700001F03EF806460B4991F863002146FFF796
:10DA800070FD07462046FFF762FD01460548801DF0
:10DA90000D18054832463946836A28469847BDE83E
:10DAA000F0810000B4930020B802002070B5044655
:10DAB000A01CFDF79CFB051E0CD0B5F86C606978C6
:10DAC000284600F0B9F820B1627AA11C012000F0CC
:10DAD0001BF900BF70BD000030B59DB005466878E9
:10DAE0001E490978884201D11DB030BD68781B49B4
:10DAF0000870022400BF285D052800DA2AE0285DAE
:10DB0000401FC0B28DF86300601C28440068199063
:10DB1000601D285C8DF868005D210DF10600FAF7A4
:10DB20005EFB9DF86320A01D29180DF10600FAF791
:10DB30002FFB00F09BFF1B900020ADF8700001A8A8
:10DB4000FDF77CFB01A8FDF736FB285D401C044473
:10DB500000BFD0E700BF00BFC6E70000D805002027
:10DB600000B5ADF2044D0548416801A8884710B1E1
:10DB700001A8FFF7B1FF0DF2044D00BD1404002011
:10DB8000F0B589B004460D4624216846FAF727FB14
:10DB900020208DF80000264881690DF1010088479A
:10DBA00037208DF8050094F8600001066120005DC3
:10DBB00001EB00416220005D01EB00216320005D6C
:10DBC000084418B1206ECDF8060002E00020CDF820
:10DBD00006008DF80A5094F864008DF80D0094F852
:10DBE0005F000021FFF7BDFC07463A46A11C0DF17E
:10DBF0000E00FAF7CDFA2846FFF758FC07463946DB
:10DC0000A01CFFF77DFD064630128DF80B00F0B228
:10DC10008DF80C0000F06CFF07469DF800100548D9
:10DC20003A46836A0DF10100984709B0F0BD000043
:10DC300048030020B802002070B504460D46FF20BE
:10DC400020702946024800F075FD0646304670BD3A
:10DC5000CC05002010B504462146024800F094FD92
:10DC600010BD0000CC05002010B5024800F0A2FD58
:10DC700010BD0000CC05002003480449086048603E
:10DC80000020088170470000C4050020CC0500205A
:10DC9000002008E0FF21C0EBC002044B03EB02129E
:10DCA0001170411C88B26428F4DB7047F4670020CF
:10DCB00070B504460D462A462146024800F07EFD16
:10DCC00070BD0000CC050020002116E0C1EBC100B2
:10DCD0000C4A02EB00100078FF280CD10120C1EBA8
:10DCE000C102084B03EB02121070C1EBC1001A46CF
:10DCF00002EB00107047481C81B26429E6DB00206B
:10DD0000F8E70000F467002070B590B006460C46B6
:10DD100015460EB1022000E001208DF800002068B9
:10DD2000CDF801000020ADF805008DF807008DF852
:10DD3000085009216846FBF7BBF910B070BD000020
:10DD400070B54948806F401C4749886700240846E1
:10DD500090F8740020B1012835D002286FD16FE00F
:10DD6000FFF782FF10B9FFF7FBFE7AE000253E497E
:10DD7000487800F03FFC051E0DD1FFF775FF3A49CA
:10DD80004978491CC9B2384A5170884202DC0020E7
:10DD90001146487065E070213348001DFAF71FFAFC
:10DDA000702229463048001DFAF7F2F900202E496A
:10DDB000C87091F86300FFF7AFFB2B498870012012
:10DDC00081F8740000BF2849C878FFF747FE26484D
:10DDD000C078401CC0B22449C870897888422CDBC6
:10DDE000214890F87C00401CC0B21F4981F87C009B
:10DDF0000A280FDB002081F87C000124022081F832
:10DE000074001A48816B022088470C20164981F85B
:10DE10007D0013E0FFF728FF13494978491CC9B278
:10DE2000114A5170884202DC0020114648700124DA
:10DE300000200D4981F8740000E0012411E00FE09A
:10DE40000224094890F87D1090F87D00401E064A93
:10DE500082F87D0019B90020114681F8740000E0B5
:10DE600000BF00BF204670BDB493002048030020CF
:10DE700033B581B00D460122694601A8FBF7D0FAFF
:10DE8000044614B99DF800003EBD0020FCE72DE9D2
:10DE9000F04104460D46164698463246294620462D
:10DEA000FBF7BEFA074617B90120BDE8F081002054
:10DEB000FBE7002107E048F2782100BF0A1EA1F12C
:10DEC000010399B2FAD1021EA0F1010398B2F2D176
:10DED000704700002DE9F04105460E4619490868D3
:10DEE000C11700EBD1614911174A11601046006853
:10DEF000801D16490860104600688700102001F058
:10DF0000D1FC804610214046FAF769F9002403E06D
:10DF1000305D0F490855641CBC42F9DB002403E066
:10DF2000285D0C490855641C102CF9DBFBF74CFCF0
:10DF3000FBF750F8102208494046FAF729F9404605
:10DF4000BDE8F0814806002044060020400600207D
:10DF5000EDAB002081AA002091AA002070B52048D6
:10DF6000807900B970BD1E4A9288152A01DC012211
:10DF700017E01B4A9288A2F11501CA1701EBD26281
:10DF80005211521C164B9B88A3F11500C31700EBCE
:10DF9000D3635B11A0EB43130BB1012300E000231B
:10DFA0001A44D5B20F49C86E804740F080040D482E
:10DFB000016F2046884700F019F80B49D1F880001E
:10DFC0008047012408E0204600F07CF80649D1F89B
:10DFD00080008047601CC4B2AC42F4DB00BFC1E7E4
:10DFE0001C04002048030020B802002030B589B08E
:10DFF00024216846FAF7F3F820208DF800002E4817
:10E0000081690DF10100884734208DF805002B4A05
:10E010009288152A01DC012217E0284A9288A2F191
:10E020001501CA1701EBD2625211521C234B9B8877
:10E03000A3F11500C31700EBD3635B11A0EB4313EF
:10E040000BB1012300E000231A44D2B28DF8062060
:10E050009DF80620521E152303EB421291B2174A77
:10E060001268101DFFF74CFB044620128DF80700C4
:10E07000E0B28DF808001049886C80478DF80900DF
:10E0800000208DF80A008DF80B000C480068011D77
:10E09000152203A8FAF77CF80948816F0020884709
:10E0A0000549C86A8047054603482946426B6846C9
:10E0B000904709B030BD0000480300201C04002038
:10E0C000B80200202DE9F0418AB00446242101A8BD
:10E0D000FAF785F820208DF80400294A9288152A3D
:10E0E00001DC012217E0264A9288A2F11501CA1725
:10E0F00001EBD2625211521C214B9B88A3F11500F7
:10E10000C31700EBD3635B11A0EB43130BB10123E7
:10E1100000E000231A44D5B20CB9002003E0601ED1
:10E12000152101EB4010C6B20CB915210EE0691E95
:10E13000A1420AD112498988A1F11500C11700EB4B
:10E14000D1614911A0EB411100E02021CFB20C4870
:10E150000068001D81193A460DF10500FAF718F81C
:10E160000848816F002088470749C86A8047804671
:10E1700005484146426B01A890470AB0BDE8F081CE
:10E180001C040020B802002048030020F0B501461E
:10E190000120264AD07110460160C8788A7800EBC9
:10E1A000022080B2214A90801646B688152E01DCE6
:10E1B000012617E01D4EB688A6F11502D61702EB10
:10E1C000D6667611761C194FBF88A7F11500C717C0
:10E1D00000EBD7677F11A0EB47170FB1012700E0D5
:10E1E00000273E44F3B200201CE008B9002203E0FF
:10E1F000421E152606EB4212D4B208B915260EE0CF
:10E200005E1E86420AD1094EB688A6F11502D617BF
:10E2100002EBD6667611A2EB461600E02026F5B298
:10E22000421CD0B29842E0DBF0BD00001C0400208C
:10E2300010B50748807900B910BD0649C86E8047FF
:10E2400040F080040348016F2046884700BFF3E791
:10E250001C0400204803002070B5044612480068E2
:10E2600000B970BD7CB91048807960B100200E49BA
:10E27000086088710D49C86E804720F080050B4802
:10E28000016F28468847012C0CD10748C079012826
:10E2900005D100200449C8710120887102E00020E6
:10E2A0000149086000BFDCE71C040020480300208F
:10E2B00010B52C4B1B6883432A4C2360231D1B681D
:10E2C0008343241D2360231D1B688343241D236077
:10E2D000231D1B688343241D236011B101290ED126
:10E2E00005E0204B1B6803431E4C236008E01D4BD8
:10E2F0001B1D1B6803431B4C241D236000E000BF53
:10E3000000BF22B1012A0FD0022A27D119E0154BF4
:10E3100008331B680343134C08342360231D1B6818
:10E320008343241D23601AE00E4B08331B6883438C
:10E330000C4C08342360231D1B680343241D2360F9
:10E340000DE0084B08331B680343064C0834236078
:10E35000231D1B680343241D236000E000BF00BF92
:10E3600010BD000000040140014908607047000032
:10E370001404014001460748006800EA010205480C
:10E380001438006800EA010312B10BB10120704794
:10E390000020FCE7140401400448006820B1034851
:10E3A0000068401E014908607047000034040020E6
:10E3B0000348006808B1012070470020FCE7000016
:10E3C000340400201CB5044620791D2817D160793B
:10E3D00008B90A2000E06079094908600846006829
:10E3E000322148430649086020798DF800006079A1
:10E3F0008DF80100022269460B2002F0FBFB1CBDD8
:10E400003404002070B504466079282819D1A07919
:10E4100000B970BD012015490870607A217A00EBBF
:10E42000012012494880A079012802D100204870BB
:10E4300002E051200D4948700D49D1F8A0008047F5
:10E4400012E00A48007878B10020084908700949AC
:10E45000C86A804705460749886A804706460648D5
:10E460002946C26A3046904700BFD2E770050020B7
:10E470004404002048030020B802002070B5044680
:10E480002848007808B9002070BD27480078B8B93E
:10E490002649C86A80470546224948782449CA6AFD
:10E4A000294690470120A0722049886A8047E0727F
:10E4B0001C484088001220731A488078607323E05B
:10E4C0001A49C86A804706461849886A804705463F
:10E4D00017483146C26A28469047164890F87A0095
:10E4E00068B10120A0721149886A8047E0720D4826
:10E4F0004088001220730B488078607304E000208D
:10E50000A072E072207360730A48D0F89C10204615
:10E5100088470548007880F0010003490870012011
:10E52000B2E70000700500207605002048030020B7
:10E53000B80200204404002008B50F208DF8000028
:10E54000044800798DF80100022269460B2000F092
:10E5500003F808BD7005002070B590B004460D4664
:10E56000164640216846F9F73AFE1F208DF8000054
:10E57000E1208DF801000949C86980478DF8020043
:10E580008DF803403246294601A8F9F701FE0348F9
:10E59000416C6846884710B070BD000048030020F9
:10E5A0004179014A117170477005002001480078D7
:10E5B000704700007005002001460D48007808B93A
:10E5C000002070470A48408800280EDD48780A7805
:10E5D00000EB0220064A5288904206D10448408847
:10E5E000401C034A50800120EBE70020E9E70000CF
:10E5F0007005002070B5054600242846FFF72AFB69
:10E60000041E25D000F032FAA16E884204D300F037
:10E610002DFAA16E401A03E000F028FAA16E081A44
:10E620000646B6F5487F0DD304F16000FCF7B2FD55
:10E6300030B194F8642004F160010020FFF764FB1E
:10E64000002070BDB4F86C00401CA4F86C0000BF42
:10E650002046F6E710B5002821D0114B0022001FFC
:10E66000196803E0814203D80A4649680029F9D1B4
:10E6700052B11368841A9C4204D100681844106097
:10E68000104602E0506000E0186039B102680B1AD1
:10E69000934203D10B681A4402604968416010BD7F
:10E6A000940600207FB5044626796579B54200DDE1
:10E6B0007FBD012D01DB142D00DDF9E7012D03D114
:10E6C000A9021A48F9F78BFD691E01EB011101EB54
:10E6D0004101164A8818332204F10801F9F758FD60
:10E6E00020798DF8000060798DF80100A0798DF80F
:10E6F0000200E0798DF80300B54211D10B48007893
:10E70000012802D0032809D103E0084801F06AF883
:10E7100005E0074801680548884700E000BF00BFE2
:10E720000421684602F086FA00BFC1E7C43E00201B
:10E73000240400202DE9F04104460E462089B04211
:10E7400002DA0020BDE8F0810E490868804725689C
:10E75000002002E06D68411C88B2B042FADB6F68AD
:10E76000686840686860D7F800803846FFF772FF35
:10E77000208910B12089401E2081024948688047C5
:10E780004046DFE7B802002010B502460B4610896C
:10E79000984201DA002010BD10684168002002E0B4
:10E7A0004968441CA0B29842FADB09B10868F2E754
:10E7B0000020F0E701460889704700002DE9F0418C
:10E7C0000546884617462889B84202DA0020BDE887
:10E7D000F081134908688047082001F063F8044677
:10E7E00004E00F49486880470020F0E7002CF8D08B
:10E7F00000206060C4F800802E6800BF02E07668E8
:10E80000411C88B2B842FADB7068606074600449E9
:10E81000486880472889401C28810120D7E70000EC
:10E82000B802002001468888704700002DE9F041B9
:10E8300004460E461449086880472088618888424B
:10E8400006D1A088A189884202DB4FF0FF3515E090
:10E850006388E789A16803FB07103A463146F9F758
:10E8600097FC6088401CA18990FBF1F201FB12002B
:10E870006080A088401CA080A08805B2024948683A
:10E8800080472846BDE8F081B80200202DE9F0411C
:10E8900004460E46134908688047208861888842EC
:10E8A00004D1A08810B94FF0FF3515E02388E7891F
:10E8B000A06803FB07013A463046F9F769FC208857
:10E8C000401CA18990FBF1F201FB12002080A0887E
:10E8D000401EA080A08805B20249486880472846AB
:10E8E000BDE8F081B802002010B520211448F9F7E6
:10E8F00076FC2022134912482030F9F749FC002405
:10E900000AE00F482030005D0F49095D48400C497E
:10E9100020310855601CC4B2202CF2DB0023084AC9
:10E920003032074901F12000FAF772FC0023044A53
:10E930002032A2F1100101F12000FAF769FC10BDAC
:10E940003B4B0020BD390108083A01080146014847
:10E95000405C7047083B010810B50446202202497C
:10E960002046F9F715FC10BD5B4B0020044890F8D9
:10E97000900008B90020704702480078FBE70000CB
:10E9800044040020384B00200148407870470000C4
:10E99000C303002001484078704700005808002059
:10E9A0000148007970470000EC10002010B50446C3
:10E9B0000B484078032803D009484078062808D13E
:10E9C000AA202070BB206070CC20A070DD20E070F9
:10E9D00004E004222146034800F0ABFF10BD000014
:10E9E00058080020CC030020014800787047000040
:10E9F000E010002017488078282803D10420164909
:10EA0000C87224E01348807810280FD11248C07AC9
:10EA1000032807D01048C07A022803D002200E49EC
:10EA2000C87214E003200C49C87210E009488078CD
:10EA300018B101200849C87209E00648807818B961
:10EA400005200549C87202E000200349C872024847
:10EA5000C07A7047F40700209C0700200421017051
:10EA60000221417000218170704700000148806FD1
:10EA700070470000B493002010B5054890F874006A
:10EA800020B9FFF7F1F808B9002010BD0120FCE71C
:10EA9000B49300200148407870470000F40700203C
:10EAA00030B501460022002010E00B4C235C03EB44
:10EAB00043040A4D05EB4404A478082C04DD441CEF
:10EAC000E5B2541C0D55E2B2441CE0B2024C647A2B
:10EAD0008442EADC0A7030BDEC1000209C1100205A
:10EAE0000148007870470000E803002000207047CC
:10EAF0000148007870470000EC100020014601EB4F
:10EB00008100400070470000F0B503460C46062522
:10EB10001F201E781D2E46D2DFE806F0450F1C1E72
:10EB20002124274545452A2C2F3145454545454556
:10EB300034383C454545454041001E4EB67806F008
:10EB40007F06052E03D1042107261E7001E008214F
:10EB500003252BE0042129E002210C2526E00121D8
:10EB6000172523E00221092520E0012115251DE0BC
:10EB700004211BE00121162518E0042116E00221E2
:10EB80000B2513E0032110253C200FE00321102565
:10EB90003C200BE001211B253C2007E000BF0221A7
:10EBA0001A253C2002E00121162500BF00BF21707C
:10EBB0001570F0BDF4070020014800787047000090
:10EBC0009C07002001480079704700009C07002046
:10EBD0000348017B0020024A10730846704700007A
:10EBE0009C0700201EB50146002009E083061A0E8E
:10EBF000084B1344D3F8E8374DF82030431CD8B203
:10EC00000328F3DB009B0B60019B4B60029B8B6036
:10EC10001EBD000000F0FF1F014800787047000093
:10EC20004003002000BF04488078052801D101205E
:10EC300070470020FCE700009C0600200248C07AD4
:10EC40000149085C70470000EC10002041617047EA
:10EC50000161704710B54FF4807303221021024800
:10EC600000F050F810BD00000008014010B500226F
:10EC70008B071C0F0F2303FA04F204290EDA204B32
:10EC80009B6893431E4CA36023469B688C07240F0C
:10EC900000FA04F423431A4CA3602FE008290EDA8B
:10ECA000174BDB689343164CE3602346DB688C0705
:10ECB000240F00FA04F42343114CE3601EE00C29F6
:10ECC0000EDA0F4B1B6993430D4C236123461B69DE
:10ECD0008C07240F00FA04F42343094C23610DE050
:10ECE000074B5B699343064C636123465B698C0762
:10ECF000240F00FA04F42343014C636110BD0000AB
:10ED000000000140F0B5044616460025002201F03F
:10ED10000F0501F0100747B1042E05D145F003059A
:10ED2000E76B1F43E76300E0354300201EE0012747
:10ED300087401F40C7B122684FEA800C0F2707FAAF
:10ED40000CF7BA43870005FA07F73A43282904D19C
:10ED5000012787401F40676105E0482903D101274B
:10ED600087401F4027612260471CB8B20828DED3C5
:10ED7000082022E0012787401F40E7B16268A0F128
:10ED800008074FEA870C0F2707FA0CF7BA43A0F1E0
:10ED90000807BF0005FA07F73A43282904D10127DD
:10EDA00087401F40676105E0482903D1012787405C
:10EDB0001F4027616260471CB8B21028DAD3F0BD4B
:10EDC00002469068084008B1012070470020FCE727
:10EDD000002101E04A1C91B28142FBDB7047000038
:10EDE00070B50024FBF708F900251BE06006040E4F
:10EDF0004FF480711A48FFF72BFF0520FFF7E8FF5B
:10EE00004FF400711648FFF7DBFF08B144F001042E
:10EE10004FF480711248FFF719FF0520FFF7D8FF64
:10EE2000681CC5B2082DE1DBFBF7FEF84FF400715A
:10EE30000B48FFF70BFF0520FFF7CAFF4FF4807167
:10EE40000748FFF705FF0520FFF7C2FF4FF4807169
:10EE50000348FFF7FBFE0520FFF7BAFF204670BD11
:10EE6000000C014070B50546FBF7DEF8002427E0F2
:10EE700005FA04F000F0800040B14FF4007128481A
:10EE8000FFF7E6FE0520FFF7A3FF07E04FF4007150
:10EE90002348FFF7DBFE0520FFF79AFF4FF4807150
:10EEA0001F48FFF7D5FE0520FFF792FF4FF4807152
:10EEB0001B48FFF7CBFE0520FFF78AFF601CC4B29A
:10EEC000082CD5DBFBF798F84FF480711448FFF756
:10EED000BFFE0520FFF77CFF002413E04FF4007114
:10EEE0000F48FFF76DFF58B94FF480710C48FFF7DA
:10EEF000ADFE0520FFF76CFFFBF796F8012070BD13
:10EF0000601CC4B2642CE9DB4FF480710448FFF745
:10EF10009DFE0520FFF75CFFFBF786F80020EEE77B
:10EF2000000C014010B54FF400710F48FFF790FE40
:10EF30000520FFF74DFF4FF480710B48FFF788FE67
:10EF40000520FFF745FF4FF400710748FFF77EFEED
:10EF50000520FFF73DFF4FF480710348FFF776FE71
:10EF60000520FFF735FF10BD000C014010B54FF430
:10EF700000710F48FFF76AFE0520FFF729FF4FF4E5
:10EF800080710B48FFF764FE0520FFF721FF4FF467
:10EF900000710748FFF75CFE0520FFF719FF4FF4EB
:10EFA00080710348FFF752FE0520FFF711FF10BDE7
:10EFB000000C014030B50B46002100BF16E00A24CA
:10EFC000B4EB107F05D9302404EB107403F8114022
:10EFD00005E0412404EB10740A3C03F811400001E1
:10EFE00000254C00641C1D554C1CE1B29142E6DB2F
:10EFF00030BD704710B50849D1F8B000804708B15E
:10F00000002010BD044890F8850008B90020F8E7FA
:10F010000248C07DF5E70000440400209C07002062
:10F02000F0B591B004460F464D4890F8800028B1E5
:10F030004C48407810B9002011B0F0BDA0780C28E1
:10F0400007D1607A042804D14548D0F8D0100120B7
:10F0500088474348007808B3FFF79CFC082803D092
:10F06000FFF798FC092819D13D4890F87F0010B1AE
:10F070003D48C07820B13D49086A8047082806D13C
:10F080003748C168E01C884708B90020D4E73448F5
:10F0900041692046884708B10020CDE7A0780428C0
:10F0A00005D1162625781B2D25DD1B2523E0A0780C
:10F0B000092802D11C261B251DE0A078072802D0B4
:10F0C000A078082802D11B261B2514E0A078202850
:10F0D0000CD1274841682046884728B13A46042188
:10F0E000E01C00F02DF9A7E70020A5E715262578FC
:10F0F000102D00DD10258DF804602A460DF1050164
:10F10000A01C00F016FC607C012814D11449D1F831
:10F1100000018047227CE17B02EB0121884204D080
:10F120000F49D1F80001804758B901A804F0E4F86C
:10F1300038B9002080E701A804F0DEF808B9002003
:10F140007AE73A460421E01C00F0FAF808B90020FA
:10F1500072E70348416A04F10F00884701206BE71A
:10F1600044040020D0030020D203002048030020E4
:10F17000240600202DE9F04391B005460E464FF0DD
:10F1800003090022402101A800F0DEFB05274FF013
:10F1900004082879242857D2DFE800F0121C1E202A
:10F1A0002428565656565656565656494E56565674
:10F1B0002C2D2E2F30313233345656565639434487
:10F1C0003E4880780E2803D10D244FF0090800E056
:10F1D0000A243DE001243BE0022439E04FF00A0814
:10F1E000032435E04FF00708052431E04FF0140800
:10F1F00006242DE000BF00BF00BF00BF00BF00BF5E
:10F2000000BF00BF4FF015080424042720E00C24A1
:10F210004FF00308052702208DF807004FF004097E
:10F2200016E000BF4FF004080C24042710E04FF054
:10F2300004080C2404270BE04FF014080B2420488A
:10F24000416AA81C884703E0002011B0BDE8F083A4
:10F2500000BF8DF80440A8788DF80500E8788DF897
:10F26000060001AA02EB0901E819424600F061FB21
:10F2700028790F2802D101208DF80700287922284B
:10F2800002D02879232809D19DF807001F2805DB23
:10F290009DF807001F38C0B28DF8070001A804F0E0
:10F2A0002BF808B90020D0E732460221A81C00F054
:10F2B00047F808B90020C8E70120C6E7F407002096
:10F2C0004404002070B500241BE0002104EBC400BE
:10F2D00000EB44120E48815400250EE004EBC401FB
:10F2E00001EB44120A491144491C01EB850000223C
:10F2F000042100F029FB681CC5B20A2DEEDB601C5E
:10F30000C4B203480C38407AA042DEDC70BD000075
:10F31000F8100020014688780B280AD1487A032883
:10F3200007D10548D1F8032002600120034A10707C
:10F3300070470020FCE700008905002088050020B8
:10F340002DE9F04105460F461446062F02DD002048
:10F35000BDE8F081042C01DB0020F9E731490868A1
:10F36000804704EBC40000EB44112F48465C0A2E92
:10F3700052DA04EBC40000EB44122B481044401C4A
:10F3800000EB86013A46284600F0D3FA274890F869
:10F390007A0050B1297A04EBC40000EB44122248F1
:10F3A0001044401C00EB86000171A87B012825D188
:10F3B0001E49D1F8000180476A7B297B02EB0121BD
:10F3C000884204D01949D1F80001804758B90B216F
:10F3D00004EBC40000EB441213481044401C00EB43
:10F3E000860001710AE00A2104EBC40000EB44121C
:10F3F0000D481044401C00EB8600017104EBC40072
:10F4000000EB44110848405C401CC1B204EBC4004E
:10F4100000EB4412044881540249486880470120A7
:10F4200096E70000B8020020F810002044040020F5
:10F430002DE9F04106468848C1683046884708B142
:10F44000BDE8F0817078042800DAF9E78349086B99
:10F45000804728B98148816E701C884700B1EFE76A
:10F460007E48D0F8A810701C884700B9E8E73078CB
:10F47000FEF730F90746FF2800D1E1E7741CFFF7DB
:10F48000B9FD002847D06079912808D0607992288A
:10F4900005D06079932802D0607994283BD16F48D9
:10F4A00090F8850002280BD1207FE17E00EB01203F
:10F4B00085B21621601DFEF723F9A8422AD0BFE7C6
:10F4C000664890F88500032817D1207FE17E00EB85
:10F4D000012085B21621601DFEF712F9A84219D04D
:10F4E00094F82000E17F00EB012085B21A21601D15
:10F4F000FEF706F9A8420DD0A2E794F82000E17FBC
:10F5000000EB012085B21A21601DFEF7F9F8A84230
:10F5100000D095E700BF6079912814D060799228D7
:10F5200011D0607993280ED0607994280BD04B4885
:10F5300090F8340038B14948016C2046884710B132
:10F5400002F008F87CE7454890F87E0048BB6079F7
:10F55000932802D1A0790E2819D0FFF71BFA0328AF
:10F5600015D0FFF717FA062811D03C48007838B1BB
:10F57000FFF710FA08280AD0FFF70CFA092806D07E
:10F5800004223749601C00F0C3F900B958E720781D
:10F59000001FC2B2611C601D00F0CBF92078001F73
:10F5A00020706078802800DA4AE701F0D3FF6078A5
:10F5B000912804D139462046FFF7DCFD49E0607808
:10F5C000922804D13946204600F058F841E02348FB
:10F5D00090F87A0050B16078932802D0607894282F
:10F5E00004D139462046FFF71BFD32E06078B7288A
:10F5F00004D11C48C168204688472AE02078182892
:10F6000015D16078A178884211D16078E17888427C
:10F610000DD160782179884209D16078617988427A
:10F6200005D111480068401C0F49086008E70B48E5
:10F63000D0F8E81020468847084890F8340028B1F0
:10F640000648016C2046884700B1F9E6204600F0E4
:10F6500067F800BFF4E60000240600204404002000
:10F66000CC030020DC050020E403002010B5044694
:10F670002046FFF7DDFE012010BD000030B589B047
:10F6800004460D46A0780C2807D1607A042804D1DE
:10F690001148D0F8D0100120884714208DF80400BC
:10F6A00010220DF10501A01C00F043F901A803F0A0
:10F6B00023FE10B9002009B030BD2A460621E01C07
:10F6C000FFF73EFE08B90020F5E70348416AE01D58
:10F6D00088470120EFE700004404002010B592B0F5
:10F6E0000D490868804740230A2201A90B4801F010
:10F6F00015FD044608494868804714B9002012B037
:10F7000010BD9DF80400801CC0B28DF8040001A853
:10F71000FDF7B4FB0120F2E7B8020020BC11002085
:10F7200010B5044640230A222146024801F0C0FCDD
:10F7300010BD0000BC11002010B541230F2202496A
:10F74000024801F0E3FC10BDE40C0020D80C0020BE
:10F7500010B50446012C04D104210848FFF776FABD
:10F760000AE0022C04D104210448F9F7DEFD03E08D
:10F7700004210248FFF76CFA10BD000000080140A8
:10F7800010B50446012C04D102210848FFF75EFAA7
:10F790000AE0022C04D102210448F9F7C6FD03E077
:10F7A00002210248FFF754FA10BD00000008014092
:10F7B000704710B5044600F00DF840B1204600F047
:10F7C0001BF8002801DA002010BD0120FCE7002012
:10F7D000FAE7000010B50248FFF724F810BD00005A
:10F7E0000404002010B5044621460248FFF71EF825
:10F7F00010BD00000404002010B504462146024854
:10F80000FFF744F810BD000004040020704700001A
:10F810004FF40041080301F0AFF872B601F0A8FD03
:10F820001A491B48FEF70CF81A4A1B49184803F0FE
:10F83000C1F901F025F8FFF70DFA02F08DFBF9F799
:10F8400009FD00BF1248D0F8AC008168012088474C
:10F8500005200F49887000BFF9F788FD0F494868F7
:10F8600080470F49D1F89400804762B6FAF7F4FC5C
:10F87000FAF748FD00BF064880780328FBD104E072
:10F8800006498868804700F02BFAF9E7000000205D
:10F890009C0600208C0200207C02002048030020EF
:10F8A00044040020F0B50B30154D20F00701002472
:10F8B000144A0FE003688B420BD38B4205D95E1AC2
:10F8C00043184768C3E9006700E04368136002C05B
:10F8D00004E0021D10680028ECD12046002802D167
:10F8E000286808B10020F0BD064A07481060074AA2
:10F8F000121A22F00702C0E9002401202860D7E78D
:10F90000980600209406002014AC002010B00020BF
:10F9100030B503460C46002107E0585C655CA84200
:10F9200001D0002030BD481CC1B29142F5DB01205E
:10F93000F8E710B50346002003E01C5C0C54441C9F
:10F94000E0B29042F9DB10BD10B50346002002E0A2
:10F950001A54441CE0B28842FADB10BD30B591B0B5
:10F9600004460D46402101A8F8F739FC1F208DF808
:10F970000400E1208DF805000B49C86980478DF827
:10F9800006000A208DF807002A46214602A8F8F74B
:10F99000FFFB0549886D804718B10348416C01A8F9
:10F9A000884711B030BD00004803002000B589B081
:10F9B0003A4890F8600008B909B000BDFDF7F2FDC3
:10F9C000012802D0022865D151E03548C0780028CE
:10F9D00040D033480079314991F87510884218DDDC
:10F9E00000202F49C87003208DF804002D49886A33
:10F9F00080478DF805004D208DF8060014208DF805
:10FA0000070005208DF80800052101A8FFF7A6FFD3
:10FA10002CE023484079401C214948710846007970
:10FA2000401C087108464079002806DD08464079E8
:10FA30001A4991F87510884202DD01201849487171
:10FA400000201749087048700A465079154A516AD3
:10FA500088470BE003208DF804001249886A80472C
:10FA60008DF80500022101A8FFF778FF13E00C488C
:10FA7000C07800B9A0E700200949C87004208DF8BB
:10FA80000400084640798DF80500022101A8FFF71F
:10FA900065FF00E000BF00BF00BF8DE74404002009
:10FAA000810500204803002010B50446184890F84E
:10FAB000600008B9002010BD6079102805D11549F3
:10FAC000886A8047217A884214D06079132802D04E
:10FAD0006079142805D10F49886A8047A17F884240
:10FAE00008D06079172810D10A49886A8047E17FD9
:10FAF00088420AD108484078FA2804DA0648407853
:10FB0000401C054948700120D5E70020D3E70000DC
:10FB100044040020480300208105002010B504465D
:10FB2000A0B2FDF715FC10BD10B504464F48D0F843
:10FB30002404B8B94FF484614C48801CF8F74FFB9B
:10FB4000A0794A49C1F82804217AE07901EB001034
:10FB50004649C1F83004217AE07901EB001098B1F0
:10FB6000012010BD217AE07901EB00103F49D1F866
:10FB70003014884201D10220F3E7217AE07901EBC9
:10FB800000103A49C1F830043848D0F82404303025
:10FB9000B0F5846F12D90020344948704FF4846165
:10FBA0003248801CF8F71BFB00203049C1F82404C0
:10FBB000C1F82804C1F82C040320D2E72B48D0F860
:10FBC0002C04401C2949C1F82C040846D0F82C0408
:10FBD000D1F82814884212D90020244948704FF4E3
:10FBE00084612248801CF8F7FAFA00201F49C1F806
:10FBF0002404C1F82804C1F82C040420B1E71B49EF
:10FC0000D1F82424891C5018302204F10901F8F796
:10FC1000BFFA1648D0F8240430301449C1F824043F
:10FC20000520134908801148D0F83004401C0F49C2
:10FC3000D1F82814884216D30C48D0F824040B4974
:10FC4000C1F8340401204870084690F82304401C91
:10FC500081F823040020C1F83804012081F83D0414
:10FC600000200349088000207BE70000F8460020C0
:10FC70007805002010B51749086D8047052801D088
:10FC8000002010BD1448407808B90020F9E7134857
:10FC9000407907280BD1002010494871012000F05D
:10FCA000BFF80B200C4981F83C040120E9E70A4821
:10FCB000D0F83804401C0849C1F838040846D0F888
:10FCC0003804B0F5967F03D900204870C1F8380495
:10FCD0000020D6E748030020F8460020BD0300209E
:10FCE00010B51348007800B910BD114890F83D04D4
:10FCF00090B100200E4981F83D040846811CD0F8DF
:10FD000024240C48F8F744FA00200949C1F82404D7
:10FD1000C1F82804C1F82C04064800F025F8022098
:10FD2000FCF734FE00200249087000BFDCE7000049
:10FD3000F8460020D44200200A4890F83C0480B1E4
:10FD4000084890F83C040B2803DD0B20054981F896
:10FD50003C04044890F83C04401E024981F83C04ED
:10FD600000BF7047F846002070B58AB005462821CC
:10FD70006846F8F734FA0026002427488169684667
:10FD80008847FE208DF8040048208DF80500DE200D
:10FD90008DF806009E208DF807002048B0F8340446
:10FDA0001F30C0F347108DF8080001208DF80900BE
:10FDB0009DF8080041012846FDF7A2FC06463012D6
:10FDC0008DF80A00F0B28DF80B00144890F8230467
:10FDD0008DF80C0013210DF10D00F8F700FA202129
:10FDE000684600F023F800F037F8C820FFF796FEC9
:10FDF0000BE02819202100F019F800F02DF832202E
:10FE0000FFF78CFE04F1200084B20448D0F83404DB
:10FE1000A042EED80AB070BD48030020F84600208A
:10FE20000149087070470000F846002070B505468B
:10FE30000C46002001F066FF0549C86A8047064667
:10FE4000E1B204483246836A28469847012070BDD3
:10FE500048030020B802002010B54FF4FA7408E0FF
:10FE6000FEF7DAFE00B110BD0220FFF757FE601E5C
:10FE700084B2002CF4D100BFF5E7000070B5012575
:10FE8000002035494872002415E0FF20324908550A
:10FE90003248005DFF2807D03048005DFE2803D0BF
:10FEA0002E48005DFB2804D12B48407A401C2A498B
:10FEB0004872601CC4B2042CE7DBFF202649C872DC
:10FEC00000241FE02548005DFB280FD0FE2807D046
:10FED000FF2813D12048047000201F4988720EE0CB
:10FEE0002846691CCDB21C490C5408E01A48C5725A
:10FEF0002846691CCDB218490C5400E000BF00BF71
:10FF0000601CC4B2042CDDDB002406E0124A105D44
:10FF1000134AD16B8847601CC4B20F48407AA04294
:10FF2000F4DC104880780C49497A884203DD0A489D
:10FF3000407A0C49887001F0EBFE0B48808D48B187
:10FF4000FEF7D6FD06460849888D054932460B6CFA
:10FF50000421984770BD0000EC100020BA04002076
:10FF6000B8020020D60300209C07002070B51E4870
:10FF7000407A012800DC70BD1C49086B804700B145
:10FF8000F9E71B480078401CC0B2194908700A28DC
:10FF900000DAF0E700201649087001F05FFD124812
:10FFA0000578002405E01049601C085C0855601CB9
:10FFB000C4B20D48407A401EA042F4DC0A48407AA0
:10FFC000401E09490D54002408E0074B195D1B1D14
:10FFD000185D084BDA6A9047601CC4B20248407A48
:10FFE000A042F2DC00BFC6E7EC1000204404002071
:10FFF000FC030020B802002030B589B0044624215B
:020000040801F1
:100000006846F8F7ECF820208DF800002C4881694C
:100010000DF10100884728208DF805002948006867
:10002000807928490968497900EB0120000A8DF898
:10003000060024480068807922490968497900EB64
:100040000120C0B28DF807001E48006800680290C9
:100050001C48006800798DF80C0020128DF80D0006
:10006000E0B28DF80E0017480068C0798DF80F00D7
:1000700014480068007A8DF8100012480068807BF0
:1000800010490968497B00EB0120000A8DF8110036
:100090000C480068807B0B490968497B00EB012014
:1000A000C0B28DF81200FEF723FD05469DF8001042
:1000B00005482A46836A0DF10100984709B030BD12
:1000C0004803002020060020B802002070B5044636
:1000D000002500F04FFA051E00D170BD1122214607
:1000E0002846F8F755F8A08AA88200F011FA0646CB
:1000F0003146284600F032FA0120EEE72DE9F041C2
:1001000006460F46002411E0204600F0F7F9051ED0
:1001100000D10FE0042231462846F8F76BF818B9F1
:10012000AC742846BDE8F081601CC4B200F0F0F960
:10013000A042E9DC00BF0020F4E7000070B50546EE
:100140002878FDF7C7FAFF2801D1002070BDAC1C4C
:10015000042225492046FFF7DBFB18B320798F28BE
:100160001ED16079DE281BD1A079482818D1E0790A
:10017000FE2815D1207A082801DD082000E0207A29
:100180001A49087000201A4908700120194908709E
:100190000F2204F108011848F7F7FAFF0120D5E70C
:1001A0000020D3E713480078E0B111490978124ADA
:1001B0000F3202EB411020222146F7F7E9FF0C48ED
:1001C0000078401CC0B20A49087008490978884282
:1001D00006DBFBF7EFFB09490872002005490870B0
:1001E0000120B3E70020B1E7CC0300203E06002049
:1001F0003D0600203C06002072A9002064A50020D6
:1002000030B587B0054601AC1122E91C2046F7F74E
:10021000BFFF0020A082607A0106A07A01EB0041B6
:10022000E07A01EB0021207B084410B9002007B0E0
:1002300030BD21792046FFF761FF38B92046FFF72E
:1002400045FF08B10120F2E70020F0E70120EEE7CA
:1002500030B5ADF20C4D9E48407930B101286ED0DA
:1002600002287DD003287CD11CE100F051F9002840
:1002700062D0FCF727F900285ED09549087900F094
:100280003DF99449086080B900F042F99049097934
:10029000491CC9B28E4A1171884202DC0020114605
:1002A000087100200DF20C4D30BD8A480068407A7C
:1002B000010688480068807A01EB004185480068A3
:1002C000C07A01EB002183480068007B014481482B
:1002D0000068807B7F4A1268527B00EB022091FB12
:1002E000F0F17C480068407A02067A480068807A1B
:1002F00002EB004277480068C07A02EB00227548A2
:100300000068007B024473480068807B714B1B6867
:100310005B7B00EB032092FBF0F300FB132008B1A2
:10032000012000E00020084469490880012048803D
:1003300048710020488101E00020B3E700BF644815
:10034000B0F80C04401C80B26149A1F80C042828C4
:1003500008DB0020A1F80C04032048710020A1E76D
:1003600010E0B1E05A494888FFF746FE002058499E
:1003700008720420C88008464089401C4881022039
:100380004871A2E05248007A012812D150484088B2
:10039000401C80B24E4948800988884203DC012015
:1003A0004B49487104E000204949488001204871C8
:1003B0008BE04748007A022844D16C4645480068E3
:1003C00050F8071F616080882081424800680068FB
:1003D000206040480068807B3E490968497B00EB0B
:1003E00001203B490988484385B2B5F5806F01DD9E
:1003F0004FF480652A4636490C3104F10A00F7F7BC
:10040000C7FE29462046FBF73BFF88B932480078F3
:100410000A280BDA31483049097800EB810021685D
:1004200001602D480078401C2B490870002039E7F6
:10043000274801792748006800F052F80020244935
:10044000487142E000BF2248C088401E80B2204967
:10045000C88030BB08464089642802DA0120487110
:100460001FE01C480068808A401C80B21949096856
:1004700088820A2805DB164801791648006800F0D2
:100480002FF800F045F812490979491CC9B2104A01
:100490001171884202DC00201146087100200C49CD
:1004A000487112E00A48B0F80C04401C80B20849B8
:1004B000A1F80C04022806DD0020A1F80C0401209C
:1004C00048710020EEE600E000BF00BF0120E9E631
:1004D00064A50020200600200A06002060A4002059
:1004E00070B504460D46FF20607429460248FEF7A9
:1004F00021F90646304670BD1406002010B50446AA
:1005000021460248FEF740F910BD00001406002005
:1005100010B50248FEF74EF910BD00001406002089
:1005200003480449086048600020088170470000C3
:100530000C0600201406002000200AE0FF2100EB3A
:10054000400202EBC002044B03EB42025174411C17
:1005500088B20A28F2DB704788A4002070B50446F0
:100560000D462A4621460248FEF728F970BD0000D4
:100570001406002000211CE001EB410000EBC1004B
:100580000E4A02EB4000407CFF2810D1012001EB15
:10059000410202EBC102094B03EB4202507401EB32
:1005A000410000EBC1001A4602EB40007047481CB6
:1005B00081B20A29E0DB0020F8E7000088A40020CF
:1005C00010B54FF4C87000F05DF804490870084693
:1005D000007808B93C20087010BD0000A405002078
:1005E00002460C2901DA0020704704488368136032
:1005F000C3685360006990600120F5E7A4050020FE
:100600000148407D70470000A40500200148407863
:1006100070470000A4050020014880887047000052
:10062000A405002070B504461348807D78B10020F1
:10063000114988751149C86A804705460F49886A7B
:10064000804706460E482946C26A304690478CB11C
:100650000948007860B108480078401E06490870D3
:100660000846007830B900F05DF8FFF7A9FF01E017
:10067000FFF7A6FF70BD0000A4050020480300207E
:10068000B80200202DE9F04106461048808B10B9D1
:100690000120F9F775FC0D48808BFA2803DD002056
:1006A0000A49888304E00948808B401C07498883F5
:1006B000B5082846F9F764FC0446281903498969F6
:1006C000471A024884613846BDE8F081A40500203D
:1006D00070B505460C460C2C01DD002070BD22468D
:1006E00029460248F7F754FD0120F7E7AC05002042
:1006F00018B10121034A517502E00021014A5175E8
:1007000070470000A405002002484078401C0149C1
:1007100048707047A4050020014988807047000098
:10072000A405002030B58BB0282101A8F7F757FDAC
:1007300020208DF804004E4881690DF1050088479E
:1007400051208DF809004B4840788DF80A004A483E
:10075000007858B1FEF71EF9082803D0FEF71AF901
:10076000092803D102208DF80B0002E001208DF84A
:100770000B003F49886A80478DF80C0000208DF8F7
:100780000D008DF80E008DF80F008DF810008DF81B
:1007900011003848407D30B19DF8110040F0010053
:1007A0008DF8110005E09DF8110000F0FD008DF8B6
:1007B00011002F49086D8047042806D19DF81100CB
:1007C00040F002008DF8110005E09DF8110000F0E6
:1007D000FD008DF811009DF80B00022806D19DF850
:1007E000110040F004008DF8110005E09DF81100A3
:1007F00000F0FB008DF811001E488088000A8DF87B
:1008000012001C4800798DF8130000208DF81400A8
:100810008DF8150017488168CDF81610C168CDF81D
:100820001A100069CDF81E001B210DF10900FCF71C
:1008300067FF0446200A8DF82300E0B28DF82400FB
:1008400001200C4988750A49C86A804705460B484B
:100850002946C26A002090470549C86A8047054674
:1008600003482946426B01A890470BB030BD0000F9
:1008700048030020A405002044040020B802002002
:1008800010B54FF4806000F06DF8002202211420B2
:1008900000F006F800220121132000F001F810BD3D
:1008A0002DE9F04103460D46164600240027A046D8
:1008B0002A48006800F4E060B0F5E06F03D100BFA3
:1008C0004FF0040830E02548006800F4E060B0F51F
:1008D000C06F03D101274FF0030825E01F480068CF
:1008E00000F4E060B0F5A06F02D10227B8461BE02B
:1008F0001A48006800F4E060B0F5806F03D1032768
:100900004FF0010810E01548006800F4E060B0F511
:10091000407F03D104274FF0000805E04FF4A060AA
:1009200000F020F80227B846C7F1040005FA00F4E9
:10093000C8F104010F20C840304004432401084896
:10094000C45403F01F01012088405911890001F1AE
:10095000E021C1F80001BDE8F08100000CED00E0ED
:1009600000E400E002490143024A116070470000C0
:100970000000FA050CED00E0034A0A400243034B75
:100980001A60BFF34F8F704780FFFF1F08ED00E034
:1009900070B590B004460D461646002240216846C8
:1009A000FEF7D2FF1F208DF80000E0208DF8010037
:1009B000FDF7EAFF8DF802008DF80340324601A9E9
:1009C0002846FEF7B6FF6846FCF758FA10B070BD2F
:1009D00038B50446E07810287ED2DFE800F0F21E39
:1009E000088A249194B29FF2F2BDBEBFECC50E22DC
:1009F0007849201DFEF79DFF0E2276493020FCF736
:100A0000B9FB7448401E407A032805D10922724977
:100A100004F10D00FEF78DFF00BF0E226D4901208D
:100A2000FFF7B6FFD3E020796C494978884204D1BA
:100A300060796A498978884202D0204602F0BCFA7F
:100A4000207966494978884203D0002062490D39EF
:100A50004883607961498978884204D001205E49E1
:100A60000D3981F8220060790E2821D1A07914284F
:100A700002D0A0791E281BD1607958498978884214
:100A800009D1607955498978884211D15348C07895
:100A9000A17988420CD05249D1F8CC008047A07986
:100AA000142810D101204C490D3981F820000AE0AA
:100AB00060790E2802D1A079142804D0002046497C
:100AC0000D3981F820001A224449491C201DFEF7E7
:100AD00030FF4449C86800E073E080471A223F496C
:100AE000491CA020FCF746FB3D48C16920468847C9
:100AF00000BF1A223949491C0320FFF749FF66E06D
:100B000002F0D2FB63E001200090201D02F00CFCFB
:100B1000012269460620FFF73BFF58E0304890F875
:100B20007A0000B953E004222F49201DFEF701FF8F
:100B300004222D49D020FCF71DFB0520FAF773F89D
:100B400000BF274890F87A0000B940E00422264907
:100B50000720FFF71DFF3AE000BF00BF2048D0F894
:100B6000C8102046884732E0207901280DD117228D
:100B70001E49201DFEF7DDFE012017490D3981F8C1
:100B80002300002081F822000FE0207902280CD1F8
:100B900017221749201DFEF7CCFE01200E490D3902
:100BA00081F82400002081F8220001200A490D3933
:100BB00081F8210000BF17220C490E20FFF7E8FE44
:100BC00005E00748D0F8DC102046884700BF00BF8A
:100BD000012038BDCD070020A9070020F407002020
:100BE0004404002024040020BE0300203308002019
:100BF0007508002070B590B004460D4616460022D8
:100C000040216846FEF7A0FE1F208DF80000E1207D
:100C10008DF80100FDF7B8FE8DF802008DF8034055
:100C2000324601A92846FEF784FE6846FCF726F9FD
:100C300010B070BD30B591B005460C46402101A8FA
:100C4000F7F7CDFAF5208DF80400AA208DF80500FD
:100C50008DF8060004F10800C0B28DF80700E1200D
:100C60008DF808000A49C86980478DF809001320EB
:100C70008DF80A00224629460DF10B00F7F788FA95
:100C800004484021826901A8904711B030BD00009E
:100C900048030020B802002030B589B00446E0784F
:100CA0001B2876D2DFE800F0D4360E493C5A4F6359
:100CB000D4767A95999AA5ABACD4D4A6D4D4ADC148
:100CC000D4CAC60007226749201DFEF732FEFAF794
:100CD000F7FEFAF7BDFE6349491E887800F0CCF9AB
:100CE000FDF706FF05465F49491EC8795E490A6B54
:100CF00029469047002508E05A49491EC8795A49B3
:100D00000A6B29469047681CC5B25848407AA842E9
:100D1000F2DC00BF072253490120FFF76BFF9DE083
:100D20000D225349201DFEF704FE00F091FF0D2215
:100D30004F490820FCF71EFA00BF0D224C49032042
:100D4000FFF758FF8AE004224A49201DFEF7F1FD13
:100D5000042248491820FCF70DFA00BF01A8FDF74E
:100D600025FE042201A90520FFF744FF76E00120BB
:100D70008DF804003C48012201A9036A2E209847FF
:100D8000394988688047012201A90720FFF732FF0F
:100D900064E05DE02046FAF7D9F85FE020790128A9
:100DA00002D0207902280DD12079012801D001201C
:100DB00000E000208DF80400012201A90A20FFF7BD
:100DC00019FF05E02079042802D12B49486E80479D
:100DD00044E02046F9F738FF40E03FE0264801A90B
:100DE000C26D20469047092201A90D20FFF702FF9E
:100DF00034E033E021480168204688472EE02DE0AA
:100E00002CE01F48807858B160791E2808D0002057
:100E10001B498870002205211948C01CFEF794FD6B
:100E20001548816B2046884718E0164841692046DE
:100E3000884713E0207900F02FFF00BF1248C07DE3
:100E40008DF80400012201A91920FFF7D3FE05E067
:100E50000948D0F8E0102046884700BF00BF0120B5
:100E600009B030BDC4030020B8020020EC100020FF
:100E70004B080020CC030020440400201404002070
:100E8000F4070020240600209C07002030B593B012
:100E900040230A2202A9214800F040F910B900209D
:100EA00013B030BD9DF80800001DC0B28DF80400DD
:100EB0000DF10500FDF77AFDFDF712FE60B100248B
:100EC00005E0214601A8FBF7A3FF601CC4B214484B
:100ED000007AA042F5DC1FE0124890F884001E283A
:100EE00013D1104890F8850078B11A210DF109004E
:100EF000FCF706FC054628128DF82300E8B28DF8B1
:100F0000240020208DF8040000BFFDF7EFFD05460A
:100F1000294601A8FBF77CFF0120C1E74814002007
:100F2000EC1000204404002070B50446074908680E
:100F3000804740230A222146054800F0B9F80546BB
:100F4000024948688047284670BD0000B80200206A
:100F50004814002070B5044640231122214603485E
:100F600000F0DCF80546284670BD00008C08002023
:100F700010B50446402311222146024800F098F89B
:100F800010BD00008C08002010B54023112202493A
:100F9000024800F0BBF810BD980800208C08002023
:100FA00010B504460D4890F8C40008B9002010BDE3
:100FB000012C07D1FCF718FD08B10020F7E708481D
:100FC000C47409E00648C07C30B100210448C174F3
:100FD00000F016FF0120EAE70020E8E744040020C3
:100FE0007B5B002010B588B00446E078182814D147
:100FF00020791249087060798870F5208DF800001A
:1010000020798DF8010060798DF802000C480322E8
:101010006946036A4FF484609847084800788DF861
:101020000000064880788DF8010002236A461721E7
:10103000612001F097FF08B010BD0000384B002080
:10104000B802002010B504460948847000F060FE24
:1010500006220849F020FCF78DF80A20FCF729FF4A
:1010600007220349491C0020FCF784F810BD00004A
:10107000C3030020D703002010B50446204600F02B
:101080007BFE00F045FE06220749F020FCF772F8CF
:101090000A20FCF70EFF054884700722411C00203F
:1010A000FCF768F810BD0000D7030020C303002040
:1010B0002DE9F0410446884615461E461249086847
:1010C000804720886188884204D1A088A84201DB3B
:1010D000002712E06288A06802FB06013246404603
:1010E000FEF727FC6088401C90FBF5F105FB110022
:1010F0006080A088401CA080012703494868804781
:101100003846BDE8F0810000B802002010B58160CB
:10111000448804800024848010BD00002DE9F04143
:101120000446884617461D461149086880472088AE
:101130006188884203D1A08808B9002612E022887D
:10114000A16802FB05102A464146FEF7F2FB208803
:10115000401C90FBF7F107FB11002080A088401E87
:10116000A08001260249486880473046BDE8F081EA
:10117000B802002070B504460E460A490868804748
:1011800020886188884203D1A08808B9002503E03F
:1011900020887043A1680D5C024948688047284652
:1011A00070BD0000B80200202DE9F04704468846D3
:1011B00017461D46DDF820901549086880472088AD
:1011C0006188884203D1A08808B900261AE02088E7
:1011D0006843A168085C484501D0022612E02288D5
:1011E000A16802FB05102A464146FEF7A2FB2088B3
:1011F000401C90FBF7F107FB11002080A088401EE7
:10120000A08001260249486880473046BDE8F08743
:10121000B80200202DE9F04F8CB0074600200A905C
:101220004AA090E8004CC068CDE905BECDF810A0FA
:1012300007900FF21C1ADAE9000ACDE9020A0FF250
:10124000101ADAE9000ACDE9000A44484068C0F300
:1012500081000B900B9820B1012804D002283FD1C7
:1012600003E03F4A3EE03F4A3CE03C48406800F42F
:10127000803CBCF5803F12D13848C06A00F08048FD
:10128000B8F1000F01D1374B00E0374B33484068CD
:1012900000F40039B9F5003F02D15B0800E0334BA0
:1012A0002E484068C0F383412C48406800F000603D
:1012B00008B141F010012948406800F0804008B1B1
:1012C00041F020010F2901D2891C06E00F2903D328
:1012D0003E2901D8491C00E03F2103FB01F201E057
:1012E0001F4A00BF00BF1D484068C0F3031504A893
:1012F000465D22FA06F419484068C0F3022502A8A8
:10130000465D24FA06F0099014484068C0F3C225EF
:101310001DF8056024FA06F0089037B1012F06D0B9
:10132000022F06D0032F0AD106E00A9208E00A94A1
:1013300006E009980A9003E008980A9000E000BFD0
:1013400000BF0A980CB0BDE8F08F0000000000005C
:101350000000000001020304060708090010024013
:1013600000127A000024F400006CDC0200093D0049
:1013700010B50020FFF74EFF044640F2026000F077
:1013800053F82548844204D14FF4800000F05CF803
:1013900015E02248844203D1002000F055F80EE009
:1013A0001F48844204D14FF4400000F04DF806E09D
:1013B0001C48844203D14FF4000000F045F840F28D
:1013C000026000F031F840F2036000F02DF840F2C6
:1013D000046000F029F840F2056000F025F84FF4B1
:1013E000C06000F021F840F2177000F01DF84FF4D3
:1013F000E06000F019F840F2017000F015F840F2DA
:10140000027000F011F840F20C6000F00DF840F2AC
:101410000F7000F009F810BD006CDC0200A24A0455
:1014200000D8B805000E2707064A02EB901109689C
:1014300000F01F0301229A401143024B03EB90126C
:101440001160704700100240044A516821F44001C5
:1014500041EA0002014B5A60704700000010024050
:101460001CB50B4803226946436A4FF484609847D1
:101470009DF80000F52807D19DF801000549087086
:101480009DF80200887002E00020024908701CBD2F
:10149000B8020020384B00201FB5224810226946B0
:1014A000436A9001984700240EE0C4F10E001DF835
:1014B0000000C4F10F011DF801104840C4F10F01F4
:1014C0000DF80100601CC4B20F2CEEDB1648037847
:1014D000C21C00F123016846F7F704FE11481022F0
:1014E0006946436A4FF48260984700240EE0C4F1D5
:1014F0000E001DF80000C4F10F011DF80110484056
:10150000C4F10F010DF80100601CC4B20F2CEEDB1A
:1015100005480378C21C00F133016846F7F7E2FD85
:101520001FBD0000B8020020384B002010B507484E
:10153000C16C0220884701200549087000204880BE
:10154000012008710020C88010BD0000B8020020F2
:101550009C07002010B50748407A00B910BD002054
:101560000449487288720448016D0020884700BF12
:10157000F4E700009C070020B8020020F0B58DB011
:1015800005464B4890F8900010B901200DB0F0BD11
:101590004848007808B90120F8E72122294604A824
:1015A000F6F7F6FD9DF81500F7F75EFD061E01DD66
:1015B0008DF8156006240DE004A8005D80F0A506F6
:1015C00004A9601C085C80F055000855601C0E548E
:1015D000A01CC4B21F2CEFDB00240DE0C4F11F00DF
:1015E00004A9085CC4F1200104AA515C4840C4F17C
:1015F00020015054601CC4B21A2CEFDB00240CE014
:1016000004F1160004A9085CA11D04AA515C48401D
:1016100004F116015054601CC4B20B2CF0DB1022F4
:101620000DF116016846F6F7B3FDFAF717FE40B163
:1016300020480378C21C0DF116016846F7F752FDE9
:1016400018E09DF815004C2809D01A48037800F1DD
:1016500023020DF116016846F7F744FD0AE015482C
:101660000378C21C0DF116016846F7F73BFD132005
:101670008DF81500212204A92846F6F789FDE87F98
:10168000002803DC95F8200000280FDD1A21681DD2
:10169000FCF736F80746E87FB0EB272F04D1F8B205
:1016A00095F82010884201D000206FE701206DE7F7
:1016B00044040020384B0020F0B589B00546454869
:1016C00090F8900008B909B0F0BD4348007800B91F
:1016D000F9E71A21681DFCF713F807463812E87776
:1016E00085F8207020202870212229466846F6F7C8
:1016F0004FFD6879F7F7B8FC061E01DD8DF805602F
:101700009DF80500412803D09DF8050042280FD11F
:101710009DF8090028280BD14C208DF805002E4893
:101720000378C21C0DF10601A81DF7F771FD14E046
:10173000FAF794FD40B128480378C21C0DF1060168
:10174000A81DF7F765FD08E02348037800F12302A0
:101750000DF10601A81DF7F75BFD00240CE004F174
:101760001600285CA11D1DF80110484004F1160167
:101770000DF80100601CC4B20B2CF0DB072409E05B
:10178000601E1DF800001DF8041048400DF804000C
:10179000601CC4B2212CF3DB06240FE01DF804000A
:1017A00080F05506601C1DF8000080F0A5000DF8C3
:1017B0000400601C0DF80060A01CC4B21F2CEDDBFF
:1017C000212269462846F6F7E3FC2020287000BF56
:1017D00079E7000044040020384B002030B591B078
:1017E000044621460720F8F7B5F905462246294662
:1017F0000720F8F7D5FA05F0400060B18DF80040F9
:1018000021460DF10200F8F7C7F98DF801000E48E6
:10181000016C6846884705F0200028B1012000F0DF
:1018200071FA204600F02AF9084A32F81410084AE2
:1018300052F82400FDF70AFA2046F8F766FB204626
:10184000F8F76AFB11B030BD480300209439010855
:101850008439010870B506460D461446284A32F808
:101860001410284A52F82400FDF7F0F92146002010
:10187000F8F76EFB244A32F81410244A52F8240078
:10188000FDF7E4F92146E120FCF7F2FA1E4A32F8AE
:1018900014101E4A52F82400FDF7DAF9202D00DD5D
:1018A0002025FBF79BFE40B1194A32F81410194A63
:1018B00052F82400FDF7CAF907E0154A32F814106F
:1018C000144A52F82400FDF7C3F920252246294680
:1018D0003046F8F793FA0A4A32F81410094A52F8D7
:1018E0002400FDF7B5F93220F7F71EFC044A32F860
:1018F0001410044A52F82400FDF7A8F970BD000046
:10190000AC3901089C3901086039010850390108D7
:10191000943901088439010800B591B000224021B2
:1019200001A8FEF711F81F208DF80400E1208DF8C2
:1019300005000A49C86980478DF806000A208DF81D
:10194000070006208DF808000DF10900FDF7A8F842
:101950000248416C01A8884711B000BD480300202F
:1019600010B512480078012800D010BD0F4840681B
:10197000401C0E49486040F2DC5188420ED20B48B0
:1019800040686421B0FBF1F201FB120058B908482D
:10199000C16D01208847FFF7BFFF04E00220034923
:1019A00008700020486000BFDFE70000F40300205B
:1019B000B802002010B504462046F8F749FA21463F
:1019C0007020F8F73DF8224601211D20F8F7E8F9CC
:1019D000224620211120F8F7E3F922461E2100209B
:1019E000F8F7DEF9224600210120F8F7D9F922465E
:1019F00001210220F8F7D4F9224603210846F8F71E
:101A0000CFF9154890F87400012803D12146F8F762
:101A10006FF90CE0104890F87400022803D12146B9
:101A2000F8F766F903E021460020F8F761F921464E
:101A30000320F8F72FF9224605214AF2554000F01D
:101A400055F82046F8F744F82046F8F725F82046E0
:101A5000F8F762FA10BD000044040020704700004F
:101A600000EB4001044A12F81110491C00EB40023F
:101A7000014B03F8121070479C11002000EB40014D
:101A8000054A02EB41014978491C00EB4002024B38
:101A900003EB4202517070479C11002070B5044660
:101AA0000D46FBF79BFD20B129460720F8F7F2F819
:101AB0001BE0012C04D0022C07D0032C0FD109E02D
:101AC00029460220F8F7E6F80EE029460120F8F74B
:101AD000E1F809E029460020F8F7DCF804E029469F
:101AE0000320F8F7D7F800BF00BF70BD7CB50446EF
:101AF0000D4616460AA103C9CDE9000120128DF852
:101B00000200E0B28DF80300324629466846F8F735
:101B10000DF933462A4669460020F8F7CDF87CBD1A
:101B20001998A4250100000070B505460C46F7F78A
:101B30004EFA21462846F8F7DEF92046F8F7ECF988
:101B4000F8F758FA70BD000010B504460548007C4F
:101B500028B12178601CF8F73FFD012010BD00205E
:101B6000FCE70000305F002070B5054600240DE062
:101B7000094800EB840104222846F6F73BFB18B91C
:101B8000054800EB840070BD601C84B203480078F7
:101B90008442EDDB0020F6E7905B00208705002003
:101BA00030B591B004460D462078401CC2B269465B
:101BB0002046FDF7BEFE104890F87E0060B19DF80B
:101BC0000000001FC0B28DF800009DF800200DF14C
:101BD0000101081DFDF7ADFE0748D0F8A4106846C6
:101BE00088479DF8001005482A46836A0DF10100D8
:101BF000984711B030BD000044040020B802002016
:101C00002DE9F04104462078062813D00E480568D7
:101C1000001D0668001D07683D4455B10822A11C3F
:101C20002846FDF7C7F9042204F112013046FDF7FA
:101C3000C1F906E00549086810B16080010CA18077
:101C400000BFBDE8F0810000E8F7FF1F002102405F
:101C5000A0200C4988720C4890F8700048700D2044
:101C600088700120C870084890F87100C872064852
:101C700090F8721003480173034890F873100148FC
:101C8000417370474A08002044040020014908704D
:101C900070470000E803002010B504460D4890F896
:101CA000850058B10B49D1F8B000804718B1012028
:101CB0000949C87505E00848C47502E000200649D6
:101CC000C8750122044917314FF4A070FBF752FA8E
:101CD00010BD0000440400209C070020064909783C
:101CE00001B1704728B90121034A11700349044A20
:101CF000916100BFF5E70000B3020020E592000803
:101D0000B80200200149087070470000400300201D
:101D100010B516488078164908720022042114482C
:101D2000001DFDF711FE1248027A011D0F48C01C6C
:101D3000FDF7FFFD0E48C07A0D49097A884204DAA2
:101D400000210B48C27A001D8154002408E0084B92
:101D5000195D1B1D185D074BDA6A9047601CC4B201
:101D60000348407AA042F2DC10BD0000D6030020F8
:101D7000EC100020B802002010B504460948C470D9
:101D80000146C878FBF7B8FB064908710879FBF7EC
:101D9000B3FB044948714879FBF7AEFB01498871F0
:101DA00010BD0000D6030020016841F04001016031
:101DB00070470146C86880B27047C16070470246EC
:101DC0009068084008B1012070470020FCE70246F7
:101DD0000020106800F441500B6818434B6818430A
:101DE0008B681843CB6818430B6918434B69184339
:101DF0008B6918431060D36923F40063D361704783
:101E000010B50D4890F8C40000B910BD0B48C07B58
:101E1000012800D1F9E70A48816B0020884707486C
:101E2000007D401CC1B2054801750121C17300212C
:101E30000174417400BFE8E7440400207B5B00208C
:101E400048030020002000213E4A126842F48032FC
:101E50003C4B1A6000BF401C3A4A126802F4003141
:101E600019B94FF6FF729042F5D1364A126802F462
:101E700000320AB900BFFEE7324AD26942F080520E
:101E8000304BDA61304A126842F440422E4B1A60FD
:101E90002C4A52682B4B5A601A4652685A601A46AE
:101EA000526842F480625A601A46526822F4403204
:101EB0005A601A46526842F440325A601A465268D2
:101EC000224B1A401F4B5A601A46526842F4501275
:101ED0005A601A46126842F080721A6000BF194AAE
:101EE000126802F00072002AF9D0174A126842F410
:101EF0008032154B1A6000BF134A526802F48032D8
:101F0000002AF9D0104A126842F400320E4B1A60CF
:101F100000BF0D4A526802F40032002AF9D0094A83
:101F2000526822F00302074B5A601A46526842F088
:101F300002025A6000BF034A526802F00802002AF7
:101F4000F9D070470010024000700040FFFFC3B797
:101F500010B5FFF777FF10BD10B5124800684FF4B9
:101F60007A71B0FBF1F4601EB0F1807F01D30120E3
:101F70000FE0601E4FF0E02148610F214FF0FF306D
:101F8000F7F790FF00204FF0E021886107200861FB
:101F9000002008B100BFFEE70F214FF0FF30F7F738
:101FA00081FF10BD1000002010B5044604480068F1
:101FB000001B81B202482C3800F05AF810BD000016
:101FC0002C04004010B50120234988750846407A4A
:101FD00070B90846807A401CC0B28872052807DDB7
:101FE00000208872012048721C48016D012088473A
:101FF0001948007A401CC0B21749087219280EDD32
:10200000002008721549C869804720B11348C16C87
:102010000220884703E01148C16C012088470E4820
:102020004088401C80B20C49488040F2DC51884214
:1020300003DD00200849087048800748C088401C1C
:1020400080B20549C880322802DD00200871C880AE
:1020500003498868804710BD9C070020B802002013
:1020600038040020C162704701460020486A70476A
:1020700041627047016841F0010101607047000052
:102080000A8882621D4A90420ED0B0F1804F0BD078
:102090001B4A904208D01B4A904205D01A4A9042EF
:1020A00002D01A4A90420BD1026822F070020260FC
:1020B00002684B881A43026002688B881A430260E8
:1020C0008A68C262124A90420AD0124A904207D0ED
:1020D000026822F4407202600268CB881A430260F0
:1020E000064A904202D0094A904201D10A7B02631B
:1020F000426942F00102426170470000002C014039
:102100000004004000080040000C00400034014082
:102110000010004000140040C2688A43C26070474B
:10212000C2680A43C2607047CA43026170470246F0
:10213000D06800EA01031069084010B10BB101201A
:1021400070470020FCE7000010B50B48007810B184
:102150000020094908700948007810B1002007499B
:1021600008700748007828B1002005490870054923
:102170000869804710BD0000EF030020F003002035
:10218000F10300202406002081621AB9436943F05C
:10219000010343617047000010B540230A22024941
:1021A0000248FEF7B3FF10BD54140020481400206D
:1021B00010B540230A2202490248FEF7A7FF10BDCE
:1021C000C8110020BC1100207047000010B50A485B
:1021D000C16B032088474FF47A70FBF7C6F80748B5
:1021E000816B0120884700200549087400210920DF
:1021F00000F094F810BD0000B80200204803002051
:10220000305F002010B50748C068401C0549C86011
:10221000052805D30020C860F8F764FBF7F7F6FB44
:1022200010BD0000305F00200020704738B5044624
:102230002079012802D0072865D140E03348A16801
:102240000160E1684160218A0181E079012822D1A1
:102250002E48807901062D48C07901EB00412B48BA
:10226000007A01EB00212948407A0D18284881693D
:102270006846884725484079244A127900EB0220B5
:1022800081B22A466846F8F743F901201F490874CD
:10229000F8F700FB0CE0E079022809D100201B4987
:1022A000087405201B4908701948816B0120884774
:1022B0001A23221D1621612000F054FE24E01A2367
:1022C000221D1621612000F04DFE60791E2803D1E9
:1022D0002046FDF729FC15E0207A15280BDC217A31
:1022E00001EB41020949113101EB0210302204F1E6
:1022F0000901F5F74DFF207A152803D10120034984
:1023000081F8310400E000BF00BF38BD305F00201D
:1023100048030020900500207047704730B589B011
:1023200005460C4618208DF80400E1208DF80500C4
:102330000A49C86980478DF8060016208DF8070005
:102340008DF8085020128DF80900E0B28DF80A00CF
:102350000248416C01A8884709B030BD48030020FD
:1023600010B50446D4F8AC000021826A204690479C
:1023700010BD10B50446D4F8AC10A06C0022CB6A96
:102380001146984710BD70B504460025D4F8AC003E
:102390002946426B2046904700BF70BD41600281D4
:1023A00043817047416002814381704741600281EF
:1023B00043817047417841F08001014A11607047C4
:1023C0004C5C004070B504460D46A078032808D147
:1023D000287930B9D4F8A8002946C2682046904729
:1023E00070BD0120FCE700000120084908600020C2
:1023F0000860091D0860054910310860034800683D
:1024000040F41F400149086070470000405C0040F4
:102410000120044908600020091D08600320091FED
:1024200008607047405C004010B50446012C04D1A0
:1024300001020548FCF70CFC04E04FF480710248EF
:10244000FCF704FC10BD000000080140F0B5034695
:102450000024002500266AB9214800EB0110C0685D
:10246000C0F309051E4800EB011080681D4F07EB03
:10247000400627E0012A23D11B4F07EB8100D0F84B
:10248000000C00F0400068B1154800EB01104068F6
:10249000C0F30905124800EB01100068114F07EB6B
:1024A00040060FE00E4800EB0110C068C0F30905BC
:1024B0000B4800EB011080680A4F07EB400601E073
:1024C0000020F0BD002405E036F8047B1F809B1C33
:1024D000601C84B2681CB4EB500FF5D32846F0E7BB
:1024E00000600040006000400050004070B58AB1BC
:1024F000134D05EB01152D68124E06EB4504002324
:1025000003E0058820C4801C5B1C551CB3EB550FF1
:10251000F7D300BF0A4B03EB01135A6000BF0A4C0C
:1025200004EB8103D3F8003C48F6BF74234083F0EA
:102530003003054D05EB8104C4F8003C00BF70BDBD
:1025400000600040006000400050004070B504464C
:102550000D46D4F8AC002946426A2046904770BD2B
:1025600030B5034601F07F00CA1142B300BF294CC9
:1025700004EB8002D2F8002C02F040027AB100BFD6
:1025800004EB8002D2F8002C48F68F74224042F00F
:102590004002204D05EB8004C4F8002C00BF00BFB2
:1025A00000BF1C4C04EB8002D2F8002C48F6BF742C
:1025B0002240184D05EB8004C4F8002C28E000BF31
:1025C000144C04EB8002D2F8002C02F480427AB161
:1025D00000BF04EB8002D2F8002C48F68F74224032
:1025E00042F480420B4D05EB8004C4F8002C00BF80
:1025F00000BF00BF074C04EB8002D2F8002C4BF662
:102600008F742240034D05EB8004C4F8002C00BFFA
:1026100030BD0000005000402DE9F04104460D4659
:1026200016461F46D4F8AC003B4632462946D0F841
:1026300020C02046E047BDE8F0812DE9F041044686
:102640000D4616461F4605F07F0000EB400104F1E1
:10265000140000EB810800233A4631464046FFF75C
:102660009DFED4F8AC002946826A20469047BDE81A
:10267000F081000030B50246002002F14401A023A1
:10268000204C23600023636040230B803039A3601B
:102690000B800B883E2B0AD90B884FF6FF7404EA97
:1026A00043135B1E43F40043164CE36006E00B88C3
:1026B0005B1C23F001035B02124CE36001200FE07E
:1026C000114C04EB8003D3F8003C48F68F74A3430D
:1026D00003430D4D05EB8004C4F8003C431CD8B205
:1026E0000428EDD3094B1B689BB2084C236043F2CE
:1026F000202323608023054C4C34236001239370F6
:1027000030BD00000060004000500040005C004010
:1027100010B500BF4A06094B03EBD252D2F8002C89
:102720004BF68F731A4082F440524B06034C04EB75
:10273000D353C3F8002C00BF10BD00000050004070
:102740002DE9F0470546894616461F4609F07F0ADF
:102750000AEB4A0105F1440000EB8108B8F80000DB
:10276000B84201DD384601E0B8F800000446D5F86B
:10277000AC0022465146C36A30469847381B82B2A5
:10278000311923464046FFF709FEBDE8F0870000F7
:102790002DE9F04305460C469E7806F07F009988A7
:1027A000002793F803C00CF0030CDFF8508258F8B0
:1027B0002CC04CEA000CDFF8489209EB8008C8F8FE
:1027C00000CC4FEAE61CBCF1000F62D000EB4008E1
:1027D00005F1440C0CEB88073980B4B9DFF824C24A
:1027E0000CEB001CCCF8002000BFC84608EB800CA6
:1027F000DCF800CC48F6BF780CEA080C8CF0200C12
:1028000009EB8008C8F800CCF6E0012CFCD1DFF819
:10281000F08108EB800CDCF800CC4CF4807C48F6AE
:102820008F780CEA080CDFF8D89109EB8008C8F81B
:1028300000CC1FFA82FCDFF8CC8108EB0018C8F846
:1028400000C04FEA124CDFF8BC8108EB0018C8F852
:1028500008C000BFC84608EB800CDCF800CC48F686
:10286000BF780CEA080C8CF0300C09EB8008C8F833
:1028700000CC00BF00BFC84608EB800CDCF800CCE1
:102880004BF68F780CEA080C09EB8008C8F800CCEE
:10289000B2E000EB400805F1140C0CEB880739801E
:1028A00034B9DFF860C10CEB001CCCF808204EE016
:1028B000012C4CD1DFF8488108EB800CDCF800CC0F
:1028C0004CF4807C48F68F780CEA080CDFF83091E5
:1028D00009EB8008C8F800CC00BFC84608EB800CA4
:1028E000DCF800CC48F68F780CEA080C4CF0400C71
:1028F00009EB8008C8F800CC00BF1FFA82FCDFF8A3
:10290000048108EB0018C8F800C04FEA124CDFF849
:10291000F48008EB0018C8F808C03E290BD9A4467B
:10292000CCEB411C4CF4004CDFF8D88008EB0018CD
:10293000C8F804C00BE001F1010C2CF0010C4FEAC7
:102940004C2CDFF8C08008EB0018C8F804C03E2902
:102950000CD94FF0010CCCEB411C4CF4004CDFF8CF
:10296000A48008EB0018C8F80CC00BE001F1010CC2
:102970002CF0010C4FEA4C2CDFF8888008EB001893
:10298000C8F80CC09CB900BFDFF8748008EB800C5D
:10299000DCF800CC4BF68F780CEA080C8CF4005C69
:1029A000DFF85C9009EB8008C8F800CC24E0012C2B
:1029B00022D100BFDFF8488008EB800CDCF800CCA7
:1029C0004BF68F780CEA080CDFF8349009EB80089E
:1029D000C8F800CC00BF00BFC84608EB800CDCF88C
:1029E00000CC48F6BF780CEA080C8CF0200C09EB00
:1029F0008008C8F800CC00BFBDE8F083203901088A
:102A0000005000400060004030B5024601F07F00F9
:102A1000CB1193B300BF334C04EB8003D3F8003CDD
:102A200003F040037BB100BF04EB8003D3F8003C0C
:102A300048F68F74234043F040032A4D05EB800491
:102A4000C4F8003C00BF00BF002400EB400502F1C9
:102A5000440303EB85039C7000BF224C04EB80030E
:102A6000D3F8003C48F6BF74234083F030031D4D7B
:102A700005EB8004C4F8003C33E0FFE700BF194CCD
:102A800004EB8003D3F8003C03F480437BB100BF28
:102A900004EB8003D3F8003C48F68F74234043F4E2
:102AA0008043104D05EB8004C4F8003C00BF00BF1C
:102AB000002400EB400502F1140303EB85039C7036
:102AC00000BF084C04EB8003D3F8003C4BF68F7436
:102AD000234083F44053034D05EB8004C4F8003CCD
:102AE00000BF30BD0050004030B5024601F07F000D
:102AF000A8B900BF244B1B6848F6BF74234083F07D
:102B00001003214C236000BF00BF23461B684BF617
:102B10008F74234083F480531B4C236033E0CB112C
:102B2000C3B1012400EB400502F1440303EB85032C
:102B30009C7000BF154C04EB8003D3F8003C48F6B2
:102B4000BF74234083F01003104D05EB8004C4F8DC
:102B5000003C18E0012400EB400502F1140303EBF4
:102B600085039C7000BF094C04EB8003D3F8003C44
:102B70004BF68F74234083F48053044D05EB80049F
:102B8000C4F8003C00BF30BD005C00400050004075
:102B900010B503464806064C04EBD050D0F8002C84
:102BA000C81110B102F0300010BD0020FCE7000099
:102BB0000050004070B504460D46164608201449E2
:102BC0000870012048704002488008464460743410
:102BD000256366630F48A0630F4844F874090F49E2
:102BE000A1670F49E167D4F8A4004068C07900F0FC
:102BF0004000400920710121E171D4F8AC1008684F
:102C00008047D4F8A410C968C868FEF7F9FF70BD02
:102C1000140000201C00002039B30008F5B20008A1
:102C2000A3B2000810B50446A078E0700420A0709C
:102C3000E07930B100BFD4F8AC100869804700BF1C
:102C400001E00321A17110BD2DE9FC419A48006803
:102C500080B20190984800689749091F096801F4FB
:102C60007F410840009095484468BDF8000000F49A
:102C7000004000287DD0A5E0BDF8040000F00F055D
:102C8000BDF8040000F01000002860D08C4901EB72
:102C90008500D0F8000C00F4004000281FD000BFD1
:102CA00001EB8500D0F8000C40F68F710840844A93
:102CB00002EB8501C1F8000C00BF114601EB850055
:102CC000D0F8000C00F4006060B14DB905EB45018F
:102CD00004F1740050F8212029462046904770E006
:102CE000BDE8FC8105EB450104F1140000EB810611
:102CF0007068D4F8AC1000220B6B29469847074641
:102D00007068384470607089384470817089318986
:102D1000884202DA3088B84212DD05EB450104F141
:102D2000740000EB8100406880B105EB450104F1BF
:102D3000740000EB8100294642682046904705E078
:102D4000D4F8AC002946826A2046904739E05C49B5
:102D500001EB8500D0F8000C00F0800088B300BFC4
:102D600001EB8500D0F8000C48F60F710840544A7A
:102D700000E030E002EB8501C1F8000C00BF05EB7C
:102D8000450104F1440000EB8106308990B905EB60
:102D9000450104F1740000EB8100806880B105EB0F
:102DA000450104F1740000EB810029468268204649
:102DB000904705E03389294620467268FFF7C0FC3A
:102DC00000BF00BF3C48006880B2019000F40040A2
:102DD00000287FF451AFBDF8000000F4805070B1BE
:102DE0006FF4805034490860E078A070607A30B9A0
:102DF00000BFD4F8AC104869804700BF00BFBDF8E1
:102E0000000000F4006060B12B48001F006800F073
:102E1000100030B92046FFF705FF6FF40060264927
:102E20000860BDF8000000F4007058B16FF4007045
:102E3000214908602348006820B1224800680168E1
:102E400020468847BDF8000000F4807018B36FF486
:102E5000807019490860A079E8B1A079401EC1B21C
:102E6000A171C1B9607A50B11348001F006820F009
:102E700010001149091F0860002161720BE00E4823
:102E8000001F006840F010000B49091F0860032173
:102E9000A17101216172BDF8000000F4806040B1B1
:102EA0006FF4806004490860D4F8AC00C169204622
:102EB000884700BF14E70000445C00401400002075
:102EC000005000405C0000200548006820F004002D
:102ED000034908600846006820F008000860704751
:102EE000405C004005494968097A012905D1044937
:102EF000096841F01001024A116070471400002077
:102F0000405C004070B505460C466078034951F8B6
:102F1000202021462846904770BD00006000002018
:102F20000348006840F00C00014908607047000049
:102F3000405C004002460120704710B5FFF762F97F
:102F400010BD000010B5012003490870F8F732FEEB
:102F500000F0AAFA10BD0000B202002070477047CE
:102F600070477047F0B589B004460D4616461F46B7
:102F7000202101A8F5F733F91F208DF8040004F093
:102F80000F0040F0E0008DF805000949C86980474E
:102F90008DF806008DF807503A46314602A8F5F73D
:102FA000F7F80348416C01A8884709B0F0BD00005C
:102FB000480300207047000010B50446607920B92E
:102FC000044841680020884703E002484168012026
:102FD000884710BD24040020F0B59DB004460022AF
:102FE00040210DA8FCF7B0FC1F208DF83400E02034
:102FF0008DF83500FBF7C8FC8DF8360005208DF8FC
:1030000037008DF8384094480078A0422ADB04EB62
:10301000440000EB84109149084490F841000228D4
:1030200020D104EB440101EB84118C4B194491F83D
:10303000402004EB440101EB8411C8180DF1390163
:10304000FCF777FC04EB440000EB84108349084450
:1030500090F842008DF834000DA8F9F70FFF012019
:103060001DB0F0BD20217E48FEF784F8054675B9F5
:10307000FF208DF8380000208DF839008DF83A00D7
:103080008DF83B000DA8F9F7F9FE0020E8E70A9556
:103090000CAA0BA90AA8FBF737FD8DF8340004EB46
:1030A000440101EB84116D4A881800224021FCF78D
:1030B0004BFC9DF8280004EB440101EB8411674AA6
:1030C0005054012004EB440101EB8411114481F8B8
:1030D000400004EB440101EB8411114481F84100EC
:1030E0005D480470002690E0701CC6B22023C82200
:1030F00002A95B480095FEF757F80746012F4CD10F
:103100009DF828000D2820D1012004EB440101EB9B
:103110008411524A114404EB440202EB84124F4BD7
:103120001A4492F84020885404EB440000EB8410C9
:103130001946084490F84000401C04EB440101EBA0
:1031400084111A46114481F8400004EB440000EB5E
:103150008410424A104404EB440202EB84123F4BB9
:103160001A4492F8402081189DF830200DF1090092
:10317000FCF7DFFB04EB440000EB84103749084404
:1031800090F840009DF83010084404EB440101EB36
:103190008411324A114481F840001FB19DF82C007F
:1031A000864231DBFF2004EB440101EB84112B4A02
:1031B000114404EB440202EB8412284B1A4492F8A7
:1031C00040208854FF2104EB440000EB84101A4691
:1031D000024404EB440000EB8410184490F84000D3
:1031E000401C115404EB440000EB841019460844C1
:1031F00090F84000801C04EB440101EB84111A4656
:10320000114481F8400005E000BF9DF82C00864283
:10321000FFF66AAF00BF04EB440101EB84110F4BD2
:10322000194491F8402004EB440101EB8411C818C3
:103230000DF13901FCF77DFB9DF8340004EB4401EE
:1032400001EB8411054A114481F842000DA8F9F7F9
:1032500015FE012004E70000FD030020E02F002000
:10326000D416002010B500F053F800200249487031
:1032700088700870C87010BDFF03002010B50948A1
:10328000C078401CC0B20749C870022800DA10BDDF
:1032900000200449C8700120887000F013F800BFB6
:1032A000F5E70000FF03002010B500F0EBF8012067
:1032B00003494870887000200870C87010BD000075
:1032C000FF03002010B50B48407890B10948007802
:1032D00009280EDA0748807858B106480078401C63
:1032E000044908700878FFF777FE0249487000200B
:1032F000887010BDFF03002010B504462023C822AB
:1033000021460248FDF7D4FE10BD0000D41600206F
:1033100010B52023C82202490248FDF7F7FE10BD70
:10332000E0160020D4160020FEB507460026002433
:103330000CE0385D10B1385D0A2800DD08E0385D2A
:103340000DF80400701CC6B2601CC4B20A2CF0DB7D
:1033500000BF06B9FEBD47490868804700240CE05D
:1033600000201DF8041001EB410202EB8111424ADA
:10337000114481F84100601CC4B2B442F0DB3F4804
:103380000078864203DB00203C4908706CE0012590
:1033900001245FE004EB440000EB8410364908444C
:1033A00090F8410000B953E03548C08B401C3449C7
:1033B000C883022005EB450101EB85112E4A11441B
:1033C00081F84100AC4202D1681CC5B240E004EB78
:1033D000440303EB8413DFF8A0C0634493F8402058
:1033E00005EB450303EB851303EB0C0104EB4403EE
:1033F00003EB841303EB0C00FCF79BFA04EB440093
:1034000000EB84101C49084490F8400005EB45018E
:1034100001EB8511184A114481F8400004EB440087
:1034200000EB84101146084490F8420005EB45017A
:1034300001EB8511114481F84200002004EB4401A6
:1034400001EB8411114481F84100681CC5B200BF32
:10345000601CC4B20948007884429BDD07480078AC
:10346000801B0649087000BF02494868804700BFBA
:1034700070E70000B8020020E02F0020FD030020CC
:103480009C070020704710B54FF4FA7408E0FBF772
:10349000C3FB00B110BD0A20F5F746FE601E84B2E2
:1034A000002CF4D100BFF5E710B51448007800B93E
:1034B00010BD1349486D804738B91248807820B94B
:1034C000012010498870F8F735FB0E48C07800B924
:1034D000EEE70C488088401C80B20A498880C828E2
:1034E00002DA00F011F807E000200649C870888071
:1034F00008460021C0F8061000BFD9E744040020A8
:1035000048030020B05E002010B588B0364800782F
:1035100010B13648C07810B9002008B010BD1C208A
:103520008DF80000324881690DF101008847302094
:103530008DF8050000208DF806008DF80700142096
:103540008DF8080004208DF8090013210DF10A0000
:10355000F4F745FE2548C07801283AD1FF208DF8C0
:1035600006008DF80700214890F87F001F4991F868
:103570007E10884203DB00201C4981F87F001B4835
:1035800090F87F10801D10F821008DF80E0017486C
:1035900090F87F10801D00EB810040788DF80F00BF
:1035A000124890F87F10801D00EB810080788DF824
:1035B00010000E4890F87F10801D00EB8100C0784D
:1035C0008DF81100094890F87F00401C074981F8E8
:1035D0007F000749C86A8047044605482146426B78
:1035E00068469047012098E744040020B05E002020
:1035F0004803002030B591B004460D46402101A893
:10360000F4F7EDFD3C208DF80400E1208DF8050075
:103610000949C86980478DF806000E208DF807001B
:103620002A46214602A8F4F7B3FD0348416C01A8DD
:10363000884711B030BD0000480300202DE9F0415B
:1036400007464FF6FF783846F9F78EFF05461248D1
:1036500000782844C82806DC2A4639460E480078F7
:1036600000F044F914E00C480078C0F1C800C6B27C
:10367000324639460848007800F038F9344605E00B
:103680000120A04028EA0008601CC4B2AC42F7DB6D
:103690004046BDE8F0810000870500202DE9F0419B
:1036A00006464FF6FF773046F9F75EFF05461E2DBA
:1036B00000DD1E250F4880F87E50002414E006EB44
:1036C0008400FEF751FAB0F1000803D10120A040B8
:1036D000874307E03046F8F743FAAA220421404620
:1036E000F4F776FD601C84B2AC42E8DB3846BDE8F6
:1036F000F0810000B05E002070B590B004462079E3
:1037000001280BD0022804D004281DD0052845D15B
:103710001FE06079A11D00F089F800BF60790DF10C
:10372000020100F05FF820B928210DF10200F4F742
:1037300056FD01208DF8000060798DF801002A21E6
:103740006846FFF757FF2AE0A01DFFF777FF054601
:1037500004E0A01DFFF7A2FF054600BF02208DF880
:103760000000C5F3090040F2FF31884201D1012079
:1037700000E000208DF80100002608E045FA06F080
:1037800000F00101B01C0DF80010701CC6B20A2E2A
:10379000F4DB0C216846FFF72DFF00E000BF00BFFF
:1037A00010B070BD00210B4A11700B4A117000203F
:1037B00006E00A4901EB800100220A60411C88B240
:1037C000C828F6DB0021064AD170918091701180E3
:1037D000704700008805002087050020905B0020CE
:1037E000B05E00202DE9F04106460F46142E02DBA4
:1037F0000020BDE8F0813046FBF780F90546002443
:103800000DE04FF6FF7000EA840807EB0800291965
:10381000054A02EB810109680160601C84B20A2C30
:10382000EFDB0120E5E70000905B00202DE9F0418F
:1038300004460E46142C02DB0020BDE8F0811CB9C2
:10384000FFF7B0FFF8F776F93046F9F78DFE054639
:103850002046FBF753F907462A46F8B2314600F0F6
:1038600045F80120E9E7000030B589B005461D485C
:103870000378C21C01A92846F5F7CAFC002409E018
:1038800001A8005D611C01AA515C4840611C5054B4
:10389000601CC4B20F2CF3DB1348102201A9036A89
:1038A000900198470F480378C21C01A905F1100048
:1038B000F5F7AEFC002409E001A8005D611C01AA37
:1038C000515C4840611C5054601CC4B20F2CF3DBA7
:1038D0000548102201A9036A4FF48260984709B095
:1038E00030BD0000384B0020B802002030B5034640
:1038F000002009E01C18084D05EB840401EB80054D
:103900002D682560441CA0B29042F3DB034C247860
:103910001444024D2C7030BD905B002087050020C0
:10392000000200000004000000000000000600008B
:1039300006FFFF09FFA10109FF95407508158025C5
:103940007F810009FF954075081580257F9100C093
:1039500000140140000C014000140140001001401F
:103960000020100008004000001401400014014035
:1039700000140140001001400040200010008000B1
:103980000E0504070014014000140140001401401A
:103990000010014000084000020010000014014027
:1039A000001401400014014000100140001080008C
:1039B000040020004053554E564F54450053756E39
:1039C000566F746531393938264A61636B506569C1
:1039D00031393732436F6F6C426F62393900104EA4
:1039E0001341144215431644174518461947204AF7
:1039F000304B404D9151925293539454A05AB05B26
:103A0000C05C00000100000052096AD53036A538BC
:103A1000BF40A39E81F3D7FB7CE339829B2FFF87B6
:103A2000348E4344C4DEE9CB547B9432A6C2233D9A
:103A3000EE4C950B42FAC34E082EA16628D924B24B
:103A4000765BA2496D8BD12572F8F664866898166C
:103A5000D4A45CCC5D65B6926C704850FDEDB9DACB
:103A60005E154657A78D9D8490D8AB008CBCD30AB9
:103A7000F7E45805B8B34506D02C1E8FCA3F0F0295
:103A8000C1AFBD0301138A6B3A9111414F67DCEA64
:103A900097F2CFCEF0B4E67396AC7422E7AD3585DD
:103AA000E2F937E81C75DF6E47F11A711D29C589E7
:103AB0006FB7620EAA18BE1BFC563E4BC6D27920C9
:103AC0009ADBC0FE78CD5AF41FDDA8338807C731D2
:103AD000B11210592780EC5F60517FA919B54A0DCA
:103AE0002DE57A9F93C99CEFA0E03B4DAE2AF5B03F
:103AF000C8EBBB3C83539961172B047EBA77D6265B
:103B0000E169146355210C7D637C777BF26B6FC593
:103B10003001672BFED7AB76CA82C97DFA5947F0D0
:103B2000ADD4A2AF9CA472C0B7FD9326363FF7CCAC
:103B300034A5E5F171D8311504C723C31896059A49
:103B4000071280E2EB27B27509832C1A1B6E5AA06C
:103B5000523BD6B329E32F8453D100ED20FCB15B57
:103B60006ACBBE394A4C58CFD0EFAAFB434D3385C0
:103B700045F9027F503C9FA851A3408F929D38F594
:103B8000BCB6DA2110FFF3D2CD0C13EC5F974417CB
:103B9000C4A77E3D645D197360814FDC222A908842
:103BA00046EEB814DE5E0BDBE0323A0A4906245CCE
:103BB000C2D3AC629195E479E7C8376D8DD54EA933
:103BC0006C56F4EA657AAE08BA78252E1CA6B4C6FF
:103BD000E8DD741F4BBD8B8A703EB5664803F60E58
:103BE000613557B986C11D9EE1F8981169D98E9447
:103BF0009B1E87E9CE5528DF8CA1890DBFE6426860
:103C000041992D0FB054BB168D01020408102040BD
:103C1000801B366CD8AB4D9A2F5EBC63C697356A55
:103C2000D4B37DFAEFC5913972E4D3BD61C29F254B
:103C30004A943366CC831D3A74E8CB8D01020408A4
:103C4000102040801B366CD8AB4D9A2F5EBC63C6EB
:103C500097356AD4B37DFAEFC5913972E4D3BD616B
:103C6000C29F254A943366CC831D3A74E8CB8D01FC
:103C7000020408102040801B366CD8AB4D9A2F5E92
:103C8000BC63C697356AD4B37DFAEFC5913972E447
:103C9000D3BD61C29F254A943366CC831D3A74E834
:103CA000CB8D01020408102040801B366CD8AB4D30
:103CB0009A2F5EBC63C697356AD4B37DFAEFC5917F
:103CC0003972E4D3BD61C29F254A943366CC831D0B
:103CD0003A74E8CB8D01020408102040801B366C3A
:103CE000D8AB4D9A2F5EBC63C697356AD4B37DFAC4
:103CF000EFC5913972E4D3BD61C29F254A94336602
:103D0000CC831D3A74E8CB000000211042206330C0
:103D10008440A550C660E770088129914AA16BB123
:103D20008CC1ADD1CEE1EFF109000000637C777B5F
:103D3000F26B6FC53001672BFED7AB76CA82C97DA7
:103D4000FA5947F0ADD4A2AF9CA472C0B7FD932638
:103D5000363FF7CC34A5E5F171D8311504C723C33C
:103D60001896059A071280E2EB27B27509832C1A80
:103D70001B6E5AA0523BD6B329E32F8453D100EDDA
:103D800020FCB15B6ACBBE394A4C58CFD0EFAAFBBE
:103D9000434D338545F9027F503C9FA851A3408F86
:103DA000929D38F5BCB6DA2110FFF3D2CD0C13EC9E
:103DB0005F974417C4A77E3D645D197360814FDC33
:103DC000222A908846EEB814DE5E0BDBE0323A0A17
:103DD0004906245CC2D3AC629195E479E7C8376D9B
:103DE0008DD54EA96C56F4EA657AAE08BA78252EC0
:103DF0001CA6B4C6E8DD741F4BBD8B8A703EB56649
:103E00004803F60E613557B986C11D9EE1F8981139
:103E100069D98E949B1E87E9CE5528DF8CA1890D28
:103E2000BFE6426841992D0FB054BB1652096AD5BE
:103E30003036A538BF40A39E81F3D7FB7CE339829F
:103E40009B2FFF87348E4344C4DEE9CB547B9432EE
:103E5000A6C2233DEE4C950B42FAC34E082EA16636
:103E600028D924B2765BA2496D8BD12572F8F6640D
:103E700086689816D4A45CCC5D65B6926C70485088
:103E8000FDEDB9DA5E154657A78D9D8490D8AB003D
:103E90008CBCD30AF7E45805B8B34506D02C1E8F66
:103EA000CA3F0F02C1AFBD0301138A6B3A911141A2
:103EB0004F67DCEA97F2CFCEF0B4E67396AC74228B
:103EC000E7AD3585E2F937E81C75DF6E47F11A7109
:103ED0001D29C5896FB7620EAA18BE1BFC563E4B42
:103EE000C6D279209ADBC0FE78CD5AF41FDDA83304
:103EF0008807C731B11210592780EC5F60517FA944
:103F000019B54A0D2DE57A9F93C99CEFA0E03B4D72
:103F1000AE2AF5B0C8EBBB3C83539961172B047EE6
:103F2000BA77D626E169146355210C7D00000001A3
:103F30000000000200000004000000080000001063
:103F40000000002000000040000000800000001B76
:103F500000000036A56363C6847C7CF8997777EE11
:103F60008D7B7BF60DF2F2FFBD6B6BD6B16F6FDE12
:103F700054C5C5915030306003010102A96767CE76
:103F80007D2B2B5619FEFEE762D7D7B5E6ABAB4DBE
:103F90009A7676EC45CACA8F9D82821F40C9C9892C
:103FA000877D7DFA15FAFAEFEB5959B2C947478E6A
:103FB0000BF0F0FBECADAD4167D4D4B3FDA2A25F32
:103FC000EAAFAF45BF9C9C23F7A4A453967272E45A
:103FD0005BC0C09BC2B7B7751CFDFDE1AE93933DBE
:103FE0006A26264C5A36366C413F3F7E02F7F7F57B
:103FF0004FCCCC835C343468F4A5A55134E5E5D1CD
:1040000008F1F1F9937171E273D8D8AB5331316291
:104010003F15152A0C04040852C7C795652323468B
:104020005EC3C39D28181830A19696370F05050A60
:10403000B59A9A2F0907070E361212249B80801B0F
:104040003DE2E2DF26EBEBCD6927274ECDB2B27F12
:104050009F7575EA1B0909129E83831D742C2C58C9
:104060002E1A1A342D1B1B36B26E6EDCEE5A5AB461
:10407000FBA0A05BF65252A44D3B3B7661D6D6B76F
:10408000CEB3B37D7B2929523EE3E3DD712F2F5E52
:1040900097848413F55353A668D1D1B9000000006A
:1040A0002CEDEDC1602020401FFCFCE3C8B1B179CC
:1040B000ED5B5BB6BE6A6AD446CBCB8DD9BEBE671C
:1040C0004B393972DE4A4A94D44C4C98E85858B06F
:1040D0004ACFCF856BD0D0BB2AEFEFC5E5AAAA4F58
:1040E00016FBFBEDC5434386D74D4D9A55333366DA
:1040F00094858511CF45458A10F9F9E90602020435
:10410000817F7FFEF05050A0443C3C78BA9F9F25B1
:10411000E3A8A84BF35151A2FEA3A35DC040408089
:104120008A8F8F05AD92923FBC9D9D214838387093
:1041300004F5F5F1DFBCBC63C1B6B67775DADAAF6A
:1041400063212142301010201AFFFFE50EF3F3FD2A
:104150006DD2D2BF4CCDCD81140C0C183513132663
:104160002FECECC3E15F5FBEA2979735CC44448847
:104170003917172E57C4C493F2A7A755827E7EFC29
:10418000473D3D7AAC6464C8E75D5DBA2B191932CE
:10419000957373E6A06060C098818119D14F4F9EDE
:1041A0007FDCDCA3662222447E2A2A54AB90903B1B
:1041B0008388880BCA46468C29EEEEC7D3B8B86B05
:1041C0003C14142879DEDEA7E25E5EBC1D0B0B16E4
:1041D00076DBDBAD3BE0E0DB563232644E3A3A74DC
:1041E0001E0A0A14DB4949920A06060C6C2424486C
:1041F000E45C5CB85DC2C29F6ED3D3BDEFACAC4390
:10420000A66262C4A8919139A495953137E4E4D3AC
:104210008B7979F232E7E7D543C8C88B5937376EC7
:10422000B76D6DDA8C8D8D0164D5D5B1D24E4E9CB3
:10423000E0A9A949B46C6CD8FA5656AC07F4F4F36B
:1042400025EAEACFAF6565CA8E7A7AF4E9AEAE4761
:1042500018080810D5BABA6F887878F06F25254A03
:10426000722E2E5C241C1C38F1A6A657C7B4B4735A
:1042700051C6C69723E8E8CB7CDDDDA19C7474E8C9
:10428000211F1F3EDD4B4B96DCBDBD61868B8B0D28
:10429000858A8A0F907070E0423E3E7CC4B5B5714D
:1042A000AA6666CCD84848900503030601F6F6F7DF
:1042B000120E0E1CA36161C25F35356AF95757AE05
:1042C000D0B9B9699186861758C1C199271D1D3A81
:1042D000B99E9E2738E1E1D913F8F8EBB398982BF3
:1042E00033111122BB6969D270D9D9A9898E8E0781
:1042F000A7949433B69B9B2D221E1E3C9287871554
:1043000020E9E9C949CECE87FF5555AA782828501B
:104310007ADFDFA58F8C8C03F8A1A15980898909E8
:10432000170D0D1ADABFBF6531E6E6D7C6424284E3
:10433000B86868D0C3414182B0999929772D2D5A28
:10434000110F0F1ECBB0B07BFC5454A8D6BBBB6D75
:104350003A16162C50A7F4515365417EC3A4171A80
:10436000965E273ACB6BAB3BF1459D1FAB58FAAC41
:104370009303E34B55FA3020F66D76AD9176CC88F9
:10438000254C02F5FCD7E54FD7CB2AC5804435260E
:104390008FA362B5495AB1DE671BBA25980EEA456C
:1043A000E1C0FE5D02752FC312F04C81A397468DCC
:1043B000C6F9D36BE75F8F03959C9215EB7A6DBFBF
:1043C000DA5952952D83BED4D32174582969E04916
:1043D00044C8C98E6A89C27578798EF46B3E589943
:1043E000DD71B927B64FE1BE17AD88F066AC20C9C4
:1043F000B43ACE7D184ADF6382311AE560335197B3
:10440000457F5362E07764B184AE6BBB1CA081FE34
:10441000942B08F95868487019FD458F876CDE9415
:10442000B7F87B5223D373ABE2024B72578F1FE373
:104430002AAB55660728EBB203C2B52F9A7BC58617
:10444000A50837D3F2872830B2A5BF23BA6A030282
:104450005C8216ED2B1CCF8A92B479A7F0F207F399
:10446000A1E2694ECDF4DA65D5BE05061F6234D1EE
:104470008AFEA6C49D532E34A055F3A232E18A05CC
:1044800075EBF6A439EC830BAAEF6040069F715ED2
:1044900051106EBDF98A213E3D06DD96AE053EDD2A
:1044A00046BDE64DB58D5491055DC4716FD40604CB
:1044B000FF15506024FB981997E9BDD6CC4340897D
:1044C000779ED967BD42E8B0888B8907385B19E7CA
:1044D000DBEEC879470A7CA1E90F427CC91E84F84B
:1044E000000000008386800948ED2B32AC70111E5D
:1044F0004E725A6CFBFF0EFD5638850F1ED5AE3D31
:1045000027392D3664D90F0A21A65C68D1545B9BEC
:104510003A2E3624B1670A0C0FE75793D296EEB4C1
:104520009E919B1B4FC5C080A220DC61694B775ACE
:10453000161A121C0ABA93E2E52AA0C043E0223CF4
:104540001D171B120B0D090EADC78BF2B9A8B62DA6
:10455000C8A91E148519F1574C0775AFBBDD99EE3C
:10456000FD607FA39F2601F7BCF5725CC53B6644E6
:10457000347EFB5B7629438BDCC623CB68FCEDB62F
:1045800063F1E4B8CADC31D7108563424022971347
:104590002011C6847D244A85F83DBBD21132F9AE84
:1045A0006DA129C74B2F9E1DF330B2DCEC52860D56
:1045B000D0E3C1776C16B32B99B970A9FA4894115E
:1045C0002264E947C48CFCA81A3FF0A0D82C7D5681
:1045D000EF903322C74E4987C1D138D9FEA2CA8C89
:1045E000360BD498CF81F5A628DE7AA5268EB7DAC9
:1045F000A4BFAD3FE49D3A2C0D9278509BCC5F6AEE
:1046000062467E54C2138DF6E8B8D8905EF7392E14
:10461000F5AFC382BE805D9F7C93D069A92DD56F15
:10462000B31225CF3B99ACC8A77D18106E639CE8E8
:104630007BBB3BDB097826CDF418596E01B79AECA9
:10464000A89A4F83656E95E67EE6FFAA08CFBC2147
:10465000E6E815EFD99BE7BACE366F4AD4099FEA50
:10466000D67CB029AFB2A43131233F2A3094A5C6FD
:10467000C066A23537BC4E74A6CA82FCB0D090E0AA
:1046800015D8A7334A9804F1F7DAEC410E50CD7FE4
:104690002FF691178DD64D764DB0EF43544DAACCE1
:1046A000DF0496E4E3B5D19E1B886A4CB81F2CC189
:1046B0007F51654604EA5E9D5D358C01737487FA0F
:1046C0002E410BFB5A1D67B352D2DB92335610E9D1
:1046D0001347D66D8C61D79A7A0CA1378E14F8598E
:1046E000893C13EBEE27A9CE35C961B7EDE51CE196
:1046F0003CB1477A59DFD29C3F73F25579CE1418FA
:10470000BF37C773EACDF7535BAAFD5F146F3DDF78
:1047100086DB447881F3AFCA3EC468B92C342438B0
:104720005F40A3C272C31D160C25E2BC8B493C2816
:1047300041950DFF7101A839DEB30C089CE4B4D893
:1047400090C156646184CB7B70B632D5745C6C4882
:104750004257B8D00000C201840346020807CA06C7
:104760008C044E05100ED20F940D560C1809DA0861
:104770009C0A5E0B201CE21DA41F661E281BEA1A61
:10478000AC186E193012F213B41176103815FA14F1
:10479000BC167E1740388239C43B063A483F8A3EF1
:1047A000CC3C0E3D50369237D435163458319A30C1
:1047B000DC321E336024A225E42726266823AA22A1
:1047C000EC202E21702AB22BF4293628782DBA2C11
:1047D000FC2E3E2F807042710473C67288774A7631
:1047E0000C74CE75907E527F147DD67C98795A7861
:1047F0001C7ADE7BA06C626D246FE66EA86B6A6A21
:104800002C68EE69B06272633461F660B8657A64F0
:104810003C66FE67C0480249444B864AC84F0A4E70
:104820004C4C8E4DD046124754459644D8411A40C0
:104830005C429E43E05422556457A656E8532A52E0
:104840006C50AE51F05A325B7459B658F85D3A5C10
:104850007C5EBE5F00E1C2E084E246E308E6CAE7B0
:104860008CE54EE410EFD2EE94EC56ED18E8DAE960
:104870009CEB5EEA20FDE2FCA4FE66FF28FAEAFB60
:10488000ACF96EF830F3F2F2B4F076F138F4FAF5F0
:10489000BCF77EF640D982D8C4DA06DB48DE8ADF70
:1048A000CCDD0EDC50D792D6D4D416D558D09AD1C0
:1048B000DCD31ED260C5A2C4E4C626C768C2AAC3A0
:1048C000ECC12EC070CBB2CAF4C836C978CCBACD10
:1048D000FCCF3ECE809142900492C69388964A9730
:1048E0000C95CE94909F529E149CD69D98985A9960
:1048F0001C9BDE9AA08D628C248EE68FA88A6A8B20
:104900002C89EE88B08372823480F681B8847A85EF
:104910003C87FE86C0A902A844AA86ABC8AE0AAFEF
:104920004CAD8EACD0A712A654A496A5D8A01AA1BF
:104930005CA39EA2E0B522B464B6A6B7E8B22AB3DF
:104940006CB1AEB0F0BB32BA74B8B6B9F8BC3ABD0F
:104950007CBFBEBE0000201C403860248070A06C6C
:10496000C048E05400E120FD40D960C58091A08D91
:10497000C0A9E0B500040101000000000000010032
:10498000040401010400010104040100040000000A
:104990000000010000040000000401010404010102
:1049A00000040000040400010400010100000001F3
:1049B00004000000040400000004000100040001E1
:1049C00000040100000401000000010100000101D9
:1049D00004040001040001000400000104000001BF
:1049E00004000100000000000404000004040100B1
:1049F00000000001000001000404010104000000A7
:104A0000000001010004010100000001000000019C
:104A10000004000004000101000001000004010086
:104A20000400000100040000040000000404000170
:104A3000040401000404010104000100000001015C
:104A40000404000104000001040400000404010047
:104A5000000401010404000000040001000400013E
:104A6000000000000400010000040100000000003C
:104A70000400010120801080008000800080000080
:104A80002080100000001000200000002000108096
:104A90002080008020000080208010800080108016
:104AA0000000008000800080000010002000000056
:104AB0002000108000801000200010002080008066
:104AC0000000000000000080008000002080100036
:104AD0000000108020001000200000800000000076
:104AE00000801000208000000080108000001080F6
:104AF00020800000000000002080100020001080B6
:104B000000001000208000800000108000801080D5
:104B10000080000000001080008000802000000065
:104B20002080108020801000200000000080000005
:104B30000000008020800000008010800000100035
:104B400020000080200010002080008020000080D5
:104B50002000100000801000000000000080008095
:104B60002080000000000080200010802080108045
:104B7000008010000802000000020208000000008F
:104B800008000208000200080000000008020200FD
:104B900000020008080002000800000808000008E1
:104BA00000000200080202080800020000000208DB
:104BB00008020000000000080800000000020208CF
:104BC00000020000000202000000020808000208C3
:104BD00008020200080200080002020000000200B1
:104BE0000802000808000000080202080002000095
:104BF000000000080002020800000008080002008F
:104C00000802000000000200000202080002000882
:104C10000000000000020000080002000802020874
:104C20000002000808000008000200000000000068
:104C30000800020808020008000002000000000846
:104C40000802020808000000080202000002020038
:104C5000080000080000020808020008080200001E
:104C60000000020808020200080000000800020814
:104C7000000202000120800081200000812000004D
:104C80008000000080208000810080000100800002
:104C900001200000000000000020800000208000B3
:104CA0008120800081000000000000008000800062
:104CB00001008000010000000020000000008000D2
:104CC0000120800080000000000080000120000022
:104CD0008020000081008000010000008020000092
:104CE0008000800000200000802080008120800063
:104CF0008100000080008000010080000020800012
:104D00008120800081000000000000000000000001
:104D10000020800080200000800080008100800052
:104D2000010000000120800081200000812000009F
:104D30008000000081208000810000000100000050
:104D40000020000001008000012000008020800081
:104D50008100800001200000802000000000800011
:104D60000120800080000000000080000020000082
:104D700080208000000100000001080200000802FD
:104D80000001004200000800000100000000004097
:104D900000000802000108400000080000010002B5
:104DA0000001084000010042000008420001080024
:104DB0000000004000000002000008400000084021
:104DC000000000000001004000010842000108420C
:104DD0000001000200000842000100400000000045
:104DE0000000004200010802000000020000004232
:104DF000000108000000080000010042000100005E
:104E00000000000200000040000008020001004213
:104E100000010840000100020000004000000842BC
:104E2000000108020001084000010000000000022B
:104E30000000084200010842000108000000004292
:104E400000010842000008020000000000000840C5
:104E500000000042000108000001000200010040C3
:104E600000000800000000000000084000010802E7
:104E70000001004010000020000040200040000021
:104E80001040402000004020100000001040402052
:104E900000004000004000201040400000004000A2
:104EA0001000002010004000004000200000002002
:104EB00010400000000000001000400010400020E2
:104EC00000400000004040001040002010000000A2
:104ED0001000402010004020000000001040400062
:104EE00000404020104000000040400000404020B2
:104EF00000000020004000201000000010004020B2
:104F000000404000104040200000400010400000E1
:104F100010000020000040000040002000000020A1
:104F200010400000100000201040402000404000D1
:104F300000004020104040000040402000000000E1
:104F40001000402010000000004000000000402041
:104F500010404000004000001000400010400020C1
:104F60000000000000404020000000201000400031
:104F7000104000200000200002002004020800046D
:104F800000000000000800000208000402082000E1
:104F90000008200402082004000020000000000097
:104FA00002000004020000000000000402002004CF
:104FB000020800000008000402082000020020008F
:104FC000000800040200000400002004000820047F
:104FD0000200200000002004000800000208000079
:104FE0000208200400082000020000000000000465
:104FF000000820000000000400082000000020003D
:105000000208000402080004020020040200200438
:10501000020000000200200000000004000800045C
:105020000000200000082004020800000208200000
:105030000008200402080000020000040208200406
:105040000000200400082000000000000200000012
:1050500002082004000000000208200000002004D4
:10506000000800000200000400080004000800001E
:10507000020020004010001000100000000004009A
:10508000401004100000001040100010400000000C
:105090000000001040000400000004104010041044
:1050A0000010040000100410401004000010000064
:1050B000400000000000041040000010001000102C
:1050C00040100000001004004000040040000410E4
:1050D000001004104010000000000000000000005C
:1050E00040000410400000100010001040100400A8
:1050F0000000040040100400000004000010041030
:1051000000100000400000004000041000100000EB
:10511000401004000010001040000000400000108B
:105120000000041040000410000000100000040003
:105130004010001000000000401004104000040067
:10514000400000100000041000100010401000107B
:1051500000000000401004100010040000100400C3
:10516000401000004010000040000400000000104B
:1051700000100410982F8A4291443771CFFBC0B5BC
:10518000A5DBB5E95BC25639F111F159A4823F9212
:10519000D55E1CAB98AA07D8015B8312BE8531246B
:1051A000C37D0C55745DBE72FEB1DE80A706DC9B2C
:1051B00074F19BC1C1699BE48647BEEFC69DC10FD8
:1051C000CCA10C246F2CE92DAA84744ADCA9B05C14
:1051D000DA88F97652513E986DC631A8C82703B0D7
:1051E000C77F59BFF30BE0C64791A7D55163CA06E5
:1051F00067292914850AB72738211B2EFC6D2C4DF1
:10520000130D385354730A65BB0A6A762EC9C281DE
:10521000852C7292A1E8BFA24B661AA8708B4BC274
:10522000A3516CC719E892D1240699D685350EF49E
:1052300070A06A1016C1A419086C371E4C77482755
:10524000B5BCB034B30C1C394AAAD84E4FCA9C5BCB
:10525000F36F2E68EE828F746F63A5781478C8841C
:105260000802C78CFAFFBE90EB6C50A4F7A3F9BEFE
:10527000F27871C60000000022AE28D7982F8A422B
:10528000CD65EF23914437712F3B4DECCFFBC0B57B
:10529000BCDB8981A5DBB5E938B548F35BC256397B
:1052A00019D005B6F111F1599B4F19AFA4823F9265
:1052B00018816DDAD55E1CAB420203A398AA07D809
:1052C000BE6F7045015B83128CB2E44EBE85312403
:1052D000E2B4FFD5C37D0C556F897BF2745DBE725D
:1052E000B196163BFEB1DE803512C725A706DC9BC2
:1052F000942669CF74F19BC1D24AF19EC1699BE4A7
:10530000E3254F388647BEEFB5D58C8BC69DC10FC0
:10531000659CAC77CCA10C2475022B596F2CE92D20
:1053200083E4A66EAA84744AD4FB41BDDCA9B05CB8
:10533000B5531183DA88F976ABDF66EE52513E98A9
:105340001032B42D6DC631A83F21FB98C82703B099
:10535000E40EEFBEC77F59BFC28FA83DF30BE0C676
:1053600025A70A934791A7D56F8203E05163CA0628
:10537000706E0E0A67292914FC2FD246850AB727BA
:1053800026C9265C38211B2EED2AC45AFC6D2C4DF3
:10539000DFB3959D130D3853DE63AF8B54730A65ED
:1053A000A8B2773CBB0A6A76E6AEED472EC9C28149
:1053B0003B358214852C72926403F14CA1E8BFA2A4
:1053C000013042BC4B661AA89197F8D0708B4BC243
:1053D00030BE5406A3516CC71852EFD619E892D1CB
:1053E00010A96555240699D62A20715785350EF4E3
:1053F000B8D1BB3270A06A10C8D0D2B816C1A419F7
:1054000053AB4151086C371E99EB8EDF4C77482720
:10541000A8489BE1B5BCB034635AC9C5B30C1C396C
:10542000CB8A41E34AAAD84E73E363774FCA9C5BA9
:10543000A3B8B2D6F36F2E68FCB2EF5DEE828F7424
:10544000602F17436F63A57872ABF0A11478C884FE
:10545000EC39641A0802C78C281E6323FAFFBE9039
:10546000E9BD82DEEB6C50A41579C6B2F7A3F9BE94
:105470002B5372E3F27871C69C6126EACE3E27CAAE
:1054800007C2C021C7B886D11EEBE0CDD67DDAEACF
:1054900078D16EEE7F4F7DF5BA6F1772AA67F0066E
:1054A000A698C8A2C57D630AAE0DF9BE04983F1147
:1054B0001B471C13350B711B847D0423F577DB28F8
:1054C0009324C7407BABCA32BCBEC9150ABE9E3C02
:1054D0004C0D109CC4671D43B6423ECBBED4C54C98
:1054E0002A7E65FC9C297F59ECFAD63AAB6FCB5FDC
:1054F0001758474A8C19446C657870616E64203384
:10550000322D62797465206B657870616E6420312C
:10551000362D62797465206BEDD3F55C1A631258F1
:10552000D69CF7A2DEF9DE140000000000000000A7
:1055300000000000000000101B132C0AA3E59CEDE6
:10554000A72963085D210621EBFFFFFFFFFFFFFF97
:10555000FFFFFFFFFFFFFFFF0F000000A3785913BD
:10556000CA4DEB75ABD841414D0A700098E8797788
:105570007940C78C73FE6F2BEE6C03521AD5258FC2
:10558000602D56C9B2A7259560C72C695CDCD6FD95
:1055900031E2A4C0FE536ECDD336692158666666EB
:1055A000666666666666666666666666666666669B
:1055B0006666666666666666666666660100000022
:1055C00000000000000000000000000000000000DB
:1055D000000000000000000000000000A3DDB7A5EF
:1055E000B38ADE6DF5525177809FF0207DE3AB6486
:1055F0008E4EEA6665768BD70F5F876759F1B226C4
:10560000949BD6EB56B183829A14E00030D1F3EE2E
:10561000F2808E19E7FCDF56DCD90624B0A00E4AD2
:10562000271BEEC478E42FAD0618432FA7D7FB3D08
:1056300099004D2B0BDFC14F8024832B800040004D
:10564000200010000800040002000100000080009B
:1056500000004000000020000000100000000800D2
:1056600000000400000002000000010000800000B3
:1056700000400000002000000010000000080000B2
:105680000004000000020000000100008000000093
:105690004000000020000000100000000800000092
:1056A0000400000002000000010000008000000073
:1056B00000000000000000000000000000000000EA
:1056C00000000000000000000000000000000000DA
:1056D00000000000000000000000000000000000CA
:1056E00000000000000000000000000000000000BA
:1056F000000000000000000000000000636363621F
:10570000636363626363636263636362C998989B64
:10571000AAFBFBF9C998989BAAFBFBF95034979018
:10572000FACF6C693357F4F299AC0F0B7BDA06EEC3
:1057300081156A87B2429E752BEE917E882B2E7F53
:10574000093E44F8BB7CDA8D90924BF3854B61ECBB
:105750008C7525143709FF99A79BB46A87177521A3
:105760000B6250353C6BAFAC9BF01BC63303F90E9C
:105770003861A93B040A06979FFA1D51E2D8D4B1BB
:10578000DAB97D8ADEB37B1D4149664CCB5BEFB451
:1057900011E2923ECF51E9238E188F6F0302010070
:1057A000070605040B0A09080F0E0D0CFD74AAD696
:1057B000FA72AFD2F178A6DAFE76ABD60BCF92B6FC
:1057C000F1BD3D6400C59BBEFEB330684E74FFB6AC
:1057D000BFC9C2D2BF0C596C41BF6904BCF7F747BF
:1057E000033E3595BC326CF9FD8D05FDE8A3AA3C5E
:1057F000EB9D9FA957AFF350AA22F6AD7D0F395EFE
:105800009692A6F7C13D55A76B1FA30A1A70F9140B
:105810008CE25FE34DDF0A4426C0A94E358743473B
:10582000B9651CA4F4BA16E0D27ABFAED13299544D
:10583000685785F09CED93104E972CBE7F1D111379
:10584000174A94E38BA707F3C5302B4D00000000E7
:105850000000000001000000FFFFFFFF010000004A
:10586000FFFFFFFF0000000000000000000000003C
:105870000000000000000000010000000000000027
:10588000010000000100000001000000AC58010808
:10589000000000209C06000034820008FC5B010828
:1058A0009C06002074B90000EAB0000813F3EF145E
:1058B00008B1F79208840E2707180AE92301081196
:1058C00024010829041AB50C180A212F0108C92E31
:1058D0000108E504180B75260108912701086125C8
:1058E0002419081AED241A4D041EE92A0108090496
:1058F0003C912B015413E9B51C08E1B36412B64C7A
:10590000088FB7081AB7041399B41B0889101A5DD9
:10591000081AE5101AA9281AFF101B2FB82812B26E
:105920001B086F041A350C41131201320216407025
:105930002F10EA10090201020301090229130101D3
:1059400025C0320904330203150921110114012273
:10595000201607058103402D0107050107100804E3
:105960000309041003531255124E1256124F1254CB
:10597000027345140C034312311A300202774203BA
:10598000831A0322DF1B20E3041365011B20E704B5
:105990001AA40C1AB60441136C023320FF13BDD7AE
:1059A0001B08A1041369D882081A55101A5904C19A
:1059B00013CF8F1408F59F1408CD9E1408FD921480
:1059C0000851D31C08E5EB04190C1325EC14087DD1
:1059D000911B083504780C55180108291B01089DF6
:1059E0001A01409EB5190108ED101351F71B0881EB
:1059F0000441131DBA1B08854C0114180AC9210162
:105A000008051D010819608F87340108A91F441378
:105A10005DEA1C08F9C17C1AC2C019081A0D041AE3
:105A20009D0413ADE91B0889041A95041E79100121
:105A300008A1081AF12C1A3D441AA198138DC91B0C
:105A400008E9141B6DF6B41ACE28191C1E710F013B
:105A500008F5141AB9D01AC5041AD104811AC5540C
:105A60001AED041A51680132021D0113C4322320B9
:105A7000031404A5E68C08B3F760138DE1140859EC
:105A8000E214085DDF1B083108398812E31B08B1F6
:105A9000041A990441180AA5370108F93601086962
:105AA000D413A5C0140815F32A086E1B05E4D819F1
:105AB000041BB9E5F019041A39041AAD04291C189D
:105AC0000A2D2201081923010849341A290C1A1B2E
:105AD0000C291813D9D11B08BD041AA9044BD9D21B
:105AE0002C1B91BB101AFA3C12F91408D26434052D
:105AF00001505AFFD01907E329021349B81F08E5DE
:105B00000F0108D5081A7D04100BB91601087D1580
:105B1000010859E91B086D040110294A1B99D36C2F
:105B20001D1E0108A13813E9D91F08B52F01085F10
:105B3000041A61041A63041A5D041365B11408E1C0
:105B4000FC1F08250601080D041B0907C419081AC3
:105B500019081EE1050108D10C1A01041AF104010B
:105B60001259B0012F323C233F12280D43313030FF
:105B700042414243444546474BF26413C4052A2040
:105B800004811AE3AC1341DD140879EA1408ADDA94
:105B90008C08C9D6F81AF02829040114130C062A17
:105BA0002004811329B21F08010201085104173D86
:105BB000010108B5C28C0851C44C415280599DE086
:105BC0003A48494A4B4C4D4E4F50515253545556FA
:105BD0005758595A6162636465666768696A6B6C95
:105BE0006D6E6F707172737475767778797A303103
:0C5BF00032333435363738392B2F0000A3
:04000005080081313D
:00000001FF
